:020000040800F2
:10000000F0FF00105DE10508F5EA0008C5A7040847
:10001000FDE10508FDE10508FDE10508000000001F
:10002000000000000000000000000000F1EA0008ED
:10003000EDEA000800000000E9EA0008916B0408FE
:10004000FDE10508FDE10508FDE10508FDE1050804
:10005000FDE10508FDE105081DBE040849BF0408CF
:100060000DBF0408D1BE040895BE040851B00508B0
:1000700041B0050831B0050821B005080DB00508EC
:10008000F9AF0508E5AF0508FDE10508FDE1050844
:10009000FDE10508FDE10508FDE1050859BE04087C
:1000A000F95A0408795B0408E95A04089D5B0408BE
:1000B0006D5B04085D5B04084D5B040811D1050805
:1000C00019D1050805D105080DD10508FDE1050880
:1000D000FDE10508A16F0408E56E0408296E040817
:1000E000E1BD0408FDE105083D020108D95A0408F4
:1000F000095B0408C95A04082D5B0408D1AF050840
:10010000FDE10508FDE105083D5B0408FDE105088A
:100110006D6D0408B16C040851E003083DE003086C
:10012000BDAF0508A9AF050895AF050881AF050863
:100130006DAF0508FDE10508FDE10508FDE10508D5
:10014000FDE10508FDE10508FDE105087DE4000885
:1001500059AF050845AF050831AF0508F56B040830
:10016000F9D0050801D10508FDE10508FDE1050804
:10017000FDE10508FDE10508FDE10508FDE10508D3
:08018000FDE10508FDE10508A1
:080188000CDD05000100000080
:100190000E0201000200000074460020D446002038
:1001A0000000000010090008130201000400000014
:1001B000F4220020D84600200000000012090008A8
:1001C0000D1001006400000028450020DC460020DE
:1001D00000000000C10304080400080080000000C3
:1001E000684400204047002000000000000000009C
:1001F000FB0101000100000000440020C047002076
:1002000000000000E1640508FC0101000900000095
:10021000CC420020C447002000000000F164050823
:10022000F701010006000000C0420020D047002076
:100230000000000016090008F90101000400000098
:10024000BC420020D847002000000000E93F04081D
:100250000A8001002800000094420020DC470020B2
:10026000000000006D040208160215003F000000A7
:100270001C2B00200448002000000000BD6505087C
:100280003400010010000000C0410020444800205C
:1002900000000000A5930208110201000800000000
:1002A0009841002054480020000000001C0900086C
:1002B0001212010004000000904100205C48002060
:1002C000000000002409000818200100320000008E
:1002D0005C41002060480020000000002D660508F9
:1002E000061001001C000000002B00209448002094
:1002F000000000000D650508FD010100210000005F
:100300006C400020B048002000000000433F04087B
:100310001220010011000000EC3D0020D448002014
:100320000000000028090008000201000B00000086
:10033000283B0020E848002000000000E9540508A0
:10034000FF11010006000000D43A0020F44800200C
:1003500000000000A1540508081203000F0000006F
:10036000E03A0020FC48002000000000F15405089D
:10037000FA01010003000000A03400200C49002015
:1003800000000000CD540508020201000300000037
:100390006C32002010490020000000000000000026
:1003A0000C020100040000004C320020144900201F
:1003B00000000000BD540508FE010100140000000B
:1003C000D032002018490020000000002554050804
:1003D000F581010068000000687A00203480002068
:1003E00000000000B38E010823200100100000006F
:1003F000007C00209C800020000000008105020895
:10040000FD07010076000000BC7F0020AC800020CA
:1004100000000000AD740108261001000E0000006D
:100420003481002024810020000000004D130108C9
:100430000B3001001A000000A07900207481002018
:10044000000000003C0900081F30010024000000EB
:100450006879002090810020000000005809000801
:100460000502010004000000C87B0020B4810020C8
:10047000000000007C090008030101000A000000E0
:10048000E8780020B881002000000000390F010842
:10049000010101000400000048930020809B00201F
:1004A0000000000000000000000101000400000046
:1004B00040930020849B0020000000008009000879
:1004C00002010100030000003C930020889B0020F3
:1004D0000000000065D20308220201001C01000098
:1004E000189900208C9B002000000000756505080D
:1004F0000C200600CC00000004970020A89C0020DF
:100500000000000029D20308010201000B000000D6
:1005100054930020749D002000000000D954050869
:100520001B02010010000000AC960020809D0020FE
:10053000000000002D5505081B1001000C000000F4
:100540004C830020909D0020000000004D8F01088A
:1005500021020100F0000000CC8100209C9D0020C1
:1005600000000000198E0108231201001000000095
:10057000D89700208C9E002000000000840900080D
:10058000371001002E0000001C9600209C9E0020C9
:100590000000000094090008161001000600000089
:1005A000B8930020CC9E002000000000C209000883
:1005B0002F100100220000005C9B0020D49E002030
:1005C00000000000C80900081E000100090000002A
:1005D00078930020F89E002000000000EA0900083F
:1005E000051001000600000094930020049F0020E5
:1005F00000000000F40900082C00040010000000B6
:100600001CAE00200CAE00200000000045230208B4
:100610002B0012002400000050AE00202CAE002061
:1006200000000000192302082920140078000000AF
:100630007CAC002074AE0020000000000000000030
:10064000F62101000C0000006CAA0020ECAE002096
:1006500000000000FC0900081C0202001C00000051
:100660005CAB00203CAF002000000000456705089F
:1006700028200100180000002CAA002058AF0020FC
:1006800000000000B12C020814000100040000006A
:1006900014AA002070AF002000000000080A000823
:1006A000012001000C00000044A1002074AF0020D4
:1006B000000000000C0A00080EF003009E0100007C
:1006C0002C9F002080AF002000000000B9880208A5
:1006D000130001000400000048A6002020B1002003
:1006E00000000000180A00081900010005000000C1
:1006F00030B700204CB80020000000001C0A0008A1
:100700001A0001000E000000B8B6002054B8002006
:1007100000000000220A0008203201000A00000048
:1007200084B5002064B8002000000000958802080D
:1007300015001000700000001CB3002070B80020ED
:1007400000000000000000002A0008006000000017
:1007500078B70020E0B80020000000006D88020893
:100760000300010001000000D8BE00200CBF0020E3
:100770000000000000000000031201003D00000026
:1007800080BE002010BF002000000000300A0008DA
:1007900025201E002C010000E4BB002050BF0020DB
:1007A0000000000000000000101001000200000026
:1007B00078BB00207CC00020000000006E0A00080A
:1007C000F821010006000000C0BB002080C000200E
:1007D00000000000700A0008020001000C00000088
:1007E000E8C100207CC200200000000000000000E2
:1007F00029020100400000001CC1002088C2002026
:1008000000000000760A00080A020100140000003F
:1008100090C00020E8C200200000000091D303082F
:10082000280204000400000018C70020ECC80020C3
:1008300000000000295505082702040004000000FC
:1008400014C70020F0C80020000000001D55050856
:100850001F020800100000005CC40020F4C8002043
:1008600000000000595405081A0201003C00000075
:1008700020C4002004C9002000000000B96605085B
:10088000381001000100000014C3002040C90020FE
:1008900000000000B60A0008270001000400000064
:1008A000C8C90020CCC9002000000000B80A000818
:1008B000100201000100000034E8002030E80020B0
:1008C00000000000BC0A000807020100020000004E
:1008D00018E8002038E8002000000000BE0A0008E8
:1008E0001D02020006000000F8E700203CE800209E
:1008F0000000000000000000060203000C000000E1
:1009000000E8002044F1002000000000A166050876
:1009100000000000010029010000C40914250000A6
:1009200001010101FFFFFFFF000000010000054D74
:10093000463454000008000200000000AE014A01E5
:100940005E012C0164010100000001000A019A010E
:10095000001E0A000002000000000000000100006C
:10096000000500000102030000000000000000007C
:1009700000000000000000000080070000000000F0
:1009800096000000000000000000000000000000D1
:100990000000000020003200C800D00796001400BC
:1009A000320028004C0440060005500014000F00DF
:1009B000080064000100010005000A000000F401C5
:1009C0009600C409000019000000000000000000AB
:1009D0000000000000000000000000000000000017
:1009E0000000000000000000000000050100000001
:1009F00000000000200001010000000000000000D5
:100A0000010000000202000003000023E80364006C
:100A1000040A000114001E004804443000002801AC
:100A200000007E05EA05B4053200E803D0070000A7
:100A300000000000000000000000000000000000B6
:100A400000000000000000000000000000000000A6
:100A50000000000000000000000000000000000096
:100A60000000000000000000000000000100000580
:100A70000101F4011400000000000000000000006B
:100A80000000000000000000000000000000000066
:100A90000000000000000000000000000000000056
:100AA0000000000000000000000000000000000046
:100AB0000000000000000000200300000000003CD7
:100AC0000403090412010002EF02014083045632BC
:100AD00000020102030100001201000202020040B4
:100AE000830440570002010203010000006002403D
:100AF000106002400000000000000000000B000039
:100B00000000000000000000000000000060024043
:100B1000286002400100000000000000060C0000F8
:100B20000000000000000000000000000060024023
:100B3000406002400200000000000000100D0000B4
:100B40000000000000000000000000000060024003
:100B5000586002400300000000000000160E000074
:100B600000000000000000000000000000600240E3
:100B7000706002400400000000000000200F000030
:100B800000000000000000000000000000600240C3
:100B900088600240050000000000000026100000F0
:100BA00000000000000000000000000000600240A3
:100BB000A0600240060000000000000030110000AC
:100BC0000000000000000000000000000060024083
:100BD000B86002400700000000000000362F00004F
:100BE000000000000000000000000000006402405F
:100BF0001064024000000000000000000038000007
:100C0000000000000000000000000000006402403E
:100C100028640240010000000000000006390000C6
:100C2000000000000000000000000000006402401E
:100C3000406402400200000000000000103A000082
:100C400000000000000000000000000000640240FE
:100C5000586402400300000000000000163B000042
:100C600000000000000000000000000000640240DE
:100C7000706402400400000000000000203C0000FE
:100C800000000000000000000000000000640240BE
:100C900088640240050000000000000026440000B7
:100CA000000000000000000000000000006402409E
:100CB000A064024006000000000000003045000073
:100CC000000000000000000000000000006402407E
:100CD000B864024007000000000000003646000033
:100CE00000000000000000000000000008000000FC
:100CF0007D00000001820008FD810008F9810008E4
:100D0000ED810008E9810008F5810008F181000803
:100D1000FDAC00087D86000809850008AD8C000840
:100D2000298D0008D18E000855830008198300081A
:100D300011830008010000000000803FD932010843
:100D4000DD37010855330108B1080108950A01088B
:100D5000C1080108DD0801088908010879080108AF
:100D6000000000000000000009022000010104C092
:100D70003209040000020806500507058102400000
:100D8000000705010240000009026400030100C0E1
:100D900032090400000103000000092111010001D3
:100DA0002236000705830309000A080B010202022C
:100DB00001000904010001020201000524001001E4
:100DC000052401000204240202052406010207058D
:100DD00082030800FF09040200020A000000070560
:100DE00001024000000705810240000009024300A3
:100DF000020100C0320904000001020201000524C2
:100E0000001001052401000104240202052406004B
:100E100001070582030800FF09040100020A00001F
:100E200000070501024000000705810240000000A4
:100E3000FF00000000FF0000000000000000AA55B5
:100E40000701000001AA5505010000007EFF08000F
:100E500030200608FF1FFF1F05010905A101A100A1
:100E600005010930093109320933093509340936D8
:100E700009371581257F7508950881020509190133
:100E8000290815002501950875018102C0C00000E0
:100E900009022200010100E03209040000010301FF
:100EA0000200092111010001223600070583030910
:100EB000000A000000000000010203040102030414
:100EC000060708092D202D2D202D2D2D2D202D2D0F
:100ED0002D2D0000000000000000000000000000B8
:100EE000000000AA550B010000AA5505010000AA48
:100EF000550902000000AA5503009F0001000000F0
:100F0000C01200006C81002000000000448100201D
:100F10000000000024A40608A0A3060800000000AA
:100F2000EDD20308A08601000400000000000000CC
:100F300000000000000000000000000000000000B1
:100F400000000000000000000000000000000000A1
:100F50000000000024A406082CA4060800000000DD
:100F600051510408E80300000400000000000000E4
:100F70000000000000000000000000000000000071
:100F80000000000000000000000000000000000061
:100F90000000000034A4060800000000000000006B
:100FA000F54303087D000000FF0000000000000082
:100FB0000000000000000000000000000000000031
:100FC0000000000000000000000000000000000021
:100FD000000000006023070800000000000000007F
:100FE000855303087D000000FF00000000000000A2
:100FF00000000000000000000000000000000000F1
:1010000000000000000000000000000000000000E0
:10101000000000004CB806080000000000000000BE
:10102000B59B03087D000000FF00000000000000E9
:1010300000000000000000000000000000000000B0
:1010400000000000000000000000000000000000A0
:10105000000000003CA406080000000000000000A2
:1010600081470408E80300000300000000000000BE
:101070000000000000000000000000000000000070
:101080000000000000000000000000000000000060
:101090000000000040A4060800000000000000005E
:1010A000E504030810270000030000000000000012
:1010B0000000000000000000000000000000000030
:1010C0000000000000000000000000000000000020
:1010D00000000000681F070800000000312002081F
:1010E00029A804085F760000050000000000000049
:1010F00000000000000000000000000000000000F0
:1011000000000000000000000000000000000000DF
:101110000000000004230708000000000000000099
:101120004DC8040810270000010000000000000066
:1011300000000000000000000000000000000000AF
:10114000000000000000000000000000000000009F
:10115000000000004CA40608000000000000000091
:10116000D93D0408E803000005000000000000006D
:10117000000000000000000000000000000000006F
:10118000000000000000000000000000000000005F
:101190000000000058A40608000000000000000045
:1011A000D1D50308204E000003000000000000001D
:1011B000000000000000000000000000000000002F
:1011C000000000000000000000000000000000001F
:1011D0000000000068A406080000000000000000F5
:1011E000CDD30308204E00000300000000000000E3
:1011F00000000000000000000000000000000000EF
:1012000000000000000000000000000000000000DE
:101210000000000078A406080000000000000000A4
:10122000954D0408400D030003000000000000007D
:1012300000000000000000000000000000000000AE
:10124000000000000000000000000000000000009E
:101250000000000088A40608000000000000000054
:10126000B50704081027000001000000000000007E
:10127000000000000000000000000000000000006E
:10128000000000000000000000000000000000005E
:1012900000000000CCA306080000000000000000D1
:1012A0007D9B0108102700000300000000000000E3
:1012B000000000000000000000000000000000002E
:1012C000000000000000000000000000000000001E
:1012D0000000000090A406080000000000000000CC
:1012E000BD570208A08601000100000000000000B8
:1012F00000000000000000000000000000000000EE
:1013000000000000000000000000000000000000DD
:101310000000000098A40608000000000000000083
:101320000946040850C3000001000000000000004E
:1013300000000000000000000000000000000000AD
:10134000000000000000000000000000000000009D
:1013500000000000A0A4060800000000000000003B
:10136000F5410408A8610000010000000000000031
:10137000000000000000000000000000000000006D
:10138000000000000000000000000000000000005D
:1013900000000000ACA406080000000000000000EF
:1013A0005DF90108A08601000100000000000000B6
:1013B000000000000000000000000000000000002D
:1013C000000000000000000000000000000000001D
:1013D00000000000B8A406080000000000000000A3
:1013E000DD740408A00F00000100000000000000F0
:1013F00000000000000000000000000000000000ED
:1014000000000000000000000000000000000000DC
:1014100000000000C4A40608000000000000000056
:101420005DF401081027000001000000000000002A
:1014300000000000000000000000000000000000AC
:10144000000000000000000000000000000000009C
:1014500000000000D0A4060800000000000000000A
:10146000ADD001081A41000001000000000000009A
:10147000000000000000000000000000000000006C
:10148000000000000000000000000000000000005C
:1014900000000000D4A406080000000000000000C6
:1014A000710F01081027000001000000000000007B
:1014B000000000000000000000000000000000002C
:1014C000000000000000000000000000000000001C
:1014D00000000000B4A306080000000000000000A7
:1014E000A538020850C30000010000000000000001
:1014F00000000000000000000000000000000000EC
:1015000000000000000000000000000000000000DB
:1015100000000000E0A40608000000000000000039
:1015200031170108400D030000000000000000001A
:1015300000000000000000000000000000000000AB
:10154000000000000000000000000000000000009B
:1015500000000000E8A406080000000000000000F1
:1015600029D30308400D0300000000000000000024
:10157000000000000000000000000000000000006B
:10158000000000000000000000000000000000005B
:1015900000000000F0A406080000000000000000A9
:1015A00001DF010850C3000003000000000000003C
:1015B000000000000000000000000000000000002B
:1015C000000000000000000000000000000000001B
:1015D00000000000FCA4060800000000000000005D
:1015E0006DE4030840420F0000000000000000000E
:1015F00000000000000000000000000000000000EB
:1016000000000000000000000000000000000000DA
:101610000000000008A5060800000000000000000F
:101620002DDA030850C30000000000000000000095
:1016300000000000000000000000000000000000AA
:10164000000000000000000000000000000000009A
:10165000000000000100000000000100E0010101A5
:10166000418001080000000000000000542206082C
:10167000FFFFFFFF0801FF0101FF0000FFFFFFFF69
:1016800045ED01080000000000000000B82A06082F
:1016900069F001080000000000000000702A060840
:1016A0002D202D2D202D2D2D2D202D2D2D00000018
:1016B000000000000000000000000000000000002A
:1016C0000000000000000000000000002C2A0608B6
:1016D000747B00209CFF2C0100000000C89A0020B1
:1016E000E0150C1700000000D09700200200000059
:1016F000642A06083093002088136F170100000049
:101700003293002088136F1700000000F645002078
:101710000000000000000000F44500200000000070
:1017200000000000F2450020000000000000000062
:10173000F04500200000000000000000EE45002001
:101740000000000000000000EC4500200000000048
:1017500000000000C805002000000000000000009C
:10176000B892002003000000542B060828930020A4
:1017700088136F1701000000BE7B002088136F17CD
:1017800000000000FD8001080000000000000000D3
:10179000642B0608D197002001000000B82B060832
:1017A000C07B002001000000C42B0608B67B00208F
:1017B00002000000CC2B0608000000000000000022
:1017C00000000000D82B0608E5800108000000009A
:1017D00000000000742C060800000000000000005B
:1017E00000000000C82C06080000000000000000F7
:1017F00000000000382D060834930020020000008D
:10180000702D0608BA7B0020E0150C1700000000C0
:10181000ECA2002040A30020D6010100000000003F
:101820000000000019240208DCA6002000000000CF
:1018300000000000000000007443060800000000E3
:1018400000000000000000002C440608000000001A
:101850000000000000000000D8430608FF00000060
:10186000FFFFFFFF21290208000000000000000028
:101870000443060801000000FA0000000100000017
:101880000100000001000000000101010000000053
:101890003EA100200000F401010000003CA1002056
:1018A0000000F401010000003AA100200000F40152
:1018B0000100000038A100200000F4010100000038
:1018C00036A100200000F4010100000034A1002036
:1018D0000000F4010100000032A100200000F4012A
:1018E00001000000BD0202088102020800000000A1
:1018F000842F060822A100200532010030A100201B
:101900006400F401010000002EA100206400C4095D
:101910000100000020A10020E803D0070100000022
:101920001EA10020E803D007010000001CA1002038
:10193000E803D007010000001AA100201E00B80B28
:101940000100000028A1002005000F000100000098
:101950002AA1002003000A000100000018A10020B5
:101960001E00F401010000002CA100200200000074
:101970001030060816A100201400640001000000C9
:1019800024A100203200E8030100000014A100207F
:101990000000C80001000000EDA0002000C8010008
:1019A000ECA0002000500100EBA00020005A010034
:1019B000E9A00020020000001C30060898AF0608CD
:1019C000A0AF0608B24500200100C40900000000D5
:1019D000B04500200100C40900000000AE45002011
:1019E0000100C40900000000AC4500200100C4094A
:1019F00000000000A84500200100C409000000000C
:101A0000AA4500200100C40900000000A6450020EE
:101A10000100C40900000000A44500200100C40921
:101A2000000000007393002000C8010072930020A2
:101A300000C80100709300200000FFFF0A000000B2
:101A40006E9300200100C800010000006C9300208C
:101A500032003075320000006A9300207EFF1400CF
:101A6000050000006893002005002C01050000001F
:101A700067930020055A05006493002000FF0100D1
:101A80006693002002000000841000206293002072
:101A900003000000382706086393002000FF0100C0
:101AA0006593002002000000841000206193002054
:101AB000030000003827060811020208A1010208ED
:101AC000000000002830060854A10020EE02CA08D9
:101AD0000100000052A1002000C8010064000000C5
:101AE00051A1002000C801006400000050A10020A6
:101AF00002000000343106084E9300200000803EB2
:101B0000050000004C93002080C1803E05000000CD
:101B1000469300200083007D0500000044930020D0
:101B200080C1803E050000003F93002000FF0100BF
:101B3000389300206400F401010000003693002077
:101B40000400000040310608359300200200000028
:101B5000543106081B9F00200D000000603106086C
:101B6000189F002000640100169F002032001027FB
:101B70000A000000149F00200D00000060310608DC
:101B8000139F00200D00000060310608129F002006
:101B9000020000009831060800000000000000006C
:101BA00000000000A43106085AA100203E000000F9
:101BB000DC31060858A100200100FF7F0100000071
:101BC00057A1002002000000D83206081D9F002007
:101BD00003000000E83206081C9F002003000000FC
:101BE000E8320608DAA00020000A0100D8A0002090
:101BF0000000E80301000000D6A000200000E80378
:101C000001000000D4A000200000E8030100000053
:101C1000D2A000200000E80301000000CAA00020BC
:101C20000000E80301000000D0A000200000E8034D
:101C300001000000CEA000200000E8030100000029
:101C4000CCA0002000140100E8A000200200000049
:101C5000F8320608E6A000200000F40101000000B0
:101C6000E4A000200000F40101000000E2A0002038
:101C70000000F40101000000E0A000200000F401D9
:101C800001000000DEA000200000A00F0100000005
:101C9000DCA000200000A00F0100000001A1002036
:101CA0001964010000A100200200000004330608AE
:101CB000FEA00020E803D0070A000000FCA00020DE
:101CC000006401000A000000F1A00020006401008F
:101CD000F0A0002000640100F8A0002000640100D2
:101CE0000A000000F7A00020006401000A000000C4
:101CF000F6A00020006401000A000000FBA0002004
:101D000000FF01000A000000FAA0002000FF01000F
:101D10000A000000F9A0002000FF01000A000000F6
:101D2000F5A0002001FF01000A000000F4A000203F
:101D300001FF01000A000000F3A0002001FF0100E4
:101D40000A000000269F00200000F40101000000AE
:101D5000249F00200000A00F01000000229F00200F
:101D60000000A00F01000000209F00200000A00F35
:101D7000010000001E9F00200000A00F01000000D5
:101D80005DA6002000C801005CA6002000640100E0
:101D90005BA60020006401005AA600200064010038
:101DA00059A600200064010058A60020FF08010089
:101DB00057A600200164010009010208CD000208B5
:101DC000000000001033060860A600200132010068
:101DD0005FA6002001000000803306085EA60020F8
:101DE000040000008833060856A6002000640100A5
:101DF00054A600201400E8030100000052A60020B1
:101E0000E80330750A00000050A6002000C8010059
:101E10004FA6002000C801004EA6002000C8010007
:101E20004DA600200032010062A60020004B0100F8
:101E300061A60020040000009C3306084CA6002088
:101E4000006401000A00000070A600200000D00716
:101E5000010000006BA6002000C801006AA6002057
:101E600000C8010069A6002000C801006EA600207D
:101E70000000D0070100000068A6002000C8010093
:101E800067A6002000C8010066A6002000C8010067
:101E90006CA600200000D0070100000065A600200D
:101EA00000C8010064A6002000C8010063A600204D
:101EB00000C80100F5FE0108DDFE01080000000079
:101EC000B03306080F9F0020005A01000E9F00202B
:101ED00000C801000C9F0020E803D00701000000AB
:101EE0000000000000000000592402084C340608DD
:101EF0004D4154454B4634303554450060930020E5
:101F0000000301005F9300200003010059830108D2
:101F10000D83010800000000A0340608CD820108EE
:101F200085820108000000003C35060875FE0108A6
:101F300031D8010800000000BC350608509300208D
:101F400001030100990302086D030208000000006C
:101F50001439060809820108BD810108000000004B
:101F60008439060805FF0108252502080000000045
:101F7000203A0608D52B0208C5030208000000001D
:101F8000C83A060845FF01080000000000000000F4
:101F9000543B0608FDFF0108A5FF010800000000F2
:101FA000B83B060891000208550002080000000036
:101FB000603C0608AD7F02084501020800000000F1
:101FC000EC3C060813A10020010601007DFF01087A
:101FD00055FF010800000000E83D0608E57E020804
:101FE000D525020800000000583E0608F57F0208CB
:101FF0009926020800000000A83F060812A1002050
:1020000001030100B5FE01088DFE0108000000007B
:102010007C4006084D80020800000000000000001F
:10202000E0400608558201085DCF0108000000006D
:1020300060410608000000000000000000000000F1
:10204000EC4106087901020811270208000000008F
:102050005C420608FFFFFFFF0000803F0000000019
:102060000000000000000000000000000000000070
:102070000000000000000000000000000000000060
:102080000000803F00000000000000000000000091
:102090000000803F00000000000000000000000081
:1020A0000000803F00000000000000000000000071
:1020B000010000000000FA430000FA430000803FE6
:1020C000C509040800000000000000000000000036
:1020D000FFFFFFFFFF00000000000000D8C200204B
:1020E0000800000000000000C8C200200800000036
:1020F00031320108A5090108C931010800000000BA
:1021000075080108B13A010819310108652D010867
:1021100000000000000000003508010811820008DE
:1021200005820008DD8B00084D8C0008318C00080A
:10213000158C0008F98B0008E931010881090108B4
:102140001D310108000000004D080108692D01083B
:10215000ED300108C52C010800000000000000005F
:1021600041080108685E0C0002010000A00F000099
:10217000B80B00000102FFFF01000000FFFF00009C
:102180005C1F0708000008020503030000000000B0
:10219000641F070801000802050403000000000096
:1021A000D0CB06080200FE01011003000000000071
:1021B00000B3060803001402000300000000000042
:1021C0006C1F070804001F02020008000000000046
:1021D000741F070805001F0202010800000000002C
:1021E000FFFFFFFF1A0300000000000000000000D6
:1021F00000000000000000000000000000000000DF
:102200000403090412010002000000408304205767
:102210000002010203010000256F0508516F050847
:10222000156F050875550508C56E0508716E05081A
:1022300065550508CC190020D16705087D550508AE
:102240007955050871550508896905086D55050812
:1022500069550508009706084D3A0108610901080B
:102260002D3901080000000000000000C530010801
:10227000D52F010800000000000000000000000051
:10228000290801081556050809560508A16F050813
:10229000BD6F0508C1550508856F0508696F0508FC
:1022A0000000040100000000000000021000000017
:1022B000070000001F0000001C0000001F000000BD
:1022C0001E0000001F0000001E0000001F00000094
:1022D0001F0000001E0000001F0000001E00000084
:1022E0001F0000000068214CFFFF0100F401000006
:1022F000A0A0060800000000000000000102030486
:1023000006070809008002021F00000053544D20F8
:102310002020202050726F647574202020202020FF
:1023200020202020302E303101000000F81900203C
:10233000000000000000000000000000000000009D
:10234000000000000000000000000000000000008D
:10235000000000000000000000000000000000007D
:10236000000000000000000000000000000000006D
:10237000000000000000000000000000000000005D
:10238000000000000000000000000000000000004D
:082800000000000000000000D0
:1080000070B4C3080D4CE25C00F00706B24004EB0C
:10801000D004D2B20020C6F108038B4228BF0B4621
:10802000C3F108052A419840C91A40EA02004FF0FE
:10803000000614F8012FEED170BC7047981A00208A
:10804000084AD2E91C31994209D0D118013391F87C
:1080500078100170C3F30A031367012070470020F2
:10806000704700BF581A0020064AD2F87838D2F874
:108070007C28934294BF4FF400600020013B9B1A80
:1080800018447047581A0020012380F85130704777
:1080900007B501A8FFF7D4FF0028FAD09DF8040027
:1080A00003B05DF804FB044BD3E91C03984288BF7E
:1080B00003F50063181A7047581A00200120704712
:1080C000024BC3F88028C3F884187047581A002060
:1080D000024BC3F88828C3F88C187047581A002040
:1080E0007047704730B4124DD5E91C239A4286BFC1
:1080F00003F50064A21A9A1A0A44B2F5006F12D866
:10810000A1B101444A1E013810F8014FE91882421A
:1081100003F1010381F87840C3F30A03F4D16B67DC
:10812000002030BC7047022030BC70470846F8E79A
:10813000581A0020212838B50C4605D022282ED008
:10814000202813D0002038BD0029FBD0072AF9D100
:108150001A4BD3F8900893F8941893F8952893F84D
:108160009638206021716271A371EBE70029E9D094
:10817000072AE7D1114DD5F884381BB10968D5F825
:1081800080089847206821796279A379C5F890081A
:1081900085F8941885F8952885F89638D2E700294F
:1081A000D0D0022ACED1054AD2F88C38002BC9D0C3
:1081B0000988D2F888089847C4E700BF581A0020F9
:1081C000024B0020C3F89808704700BF581A0020DF
:1081D000044B00200522C3F89828C3F88C08C3F884
:1081E00084087047581A0020704700BF704700BFCE
:1081F000704700BF704700BF704700BF704700BFA7
:10820000704700BF042301480B807047880100209D
:1082100010B4074A074B92F89C08122403F1140289
:108220000C8001280CBF184610465DF8044B7047BF
:10823000581A00208C010020A0B182680D4B12B1A9
:1082400007229A7070471978DA6003294FF004000A
:108250000CBF80214FF48071C3E901111A611A75B6
:1082600098707047034B41F2E47101225A545A70DE
:10827000704700BF2C5900200378022B10D00069F2
:1082800008B9012070470C4B1B78032B0EBF0B4B1A
:1082900080B24FF6F773984294BF002001207047D8
:1082A0000549436841F650028A58B3EB422F2CBF70
:1082B00001200020704700BF2C590020F7FFFF0F5E
:1082C0000378022B14D030B4104A4368006941F699
:1082D000480402F5C2511559096841F63C042B4087
:1082E00012595B0A023801FB0030104430BC704761
:1082F000064B426841F6340141F63000595818588F
:1083000000EB410000EB5220704700BF2C590020C9
:1083100000487047801A0020034B93F8240003287C
:1083200094BF002001207047581A002010B5084C57
:10833000E26D13899907FCD513891B06F9D40A202D
:108340003EF054FA206EBDE8104042F013BA00BF70
:10835000581A0020034B93F82400003818BF01205E
:10836000704700BF581A00200D4B70B5DC6D3EF011
:108370002FFBA389054642F20F7623899B0705D57B
:108380002046FF21BDE8704052F06ABE3EF020FB5F
:10839000401BB042F1DD204643F07AFFC0B270BD11
:1083A000581A002070B505460E460924FFF7DCFF79
:1083B000FF2803D1013CF9D1012070BDFE2801D076
:1083C000022070BD064933462A46C86D002154F08C
:1083D00035F9FFF7C9FFFFF7C7FF002070BD00BFE9
:1083E000581A00202DE9F04383B040F040060C0EEF
:1083F00005460A0A080C95238DF801408DF80410F3
:108400008DF800608DF802008DF803208DF805309E
:108410000824FFF7A9FFFF2802D0013CF9D11DBBBA
:108420001E4BDC6DA3890627E84642F20F76B8F1B1
:10843000000F30D018F8015B3EF0CAFA814623895C
:108440009A0715D5ADB2A5813EF0C2FA054623893B
:10845000DB0717D5013FA389E9D10924FFF784FF82
:10846000FF2802D1013CF9D1FF2003B0BDE8F08321
:108470003EF0AEFAA0EB0900B042E0DD204643F04A
:1084800007FFEAE73EF0A4FA401BB042DFDD2046DA
:1084900043F0FEFEE1E7FF25CEE700BF581A0020BB
:1084A000F8B5184F00233B62FFF75EFFFC6D3EF00E
:1084B0008FFAA389054642F20F7623899B0710D5D0
:1084C0002046FD2152F0CCFDFFF74EFFFF2811D1D1
:1084D000FFF74AFFFF280DD10423022087F824303C
:1084E000F8BD3EF075FA401BB042E6DD204643F091
:1084F000CFFEE9E7D7F8A0387B610923002087F891
:108500002430F8BD581A00202DE9F843194C94F88E
:108510002460042E0546894690461F4608D0082E42
:1085200002D00020BDE8F883FFF7BAFF0228F8D197
:10853000206E42F019F9A37E93B969021120FFF76A
:1085400051FF98B9D4F8A038C4F800900522C4E9C6
:108550000387656084F8242063610120BDE8F88307
:1085600029461120FFF73EFF0028EBD0FFF7DEFE83
:10857000D7E700BF581A0020F8B51A4C94F8A43871
:10858000002BFBD159B301444E1E451ED4F87C2864
:10859000D4F8781815F8017F531CC3F30A038B42F3
:1085A0002CBF4FF400600020C91A22440144012965
:1085B00082F8A878C4F87C380FD101203EF044FA44
:1085C000D4F87838D4F87C188B4294BF4FF400620A
:1085D00000225B1A1344012BEFD0B542D6D1002004
:1085E000F8BD00BF581A002010B5094CD4F89838CF
:1085F000084611465BB1D4F89838052B07D1002AFC
:10860000D4F8A03803DDFFF7B7FFD4F8A03810BDC9
:10861000581A002010B590F85010002380F8503000
:1086200081B10B4CD4F8982872B1D4F89828052A57
:108630000CD13C30D4F8A038FFF79EFFD4F8A03816
:10864000012010BD0120FCE71046FAE71846F8E7C4
:10865000581A0020002280F85120DBE790F85020C3
:10866000531C0244DBB280F8503082F83C1090F882
:1086700051200AB1132B00D9CCE770472DE9F843FC
:108680004379524D002B14BF0122002285F850205F
:1086900003D185F82430BDE8F88390F8018008F113
:1086A000FF3676B2044630460F4643F0D5FE02232D
:1086B000E86585F858302378002B5BD1E478002CEE
:1086C0004CD14FF48071E86D2C6650F027FF4FF4C9
:1086D0007A703EF0B9F9286E42F04CF8EC6D4FF02C
:1086E0000A08A38942F20F764FF0FF090BE0A4F8C5
:1086F0000C903EF06DF907462389D90728D5B8F1CB
:108700000108A3890DD03EF063F907462389980735
:10871000EDD43EF05DF9C01BB042F7DD204643F0DA
:10872000B7FDE96D2A4B0A89920709D50A8912F02B
:10873000800205D1D5F8A0182A7601236961A8E73F
:10874000013BF0D12A7E85F82430531C2B76A2E71A
:108750003EF03EF9C01BB042CEDDDFE7204641F0DF
:1087600025FD04460028ACD01E23C38009213DF01E
:108770005DFEA6E706EB86063E44414696F90320D9
:1087800000203EF03DFE064630B140683EF026FE39
:10879000B36885F86C3018B9002385F864308DE72C
:1087A0000C4A431E02EB43112C3291F8446002EB59
:1087B0004313AB66002EEFD11723A1F8443051F0DC
:1087C000CBFA012385F8643078E700BF581A0020FF
:1087D000A1860100880100202DE9F04FCD4DDFF882
:1087E0006483DFF86C9384460F4616460FCD4446EB
:1087F0002DED068B0FC40FCD0FC495E807008BB08D
:1088000019F84E3C029684E80700CDE906C7042B10
:1088100000F25981DFE813F0B6015701520105005B
:10882000C6019FEDBD8ADFEDBD8ABD49C8F81C10A9
:10883000BC49BD4BBD4AC8F818100299002918BFA1
:10884000134638EE887AF5EE006A86EE87AAC8F8F5
:108850002430B74FB74B03930026DFEDB77A9FED77
:10886000B79A28EE278AF0EE679A079BB34200F08A
:108870001F81039B13F8014B039306F1010B5FFA71
:108880008BF2002C00F09181DFF8C8C2002303E0D6
:108890000133152B00F0898103EB43015D001CF8C7
:1088A0000100A042F4D14944049211F8331C00297C
:1088B00000F0838120463DF07BFB036805938246F0
:1088C00018463DF061FB9AF805103DF0B5FB90F8B5
:1088D00000E0BEF1000F40F0688109EB05002509BA
:1088E0000321013D049A059B42738D42017304F0FC
:1088F0000F0C00F23381874800EB4500808D40FA71
:108900000CF414F0010400F03B81012404FA0CF390
:10891000013B1840049255F0A9FA7E4BDFF838C2AB
:10892000049A1D44032195F834307A4D18440CEB19
:10893000C0037B619971DA715CF830009AF8082005
:1089400000F13F4101F57E0105EB912191F83810CE
:1089500001F01F054909032904FA05F400F00B8111
:10896000042900F00381022900F0FB809B88089312
:10897000B3FA83F3C3F11F03C3F3CC0100EB81010E
:1089800003F007030C6A9B000F259D4024EA0504B1
:108990000C620C6A02FA03F323430B62022308A958
:1089A00009930BF00FFBDAF80030029A002A00F06E
:1089B000A28039F8502C00EE102AB8EEC00AFCEE66
:1089C000C07A17EE901A5E4A934200F08180A2F5B9
:1089D000806293427CD002F58042934278D002F5C7
:1089E0008062934274D002F58062934270D0D9F8CD
:1089F000382250084FF6FF73B0FBF1F21A44120C04
:108A0000B0FBF2F20298002865D0B2FBF1F119F840
:108A10004E0C04288BB263D007EE902AF8EE676AFA
:108A200066EE887A29EE677A19F84D0C069900915E
:108A3000A6EEA87A019051463846C7ED027A87ED36
:108A4000037A35F007F8002E60DD7B68D8F838200F
:108A500093425DD0012E59D0D8F85020934257D080
:108A6000022E53D0D8F86820934251D0032E4DD017
:108A7000D8F8802093424BD0042E47D0D8F89820C5
:108A8000934245D0052E41D0D8F8B02093423FD034
:108A9000062E3BD0D8F8C820D31A18BF01235E4653
:108AA0000122082E3B747A7407F118077FF4DDAEBB
:108AB00024480BB0BDEC068BBDE8F08F9FED228AF9
:108AC000F0EE488AB1E69FED218AF0EE488AACE6E6
:108AD000D9F838028EE719F84E0C042819469BD1B4
:108AE00007EE901A07EE102AF8EE677AF8EE476A5A
:108AF00067EEA97A96E7B0EE4A0A049356F0ECF8CE
:108B0000FCEEC07A049B17EE901A5CE70123C6E7DF
:108B10000023C4E7D0140608ACC5A737ACC5A736F8
:108B2000C9430308D93F0408853F0308CD3F040823
:108B300048000010072B00206F12833A00007A448F
:108B40000004014014000010282930386F12033946
:108B5000502B00201C2B0020882B0020C7F814E08D
:108B600023E717494D6C2C434C64FFE614490D6B09
:108B70002C430C63FAE612490D6C2C430C64F5E6A9
:108B80007C6112E79FED0F8A0F4BC8F81830002365
:108B90000E4A069301230293C8F81C200C4BF0EEFA
:108BA000488A4EE69FED0B8AEEE70B4A084BC8F861
:108BB0001C20C8F8243000207BE70B68FFDE00BFD4
:108BC000003802406F12833AD93F0408C9430308B2
:108BD000CD3F0408000000007D42030810B5044C9E
:108BE00004480A46214609F0F1FF204610BD00BFA7
:108BF0008C2D0020D0A0060810B5044C04480A466D
:108C0000214609F0E3FF204610BD00BF8C2D002057
:108C1000DCA0060810B5044C04480A46214609F0B9
:108C2000D5FF204610BD00BF8C2D0020ECA006080B
:108C300010B5044C04480A46214609F0C7FF2046F7
:108C400010BD00BF8C2D0020F8A0060810B5044C04
:108C500004480A46214609F0B9FF204610BD00BF6E
:108C60008C2D002004A1060810B509F083FF0E4CDE
:108C700048B194F82430032B10D8237E0133DBB2A3
:108C8000072B237603D9002384F8243010BDD4F8B1
:108C9000A0386361012384F8243010BDE06D4FF4E7
:108CA000807150F03BFCE8E7581A002070B51D4C6D
:108CB00094F82430042B06460D4608D0082B20D10A
:108CC000E36983422BD0FFF7EBFB022819D1206E1A
:108CD00041F04AFD00213720FFF784FB2946172089
:108CE000FFF780FBA8B9A37E6BB971021920FFF7CB
:108CF00079FB70B90823C4E9076584F824300220A1
:108D000070BD012070BD31461920FFF76BFB0028B4
:108D1000F0D0FFF70BFBFFF7A7FF032070BD022089
:108D200070BD00BF581A00202DE9F04F95B0CDE975
:108D30000223664C0646884694F82430042B0DD056
:108D4000082B07D1E369B34200F0BB80FFF7A8FB13
:108D50000228F1D0012015B0BDE8F08F206E41F05F
:108D600003FDA37E002B40F0928071021820FFF7D4
:108D700039FB002840F09F8094F82450FFF7F4FA64
:108D8000082D0CBFFC21FE21D4F85C9001913DF030
:108D90001FFEB9F80C300199054642F20F77B9F879
:108DA0000830980745D5484652F05AF994F864308F
:108DB000002B4CD005A80AF0EFFE94F86C20E36D70
:108DC000A16ECDF81C8052060C33486805920693BC
:108DD00040220023CDE90C3308920F934FF48062B8
:108DE0000A930E934FF400730B9209930AF012FF4B
:108DF000A36E05A958680AF0E1FEA36EE26D5968FA
:108E00000B6843F001030B6093889BB243F00203AD
:108E100093800299E1600399C4F80080012206233F
:108E2000002066602161227284F8243015B0BDE80C
:108E3000F08F01913DF0CCFD431BBB420199AEDDAB
:108E4000484643F025FA94F86430002BB2D1E56D22
:108E5000CDF80480AB894FF4807B42F20F79019BFF
:108E6000BBB113F8017B01933DF0B2FD82462B8923
:108E70009A0710D5BFB2AF813DF0AAFD07462B89F6
:108E8000DB0712D5BBF1010BAB89E8D1C1E7314655
:108E90006CE7FF27E8E73DF09BFDA0EB0A004845A3
:108EA000E5DD284643F0F4F9B3E73DF091FDC01B42
:108EB0004845E4DDF5E7FFF739FAFFF7D5FE032073
:108EC00049E7FFF751FAFC215EE700BF581A00207E
:108ED0002DE9F04F8B4C94F8507087B0002F00F0C4
:108EE000938194F8242042F20F75531E082B7BD8EF
:108EF000DFE813F08E00B30037017A006800090044
:108F0000EC007A00D90094F86430002B40F008821D
:108F1000E66D94F808A02368B28903EB0A2A4FF49F
:108F2000807BBAF1000F00F0A6821AF8018B3DF0A9
:108F30004FFD81463389980740F1AD811FFA88F8CB
:108F4000A6F80C803DF044FD80463389D90740F1F6
:108F5000AD81BBF1010BB389E3D1237A0133DBB2DD
:108F6000022B23723DD1E66D3DF032FDB389804680
:108F700033899A0740F184813046002152F070F81D
:108F8000E66D3DF025FDB389804633899B0740F1AE
:108F90006C813046002152F063F8FFF7E5F900F0EC
:108FA0001F00052800F08882FFF75EFEE668002EAD
:108FB00000F0B1810022236961680120B04794F874
:108FC000242092E720684FF40071FFF7EBF90128A5
:108FD00000F08C81022800F090810646002800F005
:108FE000D28194F82420531EDBB2022B00F21681AA
:108FF000D4F8A03861695B1AC82B00F20B81A2F18A
:109000000807B7FA87F77F09384607B0BDE8F08F41
:10901000206E41F0A9FB00210846FFF7E3F9064660
:10902000FFF784F9012EDCD10023206E637641F036
:109030009BFB40F2AB110820FFF7D4F9052800F0A4
:109040006D81012800F0EE80FFF770F9627E002A42
:1090500000F04582022384F82430206E41F084FB26
:10906000637E022B0CBF4FF0804600260021372084
:10907000FFF7B8F931462920FFF7B4F90646FFF7A4
:1090800055F9002EADD1637E022B00F08F81A676BC
:10909000206E41F069FB00210920FFF7A3F998B386
:1090A000FFF744F99DE70826FFF75EF9FF2800F077
:1090B0001982013EF8D16369D4F8A028FA339342AB
:1090C0008FD2FFF7D1FD94F824200EE7FFF74CF97B
:1090D000FF284FF0080605D0013EECD0FFF744F919
:1090E000FF28F9D1236A0022012B227640F2008268
:1090F000E26908210132013BC4E9072384F8241006
:109100000A467CE7581A0020BE481021FFF74AF9AA
:1091100006460028C4D101217F20FEF771FF0128F7
:109120008046BDD130460221FEF76AFF002800F0DC
:10913000A5810128B4D116213A20FEF761FF013044
:109140008002A062FFF7F2F8206E41F00DFB0021D3
:109150000A20FFF747F9002840F07281032384F8C2
:109160002430102102A8FFF71DF900287FF439AF41
:109170009DF815309DF816109DF810209DF8096097
:109180009DF80A001B01DBB243EA111303F5FA63F1
:109190006387DDF8113001F00F0184F83C101BBA31
:1091A000110902F00F0240EA062084F8381084F812
:1091B00039209DF808109DF80B206363039B2363FF
:1091C000A08584F82E1084F82F20FFF7AFF8A37E37
:1091D0006BB9206E41F0C8FA4FF400711020FFF710
:1091E00001F90646FFF7A2F8002E7FF46AAFE06DA2
:1091F000042150F093F9002204233846226284F8B7
:10920000243007B0BDE8F08F384684F8247007B0EA
:10921000BDE8F08FFFF728FD94F82420042A7FF49E
:10922000EEAEF1E6E66D0DF1080AB3893B464FF06C
:10923000040B57464FF0FF099A463DF0C9FB8046A4
:10924000338998073AD5A6F80C903DF0C1FB8046CB
:109250003389D90743D5B3899BB20FB107F8013BD6
:10926000BBF1010BE9D1574632E03DF0B1FBA0EB79
:109270000800A8427FF789AE304643F009F88CE633
:109280003DF0A6FBA0EB0800A8427FF771AE304688
:1092900042F0FEFF74E63DF09BFBA0EB0900A84204
:1092A0007FF748AE304642F0F3FF56E63DF090FBC4
:1092B000A0EB0800A8427FF748AEF3E73DF088FB3B
:1092C000A0EB0800A842BBDD3046574642F0E0FF65
:1092D0009DF80B30AB2B04BF02236376B4E63DF060
:1092E00077FBA0EB0800A842B2DDEDE76369D4F894
:1092F000A02864339342BFF474AEFFF717F8FFF76A
:10930000B3FCE6683EB10022104623696168B047AD
:1093100094F82420E9E594F82420E6E5667693E6BF
:10932000A36E39485968D3F81CE0384E384B99423F
:1093300088BF30461EF0005F00F090804668DFF87E
:10934000D4C006EA0E0616EA0C0F3FF458AE0EEA39
:109350000C03C3600B68E66D23F001030B603389D7
:10936000D80703D5B3893389D907FBD433899A0742
:10937000FCD533891B06F9D4B38823F002031B0400
:109380001B0CB380F0E5FEF7D1FFE56826760423D9
:1093900084F82430002D3FF437AED4E9002123694E
:1093A0003046A84794F82420531E1DE6206E41F055
:1093B000DBF931463A20FFF715F8E66D01900DF123
:1093C000080AB3893B464FF0040B57464FF0FF099C
:1093D0009A463DF0FDFA804633899A071CD5A6F8D7
:1093E0000C903DF0F5FA80463389DB072FD5B38921
:1093F0009BB20FB107F8013BBBF1010BE9D1574616
:1094000014E000BF981A002000600240006402408F
:109410000F6402407D0F7D0F3DF0DAFAA0EB0800EB
:10942000A842D9DD3046574642F032FF019B3BB996
:10943000FEF77CFF029B1BBAC3F38073A37627E67B
:10944000FEF774FFFFF710FC94F824204DE53DF083
:10945000BFFAA0EB0800A842C6DDE3E70668DFF824
:10946000B0C006EA0E0616EA0C0F3FF4C8AD0EEACD
:109470000C0383606EE74FF0FF0858E504212C20B1
:10948000FEF7BEFD032106464E20FEF7B9FD0C2176
:1094900081463620FEF7B4FD09F10209431C03FAA8
:1094A00009F308FA06F6A3FB0601430A43EAC1538F
:1094B000A362FEF73BFF47E6E568D4F8A038636196
:1094C000072284F82420002D3FF499ADD4E900212F
:1094D00023690120A84794F82420531E84E584F8CA
:1094E00024208CE5FEF722FF042384F824308BE54A
:1094F00008D0042384F82430FEF718FF94F82420C1
:10950000531E71E5FEF7CCFF02287FF46AADC7E574
:109510007D0F7D0F00F01F0240090123032803FA8D
:1095200002F304D004280CD0022805D07047074A63
:10953000116C0B4313647047044A516C0B43536422
:109540007047024A116B0B431363704700380240A7
:10955000002845D003682A4A03F13F4101F57E0106
:1095600002EB9122F0B592F8382002F01F04520964
:109570000121032A01FA04F13DD0042A36D0022A3F
:109580002FD00022B0F804C011460126032706FAA6
:1095900001FE3EEA0C0001F101011CD11D6807FA31
:1095A00002F425EA04051D60186806FA02F5054371
:1095B0001D609D6825EA04059D609868986058685C
:1095C00020EA0E00586058685860D86820EA040005
:1095D000D860D868D860102902F10202D7D1F0BD56
:1095E0007047084A546C21435164CAE7054A146B1A
:1095F00021431163C5E7034A146C21431164C0E79A
:10960000D014060800380240002800F06381036887
:109610009D4A03F13F4101F57E0102EB912210B416
:1096200092F8382002F01F0452090121032A01FA9E
:1096300004F100F06281042A00F05681022A00F051
:109640004A818288D40700F13381900700F11E819E
:10965000510700F10781140700F1F280D00600F1F4
:10966000DD80910600F1C880540600F1B380100639
:1096700000F19E80D10500F18980940574D45005D5
:1096800061D411054ED4D4043BD4900428D45104A1
:1096900015D4120402D45DF8044B70471A685DF8C3
:1096A000044B22F040421A601A681A60DA6822F00D
:1096B0004042DA60DA6842F08042DA607047196846
:1096C00021F04051196019681960D96821F04051A2
:1096D000D960D968120441F08051D960DBD5DDE74B
:1096E000196821F04061196019681960D96821F082
:1096F0004061D960D96841F08061D9605104C8D512
:10970000DDE7196821F04071196019681960D9689E
:1097100021F04071D960D968900441F08071D9601E
:10972000B5D5DDE7196821F44001196019681960A1
:10973000D96821F44001D960D968D40441F480018A
:10974000D960A2D5DDE7196821F4401119601968C4
:109750001960D96821F44011D960D96841F48011A9
:10976000D96011058FD5DDE7196821F44021196012
:1097700019681960D96821F44021D960D968500569
:1097800041F48021D9607FF57CAFDCE7196821F4D2
:109790004031196019681960D96821F44031D960E5
:1097A000D968940541F48031D9607FF568AFDBE773
:1097B000196821F44041196019681960D96821F4C9
:1097C0004041D960D96841F48041D960D1057FF525
:1097D00054AFDBE7196821F440511960196819602A
:1097E000D96821F44051D960D968100641F48051FC
:1097F000D9607FF53FAFDBE7196821F4406119605C
:1098000019681960D96821F44061D960D968540693
:1098100041F48061D9607FF52AAFDBE7196821F454
:109820004071196019681960D96821F44071D960D4
:10983000D96841F48071D96091067FF515AFDBE7F7
:10984000196821F0C001196019681960D96821F000
:10985000C001D960D968D00641F04001D9607FF5D8
:1098600000AFDBE7196821F0300119601968196051
:10987000D96821F03001D960D968140741F010018E
:10988000D9607FF5EBAEDBE7D0140608196821F04C
:109890000C01196019681960D96821F00C01D960B0
:1098A000D96841F00401D96051077FF5D4AED9E7FA
:1098B000196821F00301196019681960D96821F04D
:1098C0000301D960D968900741F00101D9607FF5A3
:1098D000BFAEDBE770470D4A546C21435164828868
:1098E000D4077FF5B2AEE3E7084A146B2143116356
:1098F0008288D4077FF5A9AEDAE7044A146C2143C5
:1099000011648288D4077FF5A0AED1E70038024009
:109910002DE9F0416B4C00234FF4F07220210646F4
:1099200004F54F7084F83B3357F081FD04F21C506E
:109930004FF4F072202157F07AFD94F8FD0610B133
:1099400094F8FE261AB900252846BDE8F08140F0BB
:109950002DFC0746C4F8080740F0FAFE054600282B
:10996000F1D02FB12323FB80384609213CF05EFD66
:10997000D4F80807544F40F0FDFE94F8FE06013875
:1099800040B242F069FD0223102184F80037C4F888
:1099900004074FF0C3FDB7F82C124C4842F02EFCE0
:1099A000D4F8080740F0E0FEFF218C2052F00AFEB8
:1099B0008046D4F8080740F0DDFED4F804070421FF
:1099C0004FF0ACFDB8F11B0F04D0D4F80807FFF737
:1099D0001BFEB8E7D4F80837012284F83B230BB10B
:1099E0002322DA80B7F82C12384842F007FCD4F86A
:1099F000080740F0B9FE40210A2052F0E3FDFF21A4
:109A00008A2052F0DFFDC0F38013D4F8080784F8F1
:109A10000C3740F0AFFED4F8040704214FF07EFD70
:109A200094F8FC36012B44D0022B3AD0EBB394F8D7
:109A30000D37182B09D194F80C27B7F82C32A4F85D
:109A40001067A4F81227A4F81437B7F82C121F488F
:109A500042F0D4FBB7F82C121C4842F0CFFBD4F8EC
:109A6000080740F081FE0221002052F0ABFDD4F83F
:109A7000080740F07FFE0421D4F804074FF04EFDA4
:109A800094F81D2794F81E3794F81C1784F81817BB
:109A9000C2F12002C3F1100384F81F2784F8203795
:109AA00052E70823A7F82C32C1E71023A7F82C327D
:109AB000BDE7002EF5D094F80C37002B14BF082317
:109AC0001023EFE7502B00208801002050320020A7
:109AD00000487047E82B0020002871D0F0B583883B
:109AE000B3FA83F3202B0A4683B00446C3F11F0167
:109AF00050D0344F344D07EB81036E18C3F8242740
:109B0000002196F840603CF091FCA38821682F4822
:109B1000B3FA83F3C3F11F0202F0FC0404F18044A2
:109B200004F59C3402F003024FEA820E4FF00F0C52
:109B300001F13F42A1680CFA0EFC21EA0C01A16080
:109B400002F57E02A168C2F387224FF0004C02FAB0
:109B50000EF22CFA03F30A43A260436102681C4927
:109B600022EA03020260426822EA030242600268BB
:109B70001A430260826822EA03028260C26822EA13
:109B80000302C2600A68374413430B6097F86437D6
:109B9000F02B01D803B0F0BD3544F02195F85030DA
:109BA0008DF8043003224FF4807301A887F86417FE
:109BB0008DF80520ADF8063009F084FF03B0F0BD44
:109BC000704700BF502B0020D0140608003C014015
:109BD000083C014000285FD00368374A2DE9F04176
:109BE00003F13F4404F57E0402EB9422012492F831
:109BF000382002F01F055209032A04FA05F456D052
:109C0000042A4FD0022A48D08588B5FA85F0C0F1E1
:109C10001F00C0F3CC0603EB860600F007008200AD
:109C20000F24306A944020EA04003062306A01FA5E
:109C300002F20243002132624FF0010E0A464FF059
:109C4000030C02270EFA02F838EA050002F10102BD
:109C50001CD118680CFA01F420EA04001860186896
:109C600007FA01F606431E609E6826EA04069E6017
:109C700098689860586820EA0800586058685860EA
:109C8000D86820EA0400D860D868D860102A01F1AA
:109C90000201D7D1BDE8F0817047084A556C2C43CA
:109CA0005464B1E7054A156B2C431463ACE7034ACF
:109CB000156C2C431464A7E7D01406080038024042
:109CC0002DE9F04FDFF8ACA32DED028B9AF8801749
:109CD000002297B0CAF87027CAF87427CAF8782704
:109CE000CAF87C27CAF86C2719B19AF881278AF834
:109CF0006C279AF882271AB19AF883278AF87B276B
:109D00009AF886271AB19AF887278AF876279AF858
:109D100084271AB19AF885278AF871279AF8883724
:109D200005935A1ED3B257B203937B1C00F0AA804E
:109D3000C54AC64E52F83790029602EBC70200237E
:109D40001279019308EE102A1D463446984626786B
:109D50003946304643F03AFD83463046BBF1000FAA
:109D60001ED040F023FAEA1D1321D2B220B14FF0E9
:109D7000000E827180F807E03CF034FD207843F05B
:109D800057FD4FF0070308F1010223714FF0010363
:109D900084F802806070CDF804B05FFA82F8E37056
:109DA0000135042D04F10504D1D118EE100A029EEC
:109DB000CDF81080FFF7AEFBA549A64A48680240DF
:109DC00042F440324A600FB9019B5BB9A24C482073
:109DD000FFF7A0FB2046022153F0B0F9A26842F041
:109DE0000102A2609A489C4A4168BAF88A4741F445
:109DF00000014160516821F480515160916B21F460
:109E0000401141F480119163D16841F46001D16047
:109E1000956B85F44011C1F3015101EB81011F20C5
:109E200000FA01FC25EA0C0C112505FA01F141EAC2
:109E30000C019163D16841F4E011D160956BC5F3D9
:109E40000151C1F10401C9B201EB810188404FF019
:109E5000100C25EA00000CFA01F108439063E4B10C
:109E6000BAF88C17CAF89447A1B1BAF88E27CAF885
:109E7000981762B1019B7948521A90FBF2F2CAF826
:109E80009C276BB917B0BDEC028BBDE8F08F744A0C
:109E90001288EFE7734A1188E7E7734A1488DFE70F
:109EA0004846049953F04AF9684B012003F114081D
:109EB0000723F278441CE4B252B375783279A5F1E5
:109EC0000A0101EB410105EB450C092D03FA01FEE6
:109ED00003FA0CFB02FA01F140F29F80D9F80C2042
:109EE00022EA0E0E41EA0E01C9F80C10421E02EBE6
:109EF00082021F21062801FA02FC05FA02F272D83A
:109F0000D9F8341021EA0C010A432046C9F834205C
:109F10000536B045CDD1D9F80820039942F4007236
:109F2000C9F80820D9F8082042F48072C9F808203E
:109F3000D9F80820574442F00102C9F8082097F9DF
:109F4000902702203DF05CFA044600289AD046682B
:109F500030463DF043FA454B421E03EB421393F863
:109F60004450002D8ED1059983F84510062283F8C0
:109F70004420002886D030463DF030FA4FF0ECFE09
:109F8000606809F047FE07A809F006FE049EA26873
:109F900037480792012E8CBF4FF4806300230D9346
:109FA00009F14C034FF48072CDE90A5608930990E9
:109FB0004FF4003360680C9507A94FF400674FF425
:109FC0000056CDE91023CDE90E7609F0F7FD626861
:109FD000136843F001031360D9F8083043F080435D
:109FE000C9F808304EE7C11FA0F10D0201EB810155
:109FF0004FF01F0E02EB82020C280EFA01FC0EFA43
:10A0000002F005FA01F113D8D9F8302022EA0C0247
:10A0100011432046C9F830107AE7D9F8101002FA37
:10A020000CF221EA0B0B42EA0B02C9F810205DE7A3
:10A03000D9F82C1005FA02F221EA00010A43204661
:10A04000C9F82C2064E700BF28150608BC320020A0
:10A0500000230140E030FCFF002001408038010077
:10A060002E7AFF1F2C7AFF1F2A7AFF1F88010020FB
:10A07000F0320020502B00202DE9F84F2E4F00EB3E
:10A08000C00407EB8404D4F8AC672EB1054694F8FD
:10A09000BD0700F0FF0820B14FF000084046BDE8C2
:10A0A000F88F89469A4693463CF092FC4FEA490164
:10A0B0000123C9B284F8BE1784F8BFB784F8C1374A
:10A0C00084F8C28784F8C03784F8BD3784F8BC8729
:10A0D000B288C4F8C4A791058146C4F8C8A71DD4A6
:10A0E0003388DA0510D442F20F7405E03CF070FCBE
:10A0F000A0EB0903A34215DC33889B05F6D4338813
:10A100009BB243F480733380B3889BB243F44073B3
:10A110004FF00108B3804046BDE8F88F98464046AE
:10A12000BDE8F88FB7F8143801339BB22846A7F87A
:10A13000143852F0AFFCB1E7502B002070B5464EFA
:10A1400096F8164804EB440306EBC303650093F846
:10A150001838032B6ED8DFE803F059291E02254476
:10A1600006EBC505D5F81C08002870D196F878389C
:10A170009C425FD0013404F00302934286F8162813
:10A1800058D002EB420406EBC4040223C4F81C08B6
:10A1900084F8183870BD2B1906EBC303D3F81C28BC
:10A1A00072B1013AC3F81C28002070BD2B1906EBD0
:10A1B000C303D3F81C28002AF3D1022283F81828FD
:10A1C000254406EBC50595F82438013BDBB285F83C
:10A1D00024388BBB214B96F87868D3F83012D5F829
:10A1E0002008621C02F003024B1E0324B242034407
:10A1F00085F81848B3FBF1F0C5F81C081AD099424D
:10A2000018D80138C5F81C08012070BD42F028FAA2
:10A2100080B1124B2C44D3F8302206EBC404012148
:10A2200002F51C5384F818180F33B3FBF2F3C4F88B
:10A230001C3870BD012070BD084BD3F830220120BE
:10A2400002F2E733B3FBF2F3C5F81C3870BD0138F6
:10A25000C5F81C08002070BD502B0020880100208C
:10A2600030B583B00D46012301460DF107020446C7
:10A27000074842F0FFF89DF8072035EA020304D0B2
:10A2800003482A43214642F04FF903B030BD00BFD6
:10A29000CC3300202DE9F047214D95F87CC8BCF166
:10A2A000020F04460E46174608D013460A460146DA
:10A2B00005F67C00BDE8F04742F0DCB8D5F88438FC
:10A2C00013B11A689B885383D5F880A83CF080FBB3
:10A2D000BAF80C30804642F20F79BAF808309B0782
:10A2E00013D52146504650F0BBFE3B46D5F88008BA
:10A2F0003246002152F0A2F9D5F8843813B11A6819
:10A300009B8813830120BDE8F0873CF061FBA0EB44
:10A3100008034B45E1DD504641F0BAFFE5E700BFD9
:10A32000502B0020F0B50578022D83B0044615D0DF
:10A33000012D02D0002003B0F0BD90F90400274B9E
:10A34000421C83F8BC58F5D00328F3DC0A46617937
:10A3500003F6BC0303B0BDE8F0408DE6836813B19B
:10A360001A689B885383656801913CF031FBAB8987
:10A370000199064642F20F772B89980718D528468F
:10A3800050F06EFE65683CF023FBAB89064642F256
:10A390000F772B89990716D52846012150F060FECA
:10A3A000A368CBB11A689B881383012003B0F0BD6A
:10A3B00001913CF00DFB831BBB420199DCDD28467B
:10A3C00041F066FFDEE73CF003FB831BBB42E0DDB0
:10A3D000284641F05DFFE3E70120ACE7502B002069
:10A3E0002DE9F04FCA4CCB4E94F8BD18D4F8C408F0
:10A3F000DFF82883C84D83B0C1F3400140F0C0F9B5
:10A4000094F8BD18D4F8C008C94301F0010140F028
:10A41000B7F9052301934FF01009D4F8C43833B1CC
:10A420001A689B8851690B4214BF53831383D4F875
:10A43000C03833B11A689B8851690B4214BF5383EB
:10A440001383B4F8CC38002B40F0598194F8CE181F
:10A45000D4F8D00840F094F932204FF47A710127F3
:10A46000D8F80430C3F30803002B40F01B81EFF34E
:10A470001183002B40F01681D6F8A028D5F808E00B
:10A48000D6F8A0389A42F7D1D4F8F4389E45F3D8DC
:10A49000D4F8F0A801FB0AF3A3EB0E03B3FBFAF325
:10A4A00001FB0232D8F80430C3F30803002B40F05C
:10A4B000B780EFF31183002B40F0B280D6F8A038BC
:10A4C000D5F808B0D6F8A0E87345F7D1D4F8F4E889
:10A4D000F345F3D8D4F8F0A801FB0AFEAEEB0B0E5F
:10A4E000BEFBFAFE01FB03E39B1AB3F57A7FD9D3D7
:10A4F0000138B5D1D4F8C43833B11A689B88516992
:10A500000B4214BF53831383D4F8C03833B11A6895
:10A510009B8851690B4214BF53831383B4F8CC3822
:10A52000002B40F0E08094F8CE18D4F8D00881F0E9
:10A53000010140F025F932204FF47A710127D8F853
:10A540000430C3F30803002B40F08B80EFF311833A
:10A55000002B40F08680D6F8A028D5F808E0D6F881
:10A56000A0389A42F7D1D4F8F4389E45F3D8D4F8FD
:10A57000F0A801FB0AF3A3EB0E03B3FBFAF301FB14
:10A580000232D8F80430C3F3080343BBEFF311835E
:10A590002BBBD6F8A038D5F808B0D6F8A0E873459C
:10A5A000F7D1D4F8F4E8F345F3D8D4F8F0A801FBD8
:10A5B0000AFEAEEB0B0EBEFBFAFE01FB03E39B1A99
:10A5C000B3F57A7FDDD30138B9D1019B5F1E17F057
:10A5D000FF0301937FF421AF03B0BDE8F08FEFF3E9
:10A5E000118A89F31288D5F808B02B68DB0344BFC1
:10A5F000C4F8EC78D5F808B0D6F8A038D4F8ECE870
:10A600005FFA8AFA8AF31188D4F8F0A8734401FB40
:10A610000AFEAEEB0B0EBEFBFAFE01FB03E3CEE738
:10A62000EFF3118A89F31288D5F808B02B68DB03A1
:10A6300044BFC4F8EC78D5F808B0D6F8A038D4F800
:10A64000ECE85FFA8AFA8AF31188D4F8F0A8734428
:10A6500001FB0AFEAEEB0B0EBEFBFAFE01FB03E3B1
:10A6600042E7EFF3118E89F31288D5F808A02B6822
:10A67000DA0344BFC4F8EC78D5F808A0D6F8A038BF
:10A68000D4F8EC285FFA8EFE8EF31188D4F8F0E847
:10A690001A4401FB0EF3A3EB0A03B3FBFEF301FB29
:10A6A00002326EE7EFF3118E89F31288D5F808A015
:10A6B0002B68DA0344BFC4F8EC78D5F808A0D6F8C4
:10A6C000A038D4F8EC285FFA8EFE8EF31188D4F807
:10A6D000F0E81A4401FB0EF3A3EB0A03B3FBFEF30D
:10A6E00001FB0232DEE6D4F8E838002B3FF423AF5A
:10A6F000D4F8D4280023136084F8E5381BE7D4F895
:10A70000E838002B3FF4A8AE3CF062FAA4E600BFA4
:10A71000502B0020581A002010E000E000ED00E06F
:10A720002DE9F04F83B00A23C04CC14EDFF80883F7
:10A73000C04D0193FFF754FE10274FF4FA704FF409
:10A740007A714FF0010CD8F80430C3F30803002BE2
:10A7500040F05E82EFF31183002B40F05982D6F86F
:10A76000A028D5F808E0D6F8A0389A42F7D1D4F856
:10A77000F4389E45F3D8D4F8F09801FB09F3A3EB25
:10A780000E03B3FBF9F301FB0232D8F80430C3F334
:10A790000803002B40F01B82EFF31183002B40F0E5
:10A7A0001682D6F8A038D5F808A0D6F8A0E87345E8
:10A7B000F7D1D4F8F4E8F245F3D8D4F8F09801FBD7
:10A7C00009FEAEEB0A0EBEFBF9FE01FB03E39B1A8A
:10A7D000B3F57A7FD9D30138B5D194F8BD18D4F840
:10A7E000C408C1F340013FF0CBFF94F8BD18D4F882
:10A7F000C008C94301F001013FF0C2FF06274FF036
:10A800001009D4F8C43833B11A689B8851690B42D7
:10A8100014BF53831383D4F8C03833B11A689B88AC
:10A8200051690B4214BF53831383B4F8CC38002B07
:10A8300040F0308294F8CE18D4F8D0083FF0A0FF52
:10A84000FA204FF47A714FF0010CD8F80430C3F3BA
:10A850000803002B40F09A81EFF31183002B40F0A6
:10A860009581D6F8A028D5F808A0D6F8A0389A4245
:10A87000F7D1D4F8F4389A45F3D8D4F8F0E801FBCE
:10A880000EF3A3EB0A03B3FBFEF301FB0232D8F88D
:10A890000430C3F30803002B40F05781EFF311831A
:10A8A000002B40F05281D6F8A038D5F808B0D6F881
:10A8B000A0E87345F7D1D4F8F4E8F345F3D8D4F819
:10A8C000F0A801FB0AFEAEEB0B0EBEFBFAFE01FB8D
:10A8D00003E39B1AB3F57A7FD9D30138B5D1D4F805
:10A8E000C43833B11A689B8851690B4214BF538333
:10A8F0001383D4F8C03833B11A689B8851690B426E
:10A9000014BF53831383B4F8CC38002B40F0CA81B2
:10A9100094F8CE18D4F8D00881F001013FF030FF50
:10A92000FA204FF47A714FF0010CD8F80430C3F3D9
:10A930000803002B40F0E880EFF31183002B40F078
:10A94000E380D6F8A028D5F808A0D6F8A0389A4217
:10A95000F7D1D4F8F4389A45F3D8D4F8F0E801FBED
:10A960000EF3A3EB0A03B3FBFEF301FB0232D8F8AC
:10A970000430C3F30803002B40F0A580EFF31183EC
:10A98000002B40F0A080D6F8A038D5F808B0D6F853
:10A99000A0E87345F7D1D4F8F4E8F345F3D8D4F838
:10A9A000F0A801FB0AFEAEEB0B0EBEFBFAFE01FBAC
:10A9B00003E39B1AB3F57A7FD9D30138B5D1013FB0
:10A9C00017F0FF077FF41DAF4FF47A700146102790
:10A9D0004FF0010CD8F80430C3F30803002B40F00B
:10A9E0003881EFF31183002B40F03381D6F8A02893
:10A9F000D5F808E0D6F8A0389A42F7D1D4F8F43860
:10AA00009E45F3D8D4F8F09801FB09F3A3EB0E03AD
:10AA1000B3FBF9F301FB0232D8F80430C3F30803A7
:10AA200083BBEFF311836BBB08E000BF502B00200A
:10AA3000581A002010E000E000ED00E0D6F8A03841
:10AA4000D5F808A0D6F8A0E87345F7D1D4F8F4E813
:10AA5000F245F3D8D4F8F09801FB09FEAEEB0A0EEC
:10AA6000BEFBF9FE01FB03E39B1AB3F57A7FD3D358
:10AA70000138AFD1019B013B01937FF45BAE03B082
:10AA8000BDE8F08FEFF3118987F31288D5F808A09D
:10AA90002B68DB0344BFC4F8ECC8D5F808A0D6F88F
:10AAA000A038D4F8ECE85FFA89F989F31188D4F872
:10AAB000F098734401FB09FEAEEB0A0EBEFBF9FEF3
:10AAC00001FB03E3D0E7EFF3118A89F31288D5F88D
:10AAD00008B02B68DB0344BFC4F8ECC8D5F808B055
:10AAE000D6F8A038D4F8ECE85FFA8AFA8AF311882D
:10AAF000D4F8F0A8734401FB0AFEAEEB0B0EBEFBCC
:10AB0000FAFE01FB03E354E7EFF3118E89F3128899
:10AB1000D5F808A02B68DA0344BFC4F8ECC8D5F810
:10AB200008A0D6F8A038D4F8EC285FFA8EFE8EF391
:10AB30001188D4F8F0E81A4401FB0EF3A3EB0A03E2
:10AB4000B3FBFEF301FB023211E7EFF3118A89F345
:10AB50001288D5F808B02B68DB0344BFC4F8ECC8F2
:10AB6000D5F808B0D6F8A038D4F8ECE85FFA8AFA3D
:10AB70008AF31188D4F8F0A8734401FB0AFEAEEB07
:10AB80000B0EBEFBFAFE01FB03E3A2E6EFF3118E10
:10AB900089F31288D5F808A02B68DA0344BFC4F8FB
:10ABA000ECC8D5F808A0D6F8A038D4F8EC285FFA9D
:10ABB0008EFE8EF31188D4F8F0E81A4401FB0EF3F0
:10ABC000A3EB0A03B3FBFEF301FB02325FE6EFF3F4
:10ABD000118987F31288D5F808A02B68DB0344BFDE
:10ABE000C4F8ECC8D5F808A0D6F8A038D4F8ECE83A
:10ABF0005FFA89F989F31188D4F8F098734401FB5E
:10AC000009FEAEEB0A0EBEFBF9FE01FB03E3DEE537
:10AC1000EFF3118E87F31288D5F808902B68DA03CA
:10AC200044BFC4F8ECC8D5F80890D6F8A038D4F8DA
:10AC3000EC285FFA8EFE8EF31188D4F8F0E81A44FF
:10AC400001FB0EF3A3EB0903B3FBFEF301FB02329E
:10AC50009BE5EFF3118E87F31288D5F808902B68E7
:10AC6000DA0344BFC4F8ECC8D5F80890D6F8A03889
:10AC7000D4F8EC285FFA8EFE8EF31188D4F8F0E851
:10AC80001A4401FB0EF3A3EB0903B3FBFEF301FB34
:10AC90000232C1E6D4F8E838002B3FF4D1AD3BF0E6
:10ACA00097FFCDE5D4F8E838002B3FF439AED4F85F
:10ACB000D4280023136084F8E53831E610B4B8B125
:10ACC0000D4CD4F8F838102B05D15DF8044B052154
:10ACD000002040F08DBD03EB4302224482F8FD18B2
:10ACE00001210B4482F8FC0882F8FE18C4F8F838F9
:10ACF0005DF8044B704700BF502B0020C078202126
:10AD0000DCE700BF2DE9F04F2DED108B034697B027
:10AD100004331593DFEDCACA149002238A461392B6
:10AD20008B461293149C4FEADB0604EB461202EBAF
:10AD300006103101A6EB86034FEAC60806EB46056E
:10AD4000CDE9000100EBC303043108F104001196C2
:10AD5000204421442C01C6EBC60C0394EC00119D49
:10AD600004944FEACC0405946C0106EB860E029421
:10AD7000159D009C03EB46174FEACE0E02EBC6066C
:10AD80004FEACB094FF0000C51ED01AAD3ED001AA8
:10AD900092ED007A94ED005A96ED004AD7ED007AD4
:10ADA00015ED012A50ED016A32EE07BA76EE840AFB
:10ADB0007AEE855A31EEA70A3BEE256A70EE804A9C
:10ADC00076EEC46A36EE244A36EE646A05ED014A30
:10ADD00082ED006AD0ED00BAD6ED012AD3ED019ADA
:10ADE00095ED00AA92ED016A97ED013A91ED00CA46
:10ADF000D4ED014A7BEEE23A36EEE19A32EE472A92
:10AE000073EEE98A3AEE464A39EE279A78EE838A5B
:10AE1000B0EE428AA9EE6C8ADC44E24573EEC33A96
:10AE2000B0EE441AA8EEEC1A76EEE77A33EEA97A81
:10AE30007CEE643A77EEA17A3AEE066A7AEEC51AAB
:10AE40003CEE24AA74EECC4A39EE833A35EE6A5AC7
:10AE5000F0EE639AF0EE48AAE7EE2C9AA8EEAC4A20
:10AE6000E7EE2C4AE7EE6CAAF0EE418AB0EE427AA9
:10AE7000B0EE612A7BEE656A7BEEA22A76EE4A5A34
:10AE8000A9EE2C7AA7EEAC2AA7EEAC5AE7EEEC8A34
:10AE900032EE83BA76EEC3BA35EEE09A75EEC07A3A
:10AEA00036EE0A6A76EEE26A36EE0BAA76EE836A30
:10AEB00077EEA07A34EE423A77EE290A36EE4B6A04
:10AEC0007BEEA22A39EE000A73EEAA3A78EE244A03
:10AED00037EE697A31EE055A71EEA85A32EE044A1D
:10AEE00085ED00AA82ED016A4D4441ED012A4A44F4
:10AEF000C4ED006A81ED000AC4ED017A494440EDD9
:10AF0000010A4C4487ED007AC6ED003AC3ED004AD1
:10AF100080ED003A87ED014A484486ED015A4F44DE
:10AF2000C3ED015A4E444B443FF62EAF119B072B05
:10AF300040F2C781029D149E019B03980499059AD3
:10AF4000083575190C330E95354608F108080EF1D1
:10AF50000804EB1808300831083246442C19281828
:10AF60006918AA18079305F10C030D960C940B9021
:10AF70000A91099208934FF001084FF0000E129BBE
:10AF80009E44139B03EBCE0303EBCE02109302EB24
:10AF9000CE0303EBCE01029101EBCE0101EBCE0516
:10AFA00005EBCE06D6ED007A0F93AEEB8E03019142
:10AFB00006EB031303EBCE07D3ED01AACDED067A22
:10AFC000019BD5ED007A97ED01BACDED057AD3ED71
:10AFD000007A029BCDED047AD3ED007A0F9BCDED84
:10AFE000037A07EBCE0CD3ED007ADCED01BACDEDA0
:10AFF000027A0CEBCE01D2ED007A109A009101EBAF
:10B00000CE00014691ED01DACDED017A0099D2ED45
:10B01000007A91ED01CA00EBCE0000EBCE0494ED76
:10B0200001EAD0ED01DACDED007ADDE90776DDE960
:10B030000954DDE90B01DDE90D23C44602E000BF40
:10B04000F304353F94ED009A90ED00FA91ED006A1B
:10B05000D5ED007AD3ED006A57ED014A92ED005A22
:10B0600056ED013A96ED00AA35EE060A73EEA65AA1
:10B0700039EE278A34EE8F7A70EE082A75EE87EA69
:10B0800035EE465A3EEEA26A73EEE63A06ED016AE6
:10B09000D1ED019AD2ED01FAD4ED016AD3ED011A96
:10B0A00095ED013AD0ED018A97ED004A3FEEE96A4D
:10B0B00035EE491A76EE660A31EE271A3AEE612A23
:10B0C00075EE677A70EE830A3FEEA95A74EECF9A56
:10B0D00077EE897A7AEE211AB0EE42AA74EE68FA17
:10B0E000A0EEECAADC44E24535EEC77AB0EE639AF6
:10B0F00074EE285A38EEC44AF0EE698AA1EE6C9AD2
:10B10000E7EEAC8A36EE436A7FEE644A36EE266A94
:10B11000A0EEAC2AF0EE4A0AE7EEEC0AE7EEAC4A03
:10B12000F0EE687AF0EE498A36EE833AE6EE6C8A03
:10B13000E1EE2C3AB0EE6F1AA6EE2C1A71EEE56A2B
:10B14000A6EE2C4A71EEA55A75EE031A7EEEE22A9F
:10B1500037EE43FA75EEE1EAB0EE686A76EEC08A41
:10B1600039EE044A7FEE86FA76EEC86A33EE816ADB
:10B1700038EE888A73EEC13A37EE457A2CEE2E1AF5
:10B180003FEE055A22EECC9A9DED03FA70EE266A48
:10B1900033EE077AAFEE221AAFEE2E9A7AEE244AF9
:10B1A0009DED01FA79EEA09A25EE4BAA72EE670AA0
:10B1B00037EE822A6BEE087AAFEE08AAEFEE057A38
:10B1C0002DEEA63A9DED05FA67EE6D8AAFEE073AD1
:10B1D000EFEE268A66EE6A2A9DED00FA2AEEA00AB4
:10B1E000EFEE202A6EEE02EADDED060A23EECE5ADD
:10B1F000E0EEA3EA2BEEA98ADDED023AAFEE060AF5
:10B20000A3EE848A24EE6B7A6DEE246A9DED044AE7
:10B210002FEECD6AA0EE825AA3EEA97AE4EE2F6A51
:10B22000A4EE246A75EEA15AC6ED005A83ED001A09
:10B2300083ED019A4E4447ED017A87ED00AA4B4415
:10B2400080ED003AC0ED018A4F4482ED000A484487
:10B25000C2ED012AC5ED00EA85ED015A4A44C1ED6F
:10B26000006A81ED016A4D4484ED008A84ED017A23
:10B2700049444C443FF6E6AE0E9B08330E930D9BBB
:10B2800008330D930C9B08330C930B9B08330B93E3
:10B290000A9B08330A93099B08330993089B0833D8
:10B2A0000893079B08330793119B08F10108434556
:10B2B0007FF465AE129BDDF844B0DB009BB21293C5
:10B2C00030E517B0BDEC108BBDE8F08F08480023C7
:10B2D00002461178022902F1060204D00133062B3E
:10B2E000F7D10020704703EB430300EB43007047A6
:10B2F0007C340020F0B59F4C85B0242204F62C103D
:10B30000002156F094F894F85169002E3CD135464E
:10B31000D4F864396BB39B6A5BB3974898478368EA
:10B320003BB30388DFF878C2013B9BB260466646B8
:10B3300000213778032F06F106061DD001310629BA
:10B34000F7D100220178022900F1060000F0A68062
:10B350000132062AF6D1D4F88C19052909D0481CE7
:10B3600002FB01C2C4F88C090220002193801070F6
:10B370005180284605B0F0BD062303FB0141B1F81A
:10B380002E39013B9BB2DCE794F8500904F65813C0
:10B39000C4F8543908B90025BAE73EF007FF07465C
:10B3A000C4F860093FF0D4F905460028F3D0013E07
:10B3B000022370B284F8583941F04EF80028EAD0E0
:10B3C000C4F85C092FB12023FB80384609213BF0EB
:10B3D0002DF8D4F8543998683FF0CCF9D4F85439A2
:10B3E000102158684EF09AF8644BD4F85429C4F8E8
:10B3F000842993E803000123009032208DF8041083
:10B4000084F8883900263BF01FFB052302AA694611
:10B41000D4F854098DF80A608DF8096040F026FFD1
:10B420009DF80A209DF809009DF80B10544B12025C
:10B4300042EA00420A439A4200F0938032DCA3F5CC
:10B44000F1139A425FD043DD4E4B9A4253D0023300
:10B450009A4263D14FF400724FF48073A4F86829C4
:10B46000A4F87439B4F87429B4F86839120202FBEC
:10B4700003F300204FF48071B3F1807FC4F86C298E
:10B48000C4F8703984F87609A4F86A1958D83E4B84
:10B49000C4F86439012284F87D2939E7062101FBCB
:10B4A00002C261E7394B9A4235DC053B9A4235DDF1
:10B4B000374B1344032B4CD801A252F823F000BFA2
:10B4C00007B50008F7B40008E9B4000855B400084F
:10B4D000A3F52203013B9A423BD02DDD2D4B9A422E
:10B4E00009D001339A4219D14FF48073A4F8683916
:10B4F000A4F87439B6E780224FF48073A4F8682961
:10B50000A4F87439AEE740224FF48073A4F8682998
:10B51000A4F87439A6E7204B9A42E5D0002594F8A8
:10B520005009A4F86859A4F87459C4F86C59C4F8BF
:10B53000705940F041FEEBE6184B9A42D4D0EDE74B
:10B540000123D4F8840984F87C39B7214FF0BCFD7D
:10B550009DE720224FF48073A4F86829A4F8743979
:10B5600080E74FF480621023A4F86829A4F87439A6
:10B5700078E700BF502B0020B434002040150608A7
:10B580001640E0001720C200481506081940EF00D9
:10B59000EABF10FF17BA20001870EF001860010012
:10B5A0007C3400202DE9F041C54BC64EC64DC74C3A
:10B5B0000822C3F88820336B82B043F00103336361
:10B5C00007464FF4C052284640F202338846694687
:10B5D000CDE9002308F0F6FC6B6AC4F8748F23F4FD
:10B5E00070436B626B6AC4F87C7F43F420436B62E8
:10B5F0006B6AB749C4F8781F23F470236B626B6AD7
:10B60000B448C4F8900943F420236B62736CB249C8
:10B61000C4F8941943F480437364736BAF48B04922
:10B62000C4F8A00943F0800302257363AD4F84F88A
:10B630009859AD4EAD4DC4F8E4194FF0A043C4F88D
:10B640009C39AB4AC4F8AC7903F53463A1F5D071E9
:10B65000C4F8E859C4F8B069C4F8EC39C4F8B419AE
:10B660000123DFF8BCC2C4F8A8C907F51077A5F517
:10B67000E465A6F5A066A1F58C61C4F8F079C4F87C
:10B68000A459C4F85C6A84F89B3905F5A075536128
:10B6900006F5B076C4F8201A84F8A23A1946954BFC
:10B6A000954AC4F8285AA7F5BC67A035C4F8346A8F
:10B6B000924EC4F8307AC4F8383A07F5D45703F5F7
:10B6C0006953C4F83C5A4FF050250020DFF854E28B
:10B6D000C4F8602AACF5687C02F5A042C4F8647A2C
:10B6E000C4F8686A07F5A04706F5A046C4F86C3AA6
:10B6F000C4F8705AA3F5485304F51965C4F8742AC0
:10B70000C4F87C6AC4F89C3AC4F824EAC4F82CCA89
:10B710000246C4F8787A2B4684F8A40A402683F8B7
:10B720001C21A3F822210132042AC3E9496083F8CD
:10B730001D1183F81F01C3F8300103F12803EED176
:10B74000002211462B46402083F87423A3F87A2365
:10B750000132042AC3E9DF0183F8751383F87713F4
:10B76000C3F8881303F12803EED14FF0A0436448D7
:10B770009A6822F001029A60DA6842F04002DA60C8
:10B7800007F064FD94F899390022212161F31742F2
:10B790000BB142F4801294F89319D4F89C39012922
:10B7A0009A6300F0E480DA68D4F89C6AD4F8A009BF
:10B7B000C2F3076121F0600141F0400161F31F62B3
:10B7C0000021DA603160026861F3CC22026094F8F3
:10B7D0009B29012A00F0B88010214A4808F088F817
:10B7E000484808F06BF8D4F8A00994F89139002281
:10B7F0004FF0FF31026142618161C26153B305F1D3
:10B800001407414E114607EB83074FEA830C4FF0B4
:10B81000FF0E56F8042F1368002BACBF00234FF027
:10B820009043B74213601161C2F808E0F1D105F10D
:10B830005003364963440027FF2651F8042F15684A
:10B84000002DACBF00254FF090459942156017615F
:10B850009660F2D1036994F8931943F48073012937
:10B86000036161D0D4F89C29294800239361002901
:10B870004FF0FF336FF0804151615360516114BF4D
:10B8800000231023906143F470139069D4F8781F5B
:10B8900043F4605343F008030343936193680968DA
:10B8A00043F00103936088471A4B1B4ADA606846ED
:10B8B0001A4B009308F006F902B0BDE8F08100BF12
:10B8C00000E100E00038024000000240502B002060
:10B8D000BC030020080401004000400100080050A3
:10B8E000000B00502009005040090050200B005070
:10B8F000003C0140C00500500010005000300050D6
:10B90000EC340020E0340020F434002030350020F6
:10B910000008008000ED00E00005FA054302000188
:10B920000009005020050050D4F89C29144B0363F3
:10B930006FF08041134D00234FF0FF309361516150
:10B940005060516195619EE701680F4A0F4E41F0CA
:10B9500003010160802159629E62C3F80421E02244
:10B96000C3F80821C0F24002C3F80C2134E79A68FA
:10B9700022F03E0141F02A0161F307029A6012E7CA
:10B980000301810000080080A0004000800020002A
:10B9900010B5184C94F8860F88B9174B83F85100EE
:10B9A000586594F8893F012B1ED0D4F88C3FFBB129
:10B9B00012495B68BDE81040A1F10C0018473EF049
:10B9C000F5FB94F8882F0C49003A18BF012281F842
:10B9D000512048650028E4D01F22C280FDF714FEE4
:10B9E00094F8893F012BE0D1054BC4F88C3FDFE789
:10B9F00010BD00BF502B0020581A0020E03A002054
:10BA0000D803002099B10A6B824216D9154BD3F89E
:10BA1000CC2F914221D34C3991421ED30B6B9842CB
:10BA2000F9D38B6B9842F6D80B46184670470D4BEE
:10BA3000D3F8CC1F0A6B904212D30B680BB9F4E712
:10BA40000A6B90420B4602D38A6B9042EDD951F8B3
:10BA50004C3F002BF4D1184670470023184670471E
:10BA60000A46D8E7502B00202DE9F047CC0143D1FE
:10BA70000346224A43F8082B4FF0FF32426002246B
:10BA800018467E26DFF87880D8F8D09F2644013EFD
:10BA9000051D49466FF070474FF0010A08E0A342C8
:10BAA0001CD0631C45F8043C321B1C460435CAB14B
:10BAB0000B6BA34202D88B6BA34204D22046FFF744
:10BAC000A1FF014690B10A794B6B002AE7D1A3424E
:10BAD00004D0E6D245F8042C631CE5E745F8047C65
:10BAE000631CE1E7C8F8D01FBDE8F08745F804AC57
:10BAF000321B631C4946D8E78026C3E7F8FFFF0FD7
:10BB0000502B0020F0B40D6800240CE0BCF1050FB0
:10BB100018D8A0F137030A2B14D104EB840415F8CC
:10BB2000010B03EB4404A0F13003DEB2092EA0F1B7
:10BB30006107A0F1410CF0D9052FE7D8A0F1570318
:10BB40000A2BEAD00D601460F0BC7047036870B532
:10BB50005E6A26B133460522BDE8704018470446A8
:10BB60000D464E1D00E023689B682046984700283C
:10BB7000F9D0236815F8011B1B6820469847B54289
:10BB8000F1D170BD2DE9F047154B054603F6E4747D
:10BB9000002093F9DD8F84B06F1804F5287A0646EB
:10BBA0004FF0B6092368ABB193F83830142B11D09D
:10BBB00018F1020F01D043450CD1002269462046FE
:10BBC000CDE90266CDE90057ADF808908DF80E601A
:10BBD00032F09AFDE034A245E4D104B0BDE8F0872C
:10BBE000502B00202DE9F743124E0124A0231825E5
:10BBF0005FFA84F8FF2B14DCD6F88C01E9B2C1F1AE
:10BC00001C0282725F1C026880F80B80DBB200931A
:10BC1000C1F11B01D2F8189000234246C9B2C847AF
:10BC20003B46013DE6D10134052CE0D103B0BDE82F
:10BC3000F08300BF483C002010B50A4C94F8A901DD
:10BC4000003818BF0120FDF763FE50B1064904F526
:10BC5000C87040F041FA04F5C8700FF0E9FE04F531
:10BC6000C87010BD483C00207415060870B44479B3
:10BC700041BB03684FF400524FF4007620250221A7
:10BC80003CBB1A8C22F001021204120C1A841A8B8B
:10BC9000188C22F0F30280B2120420F00A00120C79
:10BCA000014342F0010241F001011A8319841A8B09
:10BCB00022F00C021204120C1A831A8B92B270BC7E
:10BCC0001A83704700220368164615461146002C59
:10BCD000D7D0042C21D0082C38D0198C21F48051D5
:10BCE0000904090C19849C8B1D8C45F6FF7040F6E5
:10BCF000FF4128402140024342F4805241F48071C8
:10BD000099831A849A8B22F440621204120C9A834B
:10BD10009A8B92B270BC9A8370471A8C22F01002F0
:10BD20001204120C1A84188B198C89B240F6FF4247
:10BD300021F0A00102400D4342F4807245F010054D
:10BD40001A831D841A8B22F44062B3E71A8C22F402
:10BD500080721204120C1A84998B1A8C21F0F30150
:10BD600092B2090422F42062090C324342F4807238
:10BD700041F0010199831A849A8B22F00C02C4E7E6
:10BD80002DE9F04F7D4C94F82E8494F839A487B0B7
:10BD900016460B22054689464046114602959DF8F7
:10BDA00040701D463AF098F9C245834640F0A6809F
:10BDB000039040463EF0FAF917F00803024601935B
:10BDC00000F09080BBF1000F00F088809BF8071016
:10BDD000890700F18380C4E97E0BC4F8F40110B137
:10BDE00040F60B31C18005F0020ADFF8A881029B02
:10BDF000634A84F8BC5108F580710025C4E9738159
:10BE00005846C4F8E43131464FF48073C4E97133C5
:10BE1000C4F8B821C4E97555C4E97755C4F8C061C0
:10BE200084F8BD71C4F8E891C4F8105484F814542F
:10BE3000A4F8085431F062F8D4F8FC0107F00101CD
:10BE4000FFF714FF4F4A504BD4F8FC01C4F81C54C0
:10BE5000C4F82024C4F81834BAF1000F25D0D4F85F
:10BE6000007217B33A6803689A421ED00123314624
:10BE7000384684F8153431F041F8D4F8000208F55A
:10BE80000572294639F092FED4F8FC012A4608F5DD
:10BE9000077139F08BFE019B93B93C4831F04AF8A9
:10BEA0003A48012131F07CF80AE0394A002302F1D6
:10BEB000080184F8153439F079FE019B002BECD091
:10BEC000324831F041F8314807B0BDE8F08FCDE994
:10BED0000403039B13B1D9798B0716D5002007B053
:10BEE000BDE8F08F15F00103F1D105F002018A469B
:10BEF000BAF1000F22D1D4F8FCB176E70B220C2165
:10BF000050463AF0E9F8039053E750463EF04EF9B8
:10BF1000039AC4F8FC2115F0020ADDE90423C4F8F1
:10BF2000F40105F0020123D0904219D0C0B140F6CF
:10BF30000C3CA0F806C0BAF1000FDCD0B8F1000F3D
:10BF4000CCD0C4F8F82183B9BBF1000FC6D0C4F837
:10BF5000FCB112B140F60B33D3805FFA81FACAE725
:10BF6000B8F1000FBAD0C4F8F821C4F800B2F0E775
:10BF70000028DCD1DDF80CB037E700BF483C0020DA
:10BF8000C415060869450308B9CF0308003E002020
:10BF9000604000204C3E0020094B13F84E3C042B1F
:10BFA00008D9053B032B08D801231A4600B10370BA
:10BFB0001046704700230122F8E700231A46F5E7F0
:10BFC000502B00202DE9F0479AB0DDE9226ADDF818
:10BFD000909004460D461746984602E020683BF0D4
:10BFE0006DFA20683BF072FA0028F7D1014664220E
:10BFF00001A855F01CFA264B8DF80450CDF85CA032
:10C000000293002D40D0AB1E012B3FD9042D14BF4D
:10C01000002203221F4B0396D3F8A0388DF8052089
:10C020001E440123CDE9059404968DF85B3037B1A9
:10C030004246394607A855F099F98DF85A80164EB0
:10C0400096F88A9400231893B9F1000F19D196F845
:10C050008904642202FB006001A900F28C4055F0C3
:10C0600085F9012386F8899486F88A34236843B1D8
:10C0700043463A46294620461AB0BDE8F04711F03B
:10C080001DBF1AB0BDE8F0870522C3E70222C1E751
:10C0900090400020581A0020483C00209FED737A01
:10C0A00007EE901A20EE070AF8EE677A27EE800A6C
:10C0B000FDEEC07A17EE903A2033402B00F2C78095
:10C0C000DFED6B7AB4EEE70AF1EE10FAF0EE407AAB
:10C0D0000CDD9FED686ADFED686AB0EE677AB4EE5A
:10C0E000E67AF1EE10FA77EEC67AF6DC9FED637A27
:10C0F000F4EEC77AF1EE10FA0CD59FED5E6ADFED33
:10C10000606AB0EE677AB4EEE67AF1EE10FA77EE96
:10C11000867AF6D49FED5B7AF4EEC77AF1EE10FAE8
:10C1200000F38D809FED587AF4EEC77AF1EE10FAA5
:10C1300044BF9FED527A77EE677A27EEA76ADFED6C
:10C14000535A9FED537ADFED536AA6EE257A67EED8
:10C15000865AE6EE076AB6EE007AE5EEA67A27EE94
:10C16000877ADFED486A70EE267ABDEEE76A16EE52
:10C17000103A2033402B67D8B4EEE60AF1EE10FAFD
:10C180000CDDDFED3C5A9FED3C6AF0EE676AF4EEA1
:10C19000C66AF1EE10FA77EEE57AF6DCDFED376A83
:10C1A000F4EEE67AF1EE10FA0CD5DFED325A9FED9F
:10C1B000346AF0EE676AF4EEC66AF1EE10FA77EED2
:10C1C000A57AF6D4DFED2F6AF4EEE67AF1EE10FAF6
:10C1D00040DDDFED276A76EEE77A67EEA75A9FED3E
:10C1E0002B5A9FED2B6ADFED2B6AA5EE856A27EEB1
:10C1F000A55AE5EE866AB8EE006AE5EE267A67EEA5
:10C20000867AC7EE206A0023836143610362C361BB
:10C21000B7EE006A76EE865A76EE666A86EE257A84
:10C2200067EE277A66EE876AC0ED017AC0ED037A81
:10C2300080ED007A80ED027AC0ED046A70479FEDD0
:10C240000C7A77EE677A78E7DFED137AD9E79FED1E
:10C25000127A86E7DFED0C6AF4EEE67AF1EE10FA78
:10C2600044BFDFED066A76EEE77AB6E727D4D2362A
:10C27000DB0F4940DB0FC940E4CB1641DB0F49C05F
:10C28000E4CB16C1DB0FC93FDB0FC9BF92E741B951
:10C290009730083C15A82ABE000000000C480D4B42
:10C2A000D0F80C1510B40C4CC0F8FC348A1E2231A6
:10C2B000B0F826351B01A4FB03C3DB08A3F5B0636C
:10C2C00022F8023F9142F3D15DF8044B704700BF62
:10C2D000483C002075100208CDCCCCCC70B5084C81
:10C2E000251D2E4614F8010B32F0DEFB28B1037831
:10C2F00005F8013BB442F5D170BDFF23F8E700BF5C
:10C30000904100202DE9F0471C4F012607F1080558
:10C31000B2464FF03C094FF0000817F8010B3DF012
:10C3200045FF044690B180F80690C671FB7803F093
:10C330007F02012A18D013F0800F20460DD185F816
:10C3400004803EF011FA85F805802C600136052E38
:10C3500005F10805E1D1BDE8F08785F804A03EF0BD
:10C3600009FA85F805A0F0E71B0604D42046FDF77E
:10C37000EFF8FB78DFE73EF0FDF9F7E798410020A2
:10C380002DE9F04FDFF8DC91DFF8DCA183B009F193
:10C390000C05012419F8018BB8F1000F00F0BD80E5
:10C3A0004FEA1817013F032F08F00F0200F2B88080
:10C3B0000AEB4703988D40FA02F616F0010600F0EA
:10C3C000C18001239340013B1840574451F04EFD7A
:10C3D00097F834305D4E184406EBC00604236E61B6
:10C3E000F471B371002303E00133152B00F0958045
:10C3F000574903EB43025F00895C4145F4D1554B3B
:10C400001A4412F8331C002900F09E80404639F08F
:10C41000CFFD8046006839F0B7FD98F8051039F077
:10C420000BFE0378002B78D14A4B3B4404225C730B
:10C430001A73002E58D0336898F8080003F13F4271
:10C4400002F57E020AEB9222012792F8382002F0D0
:10C450001F015209032A07FA01F169D0042A62D0A8
:10C46000022A6AD0B6F804C0BCFA8CF2C2F11F02EC
:10C47000C2F3CC0103EB810102F007020E6A9200C5
:10C480000F27974026EA07060E620E6A9040304357
:10C49000002208624FF0010B11460BFA01FE3EEA42
:10C4A0000C001CD118680326964020EA060018608C
:10C4B0001F6802209040384318609F6827EA0607EB
:10C4C0009F6098689860586820EA0E005860586825
:10C4D0005860D86820EA0600D860D868D860013172
:10C4E000102902F10202D8D11B4B1C4AB3F878156F
:10C4F000B3F87A350091002001340190B2FBF3F3D8
:10C5000028469BB24146E4B231F0A4FA0123092C3B
:10C510006B7405F118057FF43DAF03B0BDE8F08FF3
:10C5200000266E615EE70E4F3A6B0A433A6399E765
:10C530000B4A176C3943116494E7094A576C394325
:10C5400051648FE76E614DE70B68FFDE882B00209A
:10C550001C2B0020502B0020483C002040420F00A4
:10C5600000380240C4410020D01406082DE9F041F3
:10C570008C4B82B093F848260190002A40F00C8141
:10C5800093F86C26B3F86E16DFED876AB3F8708601
:10C59000864D07EE102A07EE901AB8EEC76AB7EE7E
:10C5A000007AB3F86A16A5F80081F0EE475A4FEA10
:10C5B0004804E6EE665A8C42B8BF0C46A6EE267AD0
:10C5C000A6B20121F8EEE77AA5F8046167EEA67A33
:10C5D000C5ED3D5A85ED3E7AC5ED3F7A83F84816A4
:10C5E000002A00F0D680DDED017A9FED710AF8EEA9
:10C5F000677AA4B280EE270A52F0B4FB6400B0FB65
:10C60000F4F4012CB8BF0124E4B2B0FBF4F39BB204
:10C61000074685F8084100EE103ABBEEED0A85EDBD
:10C62000430A52F09FFB634BDFED636AB8FBF0F007
:10C63000A3FB0737FF0807EE907AF8EEE77A0228A7
:10C6400086EEA77AB8BF02205C4985F81001002366
:10C650009FED5B1A9FED5B6ADFED5B1ADFED5B5AC6
:10C660009FED5B2ADFED5B2A9FED5B3ADFED5B3AE6
:10C670009FED5B4A85ED457A07EE903AB8EEE77A92
:10C68000F0EE467AE7EE017AFDEEE76A16EE902AC2
:10C690002032402A7AD8B4EEE17AF1EE10FA0CDDBD
:10C6A000DFED506A9FED507AB0EE675AB4EEC75A8C
:10C6B000F1EE10FA77EEE67AF6DCF4EEE57AF1EEDA
:10C6C00010FA0CD5DFED476A9FED487AB0EE675A55
:10C6D000B4EEC75AF1EE10FA77EEA67AF6D4F4EE7D
:10C6E000C67AF1EE10FA49DD74EE677A67EEA76A52
:10C6F000F0EE624AE6EE824AF0EE430AE6EEA40A63
:10C70000B7EE007A27EEE65A77EE677AB6EE007A51
:10C71000E5EE207A67EE877A0133202BE1EC017A8F
:10C72000AAD107EE904AF8EEE77AF7EE006A86EEB5
:10C73000A77A2F4B2F4AC5F8B43703F12801A83345
:10C74000C5F8B0171020C5F8C0372021142385F88C
:10C750001146A5F8AC07A5F8BC1707EE906AF8EEED
:10C76000677AA5F8B83782ED007AC2EDAC7AC2EDEF
:10C77000AD7AC2EDAE7A02B0BDE8F081F4EEE37AB4
:10C78000F1EE10FA48BF75EEE77AAFE7F6EE007A01
:10C79000C2E7194B1A7026E7044D95F80841B5F821
:10C7A0000461BEE7483C00200AD7233C1400001077
:10C7B00000247449ABAAAAAADB0FC9412C010010BE
:10C7C0003C8C4F3EDB0FC93F0100F840DB0F49C0F6
:10C7D00092E741B99730083C15A82ABEDB0FC9BFC4
:10C7E000DB0F4940DB0FC940E4CB1641E4CB16C157
:10C7F000F415060828060010000000102DE9F84383
:10C80000204E214F96F8778687F8BD8806F2746629
:10C8100007F50C6500244FF0050916F8010B18BB4D
:10C8200028600134032C05F10405F6D16FEA0801F4
:10C83000D7F8C00801F001013DF0A2FF97F8BD183C
:10C84000D7F8C40881F00201C1F340013DF098FF20
:10C8500097F8BD18D7F8C80881F00401BDE8F8437F
:10C86000C1F380013DF08CBF3DF0A0FC0134286095
:10C87000E3B210B180F80690C3712868FCF768FE37
:10C88000D0E700BF483C0020502B00202DE9F041AC
:10C890002A4C2B4DB4F87C66A5F8CC6882B0EEB972
:10C8A00094F878063DF082FC94F87926C5F8D00813
:10C8B000003A18BF012285F8CE2848B194F87A16BC
:10C8C0002B22002914BF11210121C28039F08AFFD7
:10C8D000002002B0BDE8F0413EF068BF94F87886D1
:10C8E000002240462B2139F0F7FB074640463DF039
:10C8F0005DFCF8B1F7B12B22C5F8E808C280397A9F
:10C90000FDF768F94FF000080E4AB2FBF6F3C3F3E7
:10C910004F0000909BB23946CDF8048005F6D40054
:10C92000A4F87E6631F096F8D5F8D438C3F80080C4
:10C9300085F8E58802B0BDE8F08100BF483C0020E2
:10C94000502B002040420F002DE9F84F254C94F861
:10C950008C3684F8803604F28367002604F5D464AC
:10C960005FFA86FB0BF101085FFA88F8012117F8DE
:10C97000010F42460E448A4639F0AEFB4FF00009E3
:10C98000054640B3387804F80E9C04F80D9C04F872
:10C990000FBC04F810AC44F8045C3DF007FC18B17F
:10C9A00080F806A080F80780297AFDF713F90E4A6F
:10C9B0000021284639F07AF90C4B23600C4B221DDC
:10C9C00021462846C4E9013939F0F0F86979286828
:10C9D0004A4630F0E1FB082E04F11C04C0D1BDE84A
:10C9E000F88F00BF483C002040420F00D1D103081F
:10C9F0005D3D030870B52C4C2C4B94F8B807C4F877
:10CA0000B03700220221C4F87027C4F87427C4F894
:10CA10007827C4F8AC27A4F8B42739F05DFB0028C8
:10CA200041D0234B0668054603F1C0015A7C12B180
:10CA30005A6896422BD018338B42F7D1002394F8D2
:10CA4000B807C4F89C5684F890363DF0AFFB08B1A7
:10CA50000223C380297AFDF7BDF82846154A002134
:10CA600039F024F9144A1549C4F8A0160026111FFC
:10CA70002846134BC4F8A436C4F8A86639F096F8D3
:10CA8000697928683246BDE8704030F085BB304691
:10CA90004CF0C8FE328D0B4992B2531CB0FBF3F040
:10CAA00081F87402CAE770BD483C002000FFFF0017
:10CAB0004800001040420F00EC420020853D030872
:10CAC000253F0308880100202DE9F04FC14DDFF814
:10CAD000409385B088460446C02205F13400002109
:10CAE000CDF8048054F0A3FC99F8B937002B71D02D
:10CAF00099F8BA37002B00F08C80DFF8F8A21AF80A
:10CB0000403C012B00F0AE80022B00F08F80B24B36
:10CB1000B24E02931C460FCE0FC40FCE0FC41AF8AC
:10CB20004A7C1AF84E3C96E80700AD4EC5F82C69D1
:10CB30003E1E18BF0126072B84E8070085F84C69C4
:10CB400000F20D81042B00F21781DFF8C892DFF8A4
:10CB5000B0820026019B5FFA86FB0BF10107FFB252
:10CB6000B3423A464FF0030129DD18F8014B204645
:10CB700039F0B2FA034620461C4613B33DF016FBCB
:10CB8000C9F8140018B14FF003038371C7711AF884
:10CB90004D3C1AF84E2C002B00F0EC80E37983F02A
:10CBA00001035946204601364DF088F948B14FF04F
:10CBB0000103082E89F8113009F11809CAD1029B26
:10CBC00006E0884B884AC5F83839C5F83029002373
:10CBD000C5F84839D5F8483963B10022019883F87F
:10CBE0002C00012183F82D101A6383F82E2005B044
:10CBF000BDE8F08F7D4E7E4C0FCE0FC40FCE0FC41C
:10CC000096E80700A4F1200384E80700C5F8483936
:10CC1000EDE7784B019913F84C2C003A204618BFE9
:10CC20000122FBF7D9FDC5F84809D3E71AF84A3CB9
:10CC3000002B3FF46CAF1AF84E3C082B12D1674E14
:10CC4000674F0FCE05F6141402940FC40FCE0FC415
:10CC500096E80700012384E8070085F84C39C5F8F9
:10CC60002C797FE0644C019BC5F850390FCC634FA1
:10CC70000FC70FCC0FC794E807001AF84A4C1AF8F0
:10CC80004E3C89F8F437003CA7F6CC034FF0000681
:10CC900018BF012403935A4B85F84C4987E80700D5
:10CCA00007F15C0889F8BC67B34602933EE0F2796D
:10CCB00082F0010707F0010695F84C09013689F862
:10CCC000BB6708B187F0010720463DF041FD002811
:10CCD00062D0002C6DD0A088C8F80C407101B0FA69
:10CCE00080F041F009010BF1010BC0F11F004FF082
:10CCF0000303C8F80400C8F8141088F8107084F80A
:10CD000007B0A371204639F06DFDFB07204623D5FF
:10CD10003DF02AFD039BD8F80C205A61BBF1080FA7
:10CD200003F1180308F1200803931FD0D5F8502908
:10CD30005A451BDD029B13F8014B0293204639F044
:10CD4000FFF9064620463DF031FA1AF84D2C04460C
:10CD5000002AACD1F779ADE73DF00CFDDAE7082BFE
:10CD60007FF4F3AE274BC5F85439EEE62348C5F8F7
:10CD700048092FE7E37914E71AF84B3C224AC5F833
:10CD80005429012B05D0022B06BFB7FA87F35B09A4
:10CD9000002385F85839D8E6134A1C4BC5F8FC28FF
:10CDA000C5F8F8380F4AC5F80429012389F8BC37BB
:10CDB000DDE7710141F009014FF0FF33C8F81410AD
:10CDC000C8F80430C8F80C4088F810700BF1010B5B
:10CDD00098E700BF14000010280900104817060843
:10CDE0007D750508CD3F0408D53F04081C170608CB
:10CDF00008440020502B002074170608F408001087
:10CE0000072B00201540040845400408D93F0408BA
:10CE1000483C0020480000102DE9F84FCA4B93F819
:10CE2000200593F821553DF0C1F958B12D23C38059
:10CE30000446FCF7E9FB0A2039F0D8FC20463EF016
:10CE4000C5FF20B9C04BD3F8F837DE0001D5BDE8E7
:10CE5000F88F013D092DFAD8BB4B93F81F45E4B973
:10CE6000402033F0E9FA0028F1D090F90430B64AB6
:10CE7000092BC8BF143B92F8F51413440A2993F800
:10CE8000244400F0C681B04A93F82F3492F81E254E
:10CE9000002A08BF1C46002CD9D020463DF086F958
:10CEA0008046002800F0AE812D23C380FCF750FBA4
:10CEB000012108463DF06CFCD8F80030B8F8042099
:10CEC0001A833C2039F0C0FD002101203DF060FCB8
:10CED0009D4B93F82135002B00F0D6809B4C9C4E47
:10CEE000DFF874929B4D002794F8BD18D4F8C00861
:10CEF000C94301F001013DF043FC94F8BD18D4F89A
:10CF0000C80881F00401C1F380013DF039FCB8F19B
:10CF1000000F04D0D8F80030B8F804205A83D9F8AC
:10CF20000430C3F30803002B40F01881EFF31183A2
:10CF3000002B40F01381D6F8A028A968D6F8A038B5
:10CF40009A42F8D1D4F8F4389942F4D8D4F8F0C819
:10CF50004FF47A7000FB0CF35B1AB3FBFCF300FB9D
:10CF600002324FF0100C4FF47A710120D9F80430DE
:10CF7000C3F30803002B40F0C580EFF31183002BAF
:10CF800040F0C080D6F8A038D5F808B0D6F8A0E8B0
:10CF90007345F7D1D4F8F4E8F345F3D8D4F8F0A802
:10CFA00001FB0AFEAEEB0B0EBEFBFAFE01FB03E338
:10CFB0009B1A772BDAD994F8BD18D4F8C00801F081
:10CFC00001013DF0DDFB94F8BD18D4F8C808C1F3A9
:10CFD00080013DF0D5FBB8F1000F04D0D8F8003047
:10CFE000B8F804201A83D9F80430C3F30803002BDF
:10CFF00040F0D880EFF31183002B40F0D380D6F8B7
:10D00000A028A968D6F8A0389A42F8D1D4F8F43804
:10D010009942F4D8D4F8F0C84FF47A7000FB0CF3BE
:10D020005B1AB3FBFCF300FB02324FF0100C4FF421
:10D030007A710120D9F80430C3F30803002B40D1E2
:10D04000EFF31183002B3CD1D6F8A038D5F808B007
:10D05000D6F8A0E87345F7D1D4F8F4E8F345F3D84F
:10D06000D4F8F0A801FB0AFEAEEB0B0EBEFBFAFEF5
:10D0700001FB03E39B1A772BDCD9334B93F8213563
:10D0800001379F42FFF630AF2F4B93F81F35002B2F
:10D0900040F0AC802C4A92F82035002B7FF4D7AEBC
:10D0A00092F82235012B7FF4D2AED2F8F83713F084
:10D0B00080537FF4CCAE82F82135BDE8F84F43F0C1
:10D0C000BBBBEFF3118A8CF31288D5F808B02B683C
:10D0D000DB0344BFC4F8EC08D5F808B0D6F8A03894
:10D0E000D4F8ECE85FFA8AFA8AF31188D4F8F0A849
:10D0F000734401FB0AFEAEEB0B0EBEFBFAFE01FB16
:10D1000003E3B7E7EFF3118A8CF31288D5F808B080
:10D110002B68DB0344BFC4F8EC08D5F808B0D6F898
:10D12000A038D4F8ECE85FFA8AFA8AF31188D4F8C8
:10D13000F0A8734401FB0AFEAEEB0B0EBEFBFAFE39
:10D1400001FB03E334E700BF483C0020502B0020E4
:10D15000581A002010E000E000ED00E0EFF311812C
:10D16000102383F31288D5F808C02B68DA0304D59E
:10D170000123C4F8EC38D5F808C0D6F8A038D4F8A4
:10D18000EC28C9B281F31188D4F8F0084FF47A7111
:10D190001A4401FB00F3A3EB0C03B3FBF0F301FB18
:10D1A0000232DEE6EFF31181102383F31288D5F803
:10D1B00008C02B68DA0304D50123C4F8EC38D5F88D
:10D1C00008C0D6F8A038D4F8EC28C9B281F3118889
:10D1D000D4F8F0084FF47A711A4401FB00F3A3EB82
:10D1E0000C03B3FBF0F301FB02321EE7322039F0EF
:10D1F0002BFCB8F1000F3FF44DAF4046002139F051
:10D2000015F947E7FCF7A4F9012108463DF0C0FAFB
:10D2100057E6D2F8FC375D057FF519AE09F00CFD35
:10D2200000287FF414AE002C7FF437AE0FE600BF69
:10D23000084B03F500600DC8904202DC114602461F
:10D240000846984204DD9A42B8BF1A461046704715
:10D25000704700BF483C00200B6810B414681B1BCB
:10D26000036054684B681B1B43608B6892685DF8D1
:10D27000044B9B1A836070472DE9F047041E0D464E
:10D2800012DB092C26DC824A0B468248A0FB0410E4
:10D29000C00800EB8000A4EB40000021125C1A7073
:10D2A00059702846BDE8F08764422D23092C01F807
:10D2B000013B24D8764A774BA3FB0403DB0803EB3E
:10D2C0008303A4EB43030020D35C48700B70284613
:10D2D000BDE8F0876F4B632CA3FB04264FEAD6060C
:10D2E00021DC6B4A0B466B49A1FB0601C90801EB27
:10D2F0008101A6EB4101515C03F8011BC5E7654ABA
:10D30000632CA2FB04364FEAD60637D8604A614B3D
:10D31000A3FB0603DB0803EB8303A6EB4303D35C09
:10D3200001F8013BC7E7A3FB0627B4F57A7F4FEA74
:10D33000D7070DD2564A0B465649A1FB0701C9082B
:10D3400001EB8101A7EB4101515C03F8011BCAE726
:10D35000A3FB072842F20F7294424FEAD80836D84E
:10D360004B4A0B464B49A1FB0801C90801EB81015F
:10D37000A8EB4101515C03F8011BDDE7A2FB063776
:10D38000B4F57A7F4FEAD7070CD2414A414BA3FB51
:10D390000703DB0803EB8303A7EB4303D35C01F82C
:10D3A000013BB4E7A2FB073842F20F739C424FEAFD
:10D3B000D80821D8364A374BA3FB0803DB0803EB18
:10D3C0008303A8EB4303D35C01F8013BDEE7324A59
:10D3D000A3FB080994424FEAD90921D82C4A0B46ED
:10D3E0002C49A1FB0901C90801EB8101A9EB41010D
:10D3F000515C03F8011BB5E7274BA2FB08099C42CF
:10D400004FEAD90921D8224A224BA3FB0903DB08A2
:10D4100003EB8303A9EB4303D35C01F8013BCAE7A9
:10D420001E4AA3FB090394424FEAD30A21D80B46B4
:10D430001849174AA1FB0A01C90801EB8101AAEBAF
:10D440004101515C03F8011BCAE7144BA2FB09021E
:10D450009C424FEAD20A13D80E4B0D4AA3FB0A0393
:10D46000DB0803EB8303AAEB4303D35C01F8013B26
:10D47000CAE70A22BAFBF2F047F084FA0346D7E77C
:10D480000A22BAFBF2F047F07DFA0146E4E700BF5A
:10D4900014A10608CDCCCCCC9F8601003F420F00E2
:10D4A00070B4344890F80C38A3F13001092957D8EA
:10D4B00000F60C04224600F61B0012F8015FA5F1ED
:10D4C0003001092904D88242F7D1002070BC70478E
:10D4D000141B022C4ADD2848002101E010F8013B12
:10D4E00001EB810103EB4103161A303B022E044687
:10D4F00003F0FF01F2DC214B03FB01F1A2424FF0EC
:10D5000000030DD903EB830314F8016B5B00303B80
:10D510003344A24203F0FF03F4D1194800FB03F3A4
:10D520002E2D06D01748A0FB032301EB930070BCFF
:10D530007047013204200024157804EB8404303D48
:10D540006400092D00F1FF30A4B202D82C44A4B22B
:10D55000013210F0FF00EFD1642202FB0433E1E757
:10D5600000211D4600F60C020B46D9E7064C0021AF
:10D57000C4E700BF483C0020554400208096980036
:10D5800040420F00ABAAAAAA5444002038B5044672
:10D590000D460A460068FF2153F049FF21682944DF
:10D5A000216038BD83B50C461646054631F0EAFACF
:10D5B000204631F0E7FA0021204B0846002E08BF34
:10D5C0001E463DF0E5F8002101203DF0E1F8284637
:10D5D00039F07CFFB0B1012100203DF0D9F8284698
:10D5E00039F06CFF0746204639F06CFF0028FAD06E
:10D5F0003946204639F06EFF3846B04700210846CC
:10D600003DF0C6F8204639F061FF0028DFD0012147
:10D6100000203DF0BDF8204639F050FF0146284675
:10D62000019139F04FFF01990028F8D0284639F0D0
:10D6300051FF002108463DF0ABF8C8E725D30308A9
:10D64000F0B500230B604B608B60CB600B61026810
:10D65000DFF88CC089B004ADC2F385572E4647FA77
:10D6600003F0C007344604D513F80C0004F8010B8E
:10D6700026460133062BF2D11748C2F30324044493
:10D68000002394F8D84233708DF8184000F5387CA8
:10D69000C2F305370DF1190647FA03F0C007344607
:10D6A00004D513F80C0004F8010B26460133062BB1
:10D6B000F2D100233370C2F3834406ABCDE90134C9
:10D6C000084602F00F0305490095C2F303124BF020
:10D6D0004BF809B0F0BD00BFD01406083CA1060805
:10D6E000A017060870B5094CD4F81C28054662B18D
:10D6F0000026D4F81C082D2101363EF07FFFAE42F3
:10D70000F7DBBDE8704040F035B970BD483C002003
:10D7100038B50546084644F053F8041E0D4B0FDBA0
:10D7200093F85C2A944205DA0B48214641F0FAF856
:10D73000204638BDFF2C03D1084841F0F3F8F7E745
:10D7400093F85C2A0649013A284640F0BBF84FF0AE
:10D75000FF34EDE7140000104BA106085CA1060899
:10D760006FA10608114A013002EBC000F0B4D0F8F6
:10D77000ECC20F4E00233360336133623363336492
:10D78000336533663367BCF1000F0DD090F8E87253
:10D7900057B13F0100240CEB04030FCB35191034B3
:10D7A000A74285E80F00F6D1F0BC7047D0140608F8
:10D7B0006844002038B50F4C94F8A71801F03F01D9
:10D7C0008B1C024601F10A0584F8A53884F8A2589A
:10D7D00004F50A6084F8A32808311BF0F9FD2544FC
:10D7E00085F89E0894F8A2381C44000A84F89F0823
:10D7F00038BD00BF483C002070B51D4C0968D4F806
:10D80000CC581C4ED4F8C848D6ED9E7ADFED1A6A83
:10D81000491B00EE901A0168F8EEE00A091B60EE61
:10D82000A70A00EE101A20EEA07AB8EEC00A1C4635
:10D83000A0EE007AB1EE400AF1EEC77A67EEA67A62
:10D84000FCEEE77AC2ED007A4BF072F89FED0B7AAE
:10D85000DFED0B7AE0EE077AFDEEE77A17EE902A1D
:10D86000002ABCBF02F50C42A032226070BD00BF8E
:10D87000483C0020880100202C7D8E3FA00CB34541
:10D8800000A00C4638B50B4C002501228021204613
:10D8900032F0BEFD30B194F9040032F0EDFD08B174
:10D8A000006838BD0135082D04F10C04EDD10020CD
:10D8B000F7E700BF2845002038B5041F00F1080530
:10D8C00054F8043FD81780EA430016F0FFFEA54243
:10D8D000F6D138BD2DE9F041D24CDFEDD37AD4F842
:10D8E000603A94F8F90A07EE103A2DED028BB8EE83
:10D8F000478A28EE278A002840F0CA80D4F8042BF3
:10D9000094F8F81A94F8153B002A19DD07EE902ACE
:10D91000DFEDC66AF8EEE77AC3F1640386EEA77A14
:10D9200000EE103AB8EEC00A20EE070A29B920EE40
:10D93000000ADFEDBF7A20EE270A51F013FA80B219
:10D94000B4F8FA3AA4F8FA0A834200F0A18094F8F5
:10D95000647AB84EDFEDB88A4FF00008002594F8DD
:10D96000183B2B41DB0714D594F8F83A002B7FD1F4
:10D97000B4F8FA3A07EE103A002F00F0FB80B8EE48
:10D98000477AC8EE877A77EE887A88EE277A86ED2E
:10D99000027A0135042D06F12406E0D194F8FD5AEF
:10D9A000B4F8006B002D40F0E880002F5CD194F8B3
:10D9B000143B84F8205B84F81C3B002E54D0002DCF
:10D9C00052D007EE906A0123B8EE678ADFED9A7AAB
:10D9D00084F8243B9D42C7EE888A28D0022D43D18B
:10D9E000D4F8601A9548B0EE480A43F075F894F8F8
:10D9F000203B012B00F01181022B35D1D4F8601AA5
:10DA00008F48B0EE480A43F067F894F8203B012BAA
:10DA100000F0FE80022B27D1B0EE480ABDEC028B4D
:10DA2000D4F8601A8748BDE8F04143F055B8864AFB
:10DA3000D2ED007A78EEA76A134687EEA67A002127
:10DA400043F8041F83ED017A78EEA76A002187EE80
:10DA5000A67A996083ED037A77EEA88A002287EE92
:10DA6000A87A1A6183ED057ABDEC028BBDE8F081DE
:10DA7000B4F8FA3AD4F8601A00EE103A301DB8EE55
:10DA8000400A002F70D143F027F894F8647A80E7B9
:10DA900094F8647A002F3FF45CAF94F8FD5AB4F820
:10DAA000006B002DE0D0694A94F8FE3AD2F8442980
:10DAB00092F883201343D7D1D4F8042B94F8153B64
:10DAC000002A65DD07EE902ADFED586AF8EEE77A66
:10DAD000C3F1640386EEA77A012D00EE103AB8EE8A
:10DAE000C00A27EE000A60D051F03CF980B2A4F8D9
:10DAF000000B002F79D08642B6D00028B4D094F81D
:10DB0000203B002BB0D007EE900AB8EE678ADFED1D
:10DB10004A7A012BC7EE888A4ED0022BA4D1D4F8C2
:10DB2000601A4648B0EE480A42F0C0FE94F8203B26
:10DB3000012B6AD0022B97D1D4F8601A4048B0EE7E
:10DB4000480A42F0B3FE94F8203B012B58D0022B38
:10DB50008AD1B0EE480ABDEC028BD4F8601A39487D
:10DB6000BDE8F04142F0A2BE301D42F09FFE94F8A5
:10DB7000647A0EE7C6F8048001E7344A94F8FE3A66
:10DB8000D2F8442992F8832013437FF40EAF93E731
:10DB90000023A4F8003B002F7FF466AF94F8143BF9
:10DBA00084F8205B84F81C3B5EE720EE000ADFED82
:10DBB000207A20EE270A97E7234A1346F3EC017AEE
:10DBC00078EEA76A87EEA67A83ED017AD2ED007A25
:10DBD00078EEA76A87EEA67A83ED037A77EEA88AB5
:10DBE00087EEA87A83ED057A3EE794F8143B84F833
:10DBF000205B84F81C3B00283FF436AF0646E0E685
:10DC0000114AD2ED007A131DE8E70F4A131DDDE734
:10DC10000D4AD2ED007A131D1EE70B4AD2ED007AB1
:10DC2000131D11E714000010BD37863500409C45D8
:10DC3000CDCC4C3C780A001083F9223E3C0B0010FE
:10DC4000600B0010840B0010A80B0010483C002053
:10DC5000F8B5214C1D270E46054684F848791BF07F
:10DC6000DDFC00201BF07CFC08201BF079FC0E2062
:10DC70001BF076FC38461BF073FC04201BF070FC94
:10DC800004201BF06DFC00201BF06AFC30201BF010
:10DC900067FC00201BF064FC30461BF061FC002098
:10DCA0001BF05EFC1BF0A6FC04F649101BF0ACFB5D
:10DCB000234670B194F8492962B994F84A29302A68
:10DCC00000D03AB993F84B2922B993F84C392B700C
:10DCD0000120F8BD0120FCE7483C0020104B034424
:10DCE00010B5044693F8C00310F06AFC0D4800EB31
:10DCF00044040A23B4F95C19B1F5FA6FA8BF4FF4D4
:10DD0000FA61B1F57A7FB8BF4FF47A71A1F57A71F3
:10DD1000BDE81040B1FBF3F10920C9B210F07EBCA0
:10DD2000D0140608483C00201D4991F80C28A2B3E5
:10DD3000F0B4002605463346304637461BB991F805
:10DD40000C482D2C23D02E2A19D0CA1800EB8000A5
:10DD500092F80C48A4F13002092A4FEA40009CBF17
:10DD6000A0F13002A0180E2B14D80133CA1892F873
:10DD70000C28002AE2D106B14042F0BC70470133C2
:10DD8000002DF8D0CA182A4482F80C78DDE7012368
:10DD90001E46EBE70020F0BC70470020704700BF34
:10DDA000483C00201FB503AC8DF80C3000940023D4
:10DDB0008DF80D300EF082FF04B010BDF8B50546A9
:10DDC000262024F065FA134C0146F8B9D4F88009EE
:10DDD00090F838301E3B012B01D939F07BFB0E4FF8
:10DDE0000026AE420ADBB4F8A4390133A4F8A43902
:10DDF0000A4BD3F8A038C4F8B439F8BD17F8011BA2
:10DE0000D4F8800939F066FB0136EAE7002384F88C
:10DE1000B239EDE7483C0020CC450020581A0020DC
:10DE200010B58021044604F0F7FE2046002104F0DE
:10DE3000F3FE2046BDE8104005F02EBA2DE9F04172
:10DE4000B14C94F8CB39C4F8B80982B088465A2B43
:10DE500000F2B980DFE813F0CC00B700B700DC00B7
:10DE6000B700B700B700B700B700B700B700B700FA
:10DE7000B700B700B700B700B700B7000F01B70091
:10DE8000B700B700B700B700B700B70033017400A0
:10DE9000B700B7007400B700B700B700B700B8010B
:10DEA000B7006201B700B7007C00B7000902B700F5
:10DEB000B700B700B7005B00B700B700B700B70006
:10DEC000B700B700B700B700B700B700B700B7009A
:10DED000B700B700B700B700B700B700B700B7008A
:10DEE000B700B700B700B700B700B700B700B7007A
:10DEF000B700B700B700B700B700B700B700B7006A
:10DF0000B700B700B700B700B700B700E40194F856
:10DF1000CC399B0700F16982B4F8D239D4F8CD2905
:10DF2000D4F80C1A5BBA9BB212BAD0188842C4F863
:10DF3000183AC4F8142A03D904F02EFE002854DB42
:10DF40000020A4F8040A0546284602B0BDE8F08186
:10DF500094F8103A002B40F0FF8094F9C839002B58
:10DF600031DAD4F8003A08469B689847002840F018
:10DF70001E82B4F8D209D4F8CD29D4F80C3A40BAAC
:10DF800080B212BA15189D42C4F8180AC4F8142AAF
:10DF900007D904F001FE002827DBD4F8142AD4F8AE
:10DFA000180AD4F8083AD4F8C46903FB00F003FB5C
:10DFB00002F20225B042C4F8142AC4F8180A84F800
:10DFC000105A00F0CF8094F8DC395A1CD2B204EB1E
:10DFD000C30305204FF40051042A84F8DC2983F898
:10DFE000E009C3F8E41900F0A0814FF0FF35ABE77A
:10DFF000D4F8C439002BE6D1D4F8003A08469B681F
:10E0000098470546002840F0D281A4F8040A9BE70F
:10E010003E4B002203F1120103F8012F8B42FBD18A
:10E020003B4994F8063A94F8DC0970250D70984243
:10E030004FF00C05CD7110D004EBC300013390F804
:10E04000E0598D70B0F8E409DBB2042B40BA888146
:10E0500014BF84F8063A84F8062A94F8CF391222BD
:10E060009342A4F8042A98BFA4F8043A002528464D
:10E0700002B0BDE8F08194F8CC39DA0700F13E81B6
:10E08000D4F8003A94F8CF09DA6901EBC10102EB48
:10E0900081010A79531D834228BF0346A4F8043A3C
:10E0A000002BE3D0013B1A489BB2013319440344CF
:10E0B00011F8012D03F8012D8342F9D1D6E7154E51
:10E0C000154F35460823073EC5F10700A4F8043A6A
:10E0D000002202E092F8E0231D462B46B54203F8E9
:10E0E000012900EB030217FA82F2F3D1D4F8003AC7
:10E0F0004046DB6898470028B8D0AB7863F07F03D0
:10E10000AB70002520E700BF483C00202B490020D1
:10E110002C49002033490020D0140608D4F8003AD6
:10E12000C74A5B680846111D98470546002840F01D
:10E130003E81D4F80C3AC34AD4F8081A013B180EB1
:10E140001070180C09BAD37050701B0A0820937015
:10E150005160A4F8040AF7E6D4F8186AD4F8142A2F
:10E16000D4F8083AD4F8005AB2FBF3F24FF48057CF
:10E17000BE4228BF3E462D69B249A4F8047A404603
:10E18000B6FBF3F39BB2A8470028C0F2BC8033462D
:10E19000AC4AD4F8B809812104F072FDD4F8142AED
:10E1A000D4F8180AD4F8243A3244851B9E1BC4F8CC
:10E1B000142AC4F8185AC4F8246A002D7FF456AF04
:10E1C000032384F8103ABFE69E4E0027334606F13B
:10E1D0000C0203F8017B9A42FBD1D4F8003A404686
:10E1E0005B686A4601A998470546002840F0E98027
:10E1F000019BBDF80020013B190E52BAF371317139
:10E20000190C1B0A71710820B371022172810C2351
:10E21000BDF80220F07031727272A4F8043A93E6ED
:10E22000894E8A4F30460823073EC0F10705A4F8FF
:10E23000043A002202E092F8E82318460346864298
:10E2400003F8012905EB030217FA82F2F3D1D4F89F
:10E25000003A4046DB68984700283FF407AFF37860
:10E2600063F07F03F37000256EE694F8103A002BFC
:10E2700061D194F9C839002BFFF6A5AED4F8003A65
:10E2800008469B689847002840F09180D4F8003AEF
:10E290004046DB6898470546002840F0BA80B4F84D
:10E2A000D239D4F8CD29D4F80C1A5BBA9BB212BA81
:10E2B000D0188842C4F8183AC4F8142A00F29F8093
:10E2C000D4F8081AD4F8C40903FB01F302FB01F2E5
:10E2D0008342C4F8142AC4F8183A7FF474AEB3F534
:10E2E000805F28BF4FF480530121D4F8B809554A04
:10E2F00084F8101A9BB204F0EDFD25E6072354497B
:10E30000A4F8043ACEE694F8DC395A1CD2B204EBF5
:10E31000C30304204FF48851824284F8DC2983F837
:10E32000E009C3F8E4197FF460AE002384F8DC3917
:10E330004FF0FF3508E6D4F8186AD4F8000AD4F88C
:10E34000083AD4F8142A4569B2FBF3F2B6F5805FB7
:10E3500028BF4FF480560846B6FBF3F339499BB209
:10E36000A847002862DBD4F8142AD4F8185AD4F845
:10E37000243A3244AD1B9B1BC4F8142AC4F8185A23
:10E38000C4F8243A2DB9D4F8B809294604F0F6FDAA
:10E39000DAE5B5F5805F28BF4FF48055ABB2D4F80D
:10E3A000B809284A012104F095FD0025CCE594F830
:10E3B000DC395A1CD2B204EBC30302204FF468517B
:10E3C0000AE694F8DC3904EBC3020133DBB2022025
:10E3D0004FF46851042B82F8E009C2F8E41922D006
:10E3E00084F8DC394FF0FF35AEE594F8DC395A1C7F
:10E3F000D2B204EBC30305204FF41051ECE504F056
:10E40000CBFB0028FFF6F1ADD4F8142AD4F8183A63
:10E4100056E794F8DC395A1CD2B204EBC30302204D
:10E420004FF41C51D8E584F8DC79DEE594F8DC394A
:10E430005A1CD2B204EBC30304204FF440716BE7C3
:10E44000504600202C49002033490020D0140608F3
:10E45000A818060810B5FBF73BFB044610B11121C4
:10E4600037F0E4FF20463CF07FF9C82038F0ECFAA2
:10E470002046BDE810403CF07DB900BF2DE9F04FCB
:10E48000B34CD4F89C395A69D2078BB002D50BB083
:10E49000BDE8F08F5A699B6912EA030AF7D0CAF304
:10E4A00007431AF4002F009340F00281009B5D07A0
:10E4B00043D41AF0020F5FFA8AF503D0D4F89C39DE
:10E4C00002225A61BAF1000FC0F211821AF4006FF1
:10E4D000CAF3072740F084812E0708D59D4B9E483C
:10E4E000D3F888329847D4F89C3908225A61ED064F
:10E4F00000F1E981F80600F1A981B90600F12E8149
:10E50000009BDA0609D5934B9348D3F89832984785
:10E51000D4F89C394FF480125A61009B9B06B6D503
:10E520008C4B8D48D3F89C329847D4F89C394FF4E3
:10E5300000125A610BB0BDE8F08FD4F8A02993699E
:10E54000D26913401FFA83FBBBF1000FB1D0DFF893
:10E550000882CDF80CA045464FF0000909E05FEABB
:10E560005B0B09F1010908F1040805F1280500F029
:10E57000DA811BF0010FF2D0D4F8A0195FFA89F705
:10E5800008694A6B04EB8703FA40D3F8A839D20133
:10E590009B68D2B202431A40D007D3B216D54B6B58
:10E5A000D8F81820012000FA09F023EA00034B6391
:10E5B000684B6948D3F88032012191603946984709
:10E5C00094F89369012E00F0FC8101231A0703D50A
:10E5D000D8F8182008239360DE0603D5D8F8182051
:10E5E00010239360580603D5D8F818204023936071
:10E5F000990703D5D8F81820022393601A06AED5E0
:10E60000D5E94C60D5F82431D8F818C0311A8B42BE
:10E61000DCF8182028BF0B46033392B2B2EB930FFD
:10E620009DD9D4F8A029323704EB8703CDE90198AE
:10E6300090469946B04238D2BEB3D5F8241194F82A
:10E640009339D5F82821371AB94228BF394601F144
:10E65000030E4FEA9E0E83B98FB20337BF10D9F86D
:10E6600098A90AD0013352F8040BCAF800009F425F
:10E67000F8D1D5E94C60D5F82821DCF818300844E9
:10E680000A44B042C5F82821C5F834010AD195F8EA
:10E690001C11D8F83420012707FA01F122EA0102FF
:10E6A000C8F834209BB29E45C4D3DDE9019856E7F3
:10E6B000D4F8A0399D69DB691D402D0C3FF4F6AEFE
:10E6C00004F51966DFF88CB0B046B146002708E0C3
:10E6D0006D0807F1010706F1040608F128083FF468
:10E6E000E5AEEB07F4D5F9B204EB8102D4F8A0391A
:10E6F000D2F8E42992685B691A40D007D3B218D5E2
:10E7000094F89309726D01239842936007D11269BE
:10E71000D8F87C33C2F312029B1AC8F88C33DBF8AA
:10E720007C324846984794F89339012B00F0578182
:10E7300001239A0702D5726D022393601B07C7D588
:10E74000DBF8843248469847736D08229A60BFE729
:10E75000502B002088010020E0340020D4F8A0399C
:10E76000D4F8A8199A680868C2F34102022A08BFBF
:10E7700003224FF0000514BF65F30A0062F30A009C
:10E7800008605A6842F480725A6006A805F0CCFB13
:10E79000D4F89C29D4F8A009D368BF49079D6FF32A
:10E7A0008D23D3608068C0F34100014491F8F013D9
:10E7B000032900F0CF80B949B9480126294484F8DB
:10E7C000926981424FF04006A4F8946900F21581E5
:10E7D0000E2161F38D234FF40051D36051618FE618
:10E7E000B04B94F8A22AD3F89032AF4800218DF8AC
:10E7F00017108DF817209847D4F8A019D4F89C2941
:10E8000094F89A3988684FF400615161002B3FF405
:10E8100063AEC3077FF560AE94F8A53A012B7FF491
:10E820005BAE9DF81730032B7FF456AED4F89C3ABC
:10E830009E491A6842F001021A601A6842F0030207
:10E840001A600B6943F006030B6145E6D4F8A02972
:10E85000954853684FF0000823F001034146536088
:10E8600005F046F894F89169414656B1904BFF2265
:10E8700003EB860653F8045FD86BAA609E42826061
:10E88000F8D1D4F8A03988484FF0FF329A614FF0A0
:10E890000112DA610B2262F3070162F30708C3F881
:10E8A000148019611A686FF30A121A6004F0F4FCFC
:10E8B000D4F89C297B4B7C48D3F88C324FF48051A0
:10E8C0005161984719E6D4F89C399A6922F01002F0
:10E8D0009A611A6AC2F34340022802F00F0144D041
:10E8E000062823D09A6942F010029A6102E694F851
:10E8F0009A393BB1D4F89C2A136823F0030161F3E1
:10E9000007031360D4F8A02966495368D1F894121C
:10E91000654823F0010353608847D4F89C394FF0D1
:10E9200000425A61D2E5DDF80CA0C2E501EB81019D
:10E93000D4F8605A04EBC1012E68D1F81C0DC4F85C
:10E940005C6FC2F30A1202442868C4F8600FC1F871
:10E950001C2DC7E700214FF4007084F8921909219B
:10E96000A4F8940961F38D2335E747F6F07010425F
:10E97000B8D001EB8100C2F30A1204EBC00002F12F
:10E98000030C5FEAAC0CD0F8105DD4F860EA4FEAF3
:10E99000810818BF002006D00130DEF8006045F87D
:10E9A000046B8445F8D1414404EBC101D1F8105DFA
:10E9B000D1F81C0D15440244C1F8105DC1F81C2D9E
:10E9C00090E7B9F1000F7FF400AE94F8A13A042B60
:10E9D0007FF4FBAD344804F05FFC3346F6E5002FCE
:10E9E0007FF4A6AE94F8A12A052A7FF4A1AE48468A
:10E9F000019304F051FC019B9BE62E48A5F57401A0
:10EA0000A1F51051814203D80D2161F38D23E2E677
:10EA100029492A482944814203D20C2161F38D23DC
:10EA2000D9E62748A5F18C71A1F54341814203D86D
:10EA30000B2161F38D23CEE62249234829448142EC
:10EA400003D20A2161F38D23C5E6204920482944D9
:10EA5000814203D2092161F38D23BCE61D48A5F153
:10EA6000B771A1F55851814203D2082161F38D237A
:10EA7000B1E6194919482944814203D2072161F3BB
:10EA80008D23A8E6164917482944814234BF062140
:10EA9000052161F38D239EE6D0140608401E1BFF5E
:10EAA0003F420F0088010020E034002000ED00E02C
:10EAB000F4340020DFC810002013FBFE20D6130022
:10EAC000FF69180000D3CEFE40771B00C05BB3FE89
:10EAD000C091210040AC2700C01D6AFE40E1330018
:10EAE000803C36FEE09C4100704700BF704700BF8D
:10EAF000704700BF704700BF2DE9F0414FF0FF3570
:10EB0000324A33482C46002304E001330B2B02F138
:10EB1000100215D0917A0429F7D103F5B17100EBF9
:10EB20000111C979CF07F0D4661C116801D0A94240
:10EB3000EBD21C4601330B2B0D4602F11002E9D13A
:10EB4000631C02D10120BDE8F081214D04F5B177AD
:10EB500005EB07139988F1B9DFF880802601AB191E
:10EB6000D8F88C2F1B4916691B4A41F2186001EB3B
:10EB7000442118580023B047D0B1022808D141F2EF
:10EB8000CC6205EB0717AB58013B0121AB50B971C3
:10EB90000020BDE8F081DFF8448005EB0413D8F8CD
:10EBA0008C2F41F21860D268185826019047D6E79A
:10EBB00041F2CC6205EB0717AB580321B97141F262
:10EBC000D061013B0124AB506C54BCE7486F00207E
:10EBD0002C59002044590020F9EB0008502B00204C
:10EBE000044B41F2E472995C09B901219954012264
:10EBF0005A7070472C59002038B5174D174B41F209
:10EC0000D0640020285504E001300B2803F11003E4
:10EC100014D053F80E4C8C42F6D11C78032CF3D14F
:10EC20006AB10F4B03EB40239A4201D0FFF7D8FFA4
:10EC300000F5B17005EB00100123837138BD41F27E
:10EC4000CC6100F5B1736A5805EB0313042001325F
:10EC500098716A5038BD00BF2C590020526F0020B7
:10EC60004459002038B5134B00209C7B14B11D681B
:10EC70008D4205D001300B2803F11003F5D138BDCA
:10EC800072B10D4B03EB40239A4210D0FFF7A8FF5F
:10EC90000A4B00F5B17003EB00100123837138BDFE
:10ECA000064B00F5B17003EB0010827138BD022CE9
:10ECB000ECD1EDE7446F0020445900202C5900208E
:10ECC0002DE9F84F12F0020E9B4606D028B9FFF747
:10ECD00087FF02252846BDE8F88F804C41F63805AD
:10ECE0006559002D5BD14FF0FF367D4FB146B046E0
:10ECF000B24600253B68984200F0B68097F80EC0F7
:10ED0000BCF1000F5BD0BCF1010F15D105F5B17C52
:10ED100004EB0C1C9CF807C01CF0010F0CD11CF07C
:10ED20007E0F09D15FEADC1340F0A880D7F808C055
:10ED3000D44501D2E246A94601350B2D07F1100753
:10ED4000D8D1751C04D1B8F1FF3F00F09F80464632
:10ED500041F2C86806F5B17754F80850013544F817
:10ED6000085004EB061C41F21C694FEA07184CF8E6
:10ED7000095044F8085041F2186904EB07154FF0A8
:10ED800000084CF80900C5F8048004EB0715AD79BC
:10ED9000042D9CD8DFE805F01A330F334D0004F53D
:10EDA000C25741F63C063F68A65907FB0565A842D5
:10EDB00099D3FFF715FF00252846BDE8F88F2E46AA
:10EDC00001350B2D07F1100794D1BAE712F0010CB1
:10EDD00070D104EB0710D51090F80780BBF1030F3A
:10EDE00065F3C71880F8078062D94FF6FF70834536
:10EDF0005B4628BF03469BB204EB07108380BEF13D
:10EE0000000F16D004EB061303F5B0531833987BAC
:10EE100004280ED041F2C8654FF0040C605901304F
:10EE2000605141F2CC65586083F80EC063590133DC
:10EE30006351500705D504EB0710C37943F0010374
:10EE4000C371D30608D504EB0714E379C3F3450275
:10EE5000013262F34603E371224B012503EB4626A0
:10EE60000E602846BDE8F88F05F5B17704EB07166C
:10EE70004FEA071CB67986B92E4669E7A8460135E0
:10EE80000B2D07F110077FF435AF5AE7B9F1FF3FBB
:10EE900018BF4E467FF45CAF8DE741F2C8682E463E
:10EEA00054F80850013544F8085044F80C506CE709
:10EEB0006346A1E70C4B0B49D3F88C3F0B4AD3F8C0
:10EEC000088001EB46210023C04700283FF473AFC0
:10EED00004EB07140223A371FCE600BF2C590020A9
:10EEE000446F002044590020502B002065EC00089E
:10EEF000F0B5124D2B7841F63002022B0BBF070AFA
:10EF0000C0F3D417C4B200F07F04A85883B00E46F3
:10EF100000230122384401A9FFF7D2FE01280AD1BB
:10EF20002B78022B019B16BF53F8243033F8143092
:10EF300023F07043336003B0F0BD00BF2C590020B4
:10EF400010B5144602070B4610D50B4941F2C472A6
:10EF5000581C8B58834204D305D100232360012021
:10EF600010BDFFF73DFE2060012010BD2146184670
:10EF7000BDE81040BCE700BF2C5900202DE9F0414E
:10EF80004268C2F308030B44B3F5007F82B0044625
:10EF90000D4657D390F91A30591C0AD0304A03F560
:10EFA000B17302EB0313FF21DA796FF30002DA7118
:10EFB000817694F91B305A1C0FD0294A03F5B1739E
:10EFC00002EB0313FF20DA79C2F34501013921EA8C
:10EFD000E17161F34602DA71E0762378022B37D0D3
:10EFE0001F4A02F5C2531B68B5EB432F4FEA432873
:10EFF00024DC41F648036768D6583E407342AB4272
:10F000001CDCAB19434511D32169207E01AAFFF70F
:10F0100097FF012812D16768236963614744019B08
:10F020002361A5EB0801BF1B67608D192046F9F726
:10F0300023F920B93D446560012000E0002002B0C2
:10F04000BDE8F08115444560012002B0BDE8F081C3
:10F05000616801202944616002B0BDE8F08100BF11
:10F060002C59002070B5154604460E46FFF786FF62
:10F0700050B994F8280028B9022384F82830C4E94C
:10F080000B5670BD022070BD1DB12046A84701205F
:10F0900070BD012070BD00BF10B4D0E9011390F91C
:10F0A0001A208B4238BF0B46511C83600AD0144B88
:10F0B00002F5B17203EB0212FF21D3796FF3000363
:10F0C000D371817690F91B305A1C0FD00C4A03F58E
:10F0D000B17302EB0313FF24DA79C2F3450101395E
:10F0E00021EAE17161F34602DA71C4760022436AD3
:10F0F0005DF8044B4261426011460361B2E700BF14
:10F100002C59002038B544220021114852F08FF9C3
:10F11000104B41F602011A784FF6FF745C52022A36
:10F1200041F2E87118BF032203F5C05041F64C05C7
:10F130005A5441F60C0441F6010203215D5900F8CE
:10F14000181910211D519954FFF7A6FF012038BD51
:10F15000147100202C5900202DE9F041B1F9043040
:10F160000F2B82B00C461646054632D02846F9F7DA
:10F17000A7F895F91B80B8F1FF3F074633D02D4B18
:10F1800041F2186203EB08118A58904211D11833EA
:10F1900003EB4823A188013109B203EB4113A1809D
:10F1A00028463360F9F78CF82060012002B0BDE8F2
:10F1B000F081FFF715FD2846F9F75EF828B1002326
:10F1C0000120336002B0BDE8F081002002B0BDE84C
:10F1D000F0814FF40071FFF7D1FE0028F5D04FF613
:10F1E000FF73A380C2E72846F9F746F80028E2D16A
:10F1F0000FB9FFF7F5FC38460023112201A9FFF7EC
:10F200005FFD0128D7D1019B0B4A9A1A48BF02F231
:10F21000FF12B2F5B05F4FEA622106D24FFA81F8D1
:10F2200085F81B80002BB5D1C5E7FFF7D9FC019B02
:10F23000F6E700BF2C5900204459002030B50446A1
:10F24000C06983B010B9012003B030BD0D46002362
:10F25000032201A9FFF734FD0128F5D1B4F92030CC
:10F26000002B03DAFFF7BCFC0220EDE7019A012D29
:10F270004FEA431102EB431303D0022D12D1E525CF
:10F280005554A268DA612278032A04D100221A7741
:10F290005A779A77DA77626A5A83C2F30F429A8270
:10F2A00003B030BDE268DA61EDE700BF10B5037866
:10F2B000023B012B0446037E02D913F0060F5AD1FC
:10F2C00098063AD494F91A30591C0AD02D4A03F5FD
:10F2D000B17302EB0313FF21DA796FF30002DA71E5
:10F2E000A17694F91B305A1C0FD0264A03F5B1734E
:10F2F00002EB0313FF20DA79C2F34501013921EA59
:10F30000E17161F34602DA71E076237E1B070BD5CB
:10F310001C4841F2C873C35C072B01D0FFF760FCA7
:10F3200041F2C8730022C254E26A0023237084F8B9
:10F330002830FAB1BDE81040104700231249E069B7
:10F340001A018A58904206D001330B2BBAD01A0109
:10F350008A589042F8D10B4A03F5B17302EB0313BC
:10F36000DA79C2F34501013921EAE17161F346021C
:10F37000DA71A7E710BD0121FFF760FF0128F9D17D
:10F38000237E9DE72C590020446F002030B1027885
:10F3900022B190F828201AB1002070470120704750
:10F3A00010B5D0E90142A242C16238BF2246032112
:10F3B000826080F82810FFF779FF012010BD00BFA0
:10F3C0002DE9F04FDFF868918A4699F80010DAF8D5
:10F3D00000300229174683B0834641F6300240F0E0
:10F3E0008B8059F80250DEB2A6EB030805EB13251B
:10F3F000B8444FF480729044BB4208F1FF38B8FB28
:10F40000F2F875D2A844032906EB0704A4EB030421
:10F410000CBF80224FF48072944228BF1446A8EBA0
:10F42000050366B994422CBF0A220B2201A9284683
:10F43000FFF746FC012809D003B0BDE8F08F0B228E
:10F4400001A92846FFF73CFC0128F5D199F80020D6
:10F45000DAF80010022A01F1010321D0A64210D2ED
:10F46000019906F18042013A081F00EB840001EB8C
:10F47000820242F8043F824203F10103F9D1DAF833
:10F480000010A61B7318BBF1010FCAF800301BD087
:10F490009F4205F101052BD999F800100026B2E72B
:10F4A000A642EED2DDF804C006F10042013AACF10A
:10F4B000020000EB44000CEB420222F8023F9042B3
:10F4C00003F10103F9D1DCE7BB42E1D199F8003047
:10F4D000022B21D004F18044019B013C4FF0FF320C
:10F4E00043F82420DAF800309F4205F10105D3D813
:10F4F000012003B0BDE8F08F59F8022003F07F0629
:10F500000329C3F3D415A6EB03081544B84414BF6C
:10F510004FF4807280226EE704F10044019B013CAD
:10F520004FF6FF72584623F8142003B0BDE8F08F61
:10F530002C5900202DE9F04190F838300446032B77
:10F5400051D8DFE803F002323B462D4BC0681978F2
:10F55000E76A03F5C252032911680CBF80264FF4F5
:10F56000807601FB06F141F2C47C00EB412041F2C0
:10F57000A87841F2AC7E53F80C20E06053F80E00FE
:10F5800053F808502261A5EB4125A0EB41219019C9
:10F5900043F8085043F80E1043F80C00C4E90C205F
:10F5A0005FBB6262012384F8383016480021FFF700
:10F5B00045FE012811D1022384F83830626B04F132
:10F5C00030010120FFF7FCFE012806D1032384F857
:10F5D000383000212046FFF731FE431EDBB2012BFD
:10F5E00002D9BDE8F081022094F82830062B04BF30
:10F5F000002384F82830BDE8F081921B2263D1E714
:10F600002C590020CC7000202DE9F04FDFF8248128
:10F6100098F80060012887B08CBF00230123032ED7
:10F6200002930C460B68154639D0022E62D14FF476
:10F6300080724FEA1329DFB201920138012823D8E2
:10F64000012203929D421AD9384E06F1880A06F12A
:10F650001C0B32681AB1DBF8001099424ED0DAF870
:10F66000000000234844092205A9FFF729FB0128CF
:10F670001FD002280FD020B123689D42E9D8256011
:10F68000032007B0BDE8F08F87B1FFF7A9FA022089
:10F6900007B0BDE8F08F022007B0BDE8F08F8022F0
:10F6A0000192C3F3D41903F07F07C6E7019A0392CE
:10F6B000C8E7DDE902C1059ADDF804E098F80030FA
:10F6C000022B14D0032BE6D152F8273023F07043DD
:10F6D000B3FA83F35B0963450F44236823D00B44DB
:10F6E00077452360EAD309F101090027C5E732F81D
:10F6F0001730EDE74FF480720192D2E70C490968A8
:10F70000013A02EB41224902B2FBF1F203991344A0
:10F71000B3FBF1F201FB12320AB10B449B1A9D427A
:10F72000236096D8ABE7AB42ABD3A8E7D4700020F8
:10F730006C7100202C590020F0B5104D2B7841F64B
:10F740003002022B0BBF070AC0F3D417C4B200F07B
:10F750007F04A85883B00E4600230322384401A931
:10F76000FFF7AEFA012807D12B78022B019B0CBFC3
:10F7700023F8146043F8246003B0F0BD2C59002036
:10F780002DE9F04390F83C30002983B0044614BFC3
:10F7900002210021042B7BD8DFE803F0030C3C4757
:10F7A0006900FFF74BFD012870D1626B002A75D10B
:10F7B00084F83C00404EDFF80881404D4FF6F77763
:10F7C0001DE01FFA80F9B94594BF4FF000094FF0D2
:10F7D000010901A9B9F1000F46D1FFF789FB012802
:10F7E000494650D1206BFFF7A7FF01284BD1019B61
:10F7F0002A682363013B934228BF13462B6033786A
:10F80000206B032BDDD1404594BF4FF000094FF032
:10F810000109DEE7426B04F130010020FFF7D0FD63
:10F82000012833D1032384F83C30234BE16A41F2B1
:10F83000C47003F5C2521D581268195041F2A877DE
:10F8400041F2AC76D8596D1A995902FB05F200EBDA
:10F85000422501EB422203F5BD500021DD519A51B2
:10F86000FFF7ECFC012811D1042384F83C3094F814
:10F870002830042B04BF002384F82830A36B8BB1FD
:10F8800020469847012003B0BDE8F0830228FAD152
:10F8900094F82830042B09D00220F4E7022384F8DE
:10F8A0003C30B8E7012003B0BDE8F083002384F8C2
:10F8B00028300220E7E700BF2C590020707100209B
:10F8C000F7FFFF0F38B590F834300446052B46D8C3
:10F8D000DFE803F01F033F101963006B4FF0FF31A7
:10F8E000FFF72AFF01283AD1E06A002839D1032323
:10F8F00084F8343000212046FFF7A0FC01282ED1E7
:10F90000042384F8343094F82830082B2DD00120BB
:10F9100038BD41F63803224DEA5800F13001023279
:10F920000120FFF771FE012824D00238C0B201285F
:10F9300015D8052384F8343094F82830082B04BFF8
:10F94000002384F8283041F2E5730122EA540220B2
:10F9500038BDC06A216BFFF7EFFE0128C7D0002039
:10F9600038BD022384F83430F4E7002384F82830CB
:10F97000012038BD05F5C252E3681168D4E90B20B7
:10F9800003EB412341F644016850C4E9033002B956
:10F990006062012384F83430A0E7014DCCE700BF5A
:10F9A0002C5900202DE9F04F436883B0C3F30808B9
:10F9B0001646002A00F0E180714B05468946A3F106
:10F9C000180B4FF0000AC8F5007495F91A70B4428C
:10F9D00028BF3446791C28462ED0F8F771FC0BEB73
:10F9E000071341F218629B58984205D0FFF7F8F8C8
:10F9F000504603B0BDE8F08F614B03EB4720224631
:10FA00004946404451F0B2FC002221462846FFF707
:10FA100029FBA2440028EBD02B7E1B0706D5594BAF
:10FA20002A691B689A4201D3FFF7DAF8361BA14412
:10FA30004FF00008C7D1DBE7F8F71EFC002849D1DA
:10FA40002846F8F73DFC6968C1F308032BBB21F495
:10FA5000FF7323F0010303F50072AB689A422CBFD9
:10FA6000062207222B7E03F00C030C2B1CD0002354
:10FA700001A9FFF725F90128BAD10198404BC31A13
:10FA800048BF03F2FF13B3F5B05F4FEA63224FD2D2
:10FA900057B2AF760028B2D1AAE72B7E03F00C0351
:10FAA0000C2B4FF00702E2D19BF800C0364BBCF1A3
:10FAB000030F1B680CBF4FF0800C4FF4807C03FBDE
:10FAC0000CF34FEA432C0CF1FF3C0CEA0101A3EBD1
:10FAD0005123CDE72B7E1A072ED59BF800102A4B19
:10FAE00095F828201B6803290CBF80214FF48071F2
:10FAF00003FB01F3062A4FEA43233FF479AF23497E
:10FB00000868834230D891F83D30002B7FF470AF05
:10FB1000002A7FF46DAF6B6985F83820062185F8DF
:10FB20002810EB622846FFF705FD012888D05FE723
:10FB3000FFF756F80198ACE7154B1A78002A7FF4C6
:10FB400057AF95F82820002A7FF452AF082185F896
:10FB5000342085F82810D3F85F206B692846C5E962
:10FB60000B32FFF7AFFEE0E741F2E57301225046AA
:10FB70000BF8032003B0BDE8F08F924638E700BFD2
:10FB800044590020F07000206C710020D4700020D7
:10FB9000117100202DE9F04390F8384083B00546FC
:10FBA000032C00F2A180DFE804F0021A8B0BFFF7B0
:10FBB00089FE012811D002280BD1032385F83830A3
:10FBC0002B6C002085F82800002B00F089809847D6
:10FBD0000224204603B0BDE8F08385F838002B7876
:10FBE000022B79D0414A6F6841F64803D3581F4031
:10FBF000C7F34F272846F8F763FBDFF8F480064683
:10FC00003F1A0AE0D8F800305A1E91454AD2FFF751
:10FC1000B5F908B9FEF7E4FF0136022201A9002375
:10FC20003046FFF74DF8BC1901281FFA84F94FF44C
:10FC300000724FF000010446CBD1019851F0F7FB60
:10FC4000EB694FF400712846002BDBD06B68002B6A
:10FC5000D8D1019B4FF020324FF02E0C1A605A6021
:10FC600083F800C0C3F807204FF0100E6C6A1A62C8
:10FC70005A6283F820C083F821C0C3F8272083F894
:10FC80000BE0EA6B5C83C2F30F4CC4F30F4483F8C0
:10FC90002BE05A879C82A3F834C0D8F800305A1E53
:10FCA0009145B4D3C3EBC353590201F50071284603
:10FCB000FFF764F908B9FEF793FF022385F838309F
:10FCC0002B6C002285F8282063B128469847012430
:10FCD000204603B0BDE8F0836F68C7F34F2789E77C
:10FCE000022476E7012474E7002472E72C590020EF
:10FCF0006C7100202DE9F04F90F8303089B0044647
:10FD0000042B00F2A880DFE813F0A900B200050080
:10FD10008A00E800B64D41F61003EB5C002B40F082
:10FD20009A80B44F04F11C09B84607F1380BBA4663
:10FD300001AE324649464046FFF70EFA012840F030
:10FD400018810198002800F0FA800378E52B01D093
:10FD5000002BEED1A84A821A48BF02F2FF12B2F578
:10FD6000B05F4FEA622380F03C811B01A34A134439
:10FD70009A7B042A0CD041F2C86104266A580132E9
:10FD80006A5041F2CC615A609E736B5801336B50DC
:10FD900041F60202AB565E1C09D003F5B17305EBC8
:10FDA0000313FF26D979AE546FF30001D97141F6E0
:10FDB00003016B565A1C0ED003F5B17305EB031308
:10FDC000FF26DA796E54C2F34501013921EAE17167
:10FDD00061F34602DA712022002151F028FB23460C
:10FDE000019A53F8311F58685060116019899B7A45
:10FDF00093721181019B627EDA7205A844F08CFE39
:10FE0000BDF81430002B40F02F8144F2817201992B
:10FE100003200A82CB810A83CB8284F83000237EC0
:10FE2000980600F1A9802046FFF736F92369002BD8
:10FE300000F0AE80237E03F0F70213F00403227675
:10FE400040F0B480122A00F0BA80002384F82830F1
:10FE50002046E36A984709B0BDE8F08F6548FFF790
:10FE60001BF94FF6FF720123228484F83030614F72
:10FE700004F11C0801AE04F131093246414638460E
:10FE8000FFF76AF901282FD00228E4D1584D41F636
:10FE90000202AB56591C09D003F5B17305EB0313ED
:10FEA000FF20D979A8546FF30001D97141F60301FD
:10FEB0006B565F1C0ED003F5B17305EB0313FF20E7
:10FEC000DA796854C2F34501013921EAE17161F33D
:10FED0004602DA71042384F830300020E36A20708F
:10FEE000984709B0BDE8F08F019D0B22494628468E
:10FEF000002D00F087802B78002B00F0838095F890
:10FF00000BA01AF0080FB8D151F0BDFA0028B4D1F7
:10FF1000637E8AEA0303DB0640F1C780344D41F675
:10FF200002016B565F1CC1D003F5B17305EB0313DF
:10FF3000FF26DA796E5460F30002DA71B6E73B7897
:10FF40002F49022B4FF009025046C3D00B78002BEB
:10FF5000C0D1C1E905330A708BF800304A6B0B73CE
:10FF600051F8143CC1E90132FFF714FE01283FF4B7
:10FF7000E0AE0228AED06EE7E0690023112205A9A9
:10FF8000FEF79EFE01283FF44EAF09B0BDE8F08FAA
:10FF9000237E19077FF559AF154A41F2C873D15C2A
:10FFA00000297FF458AF0721D1544EE70023E26ABD
:10FFB000A16884F828302046FFF754F84BE7626ABE
:10FFC000E06AA0630421C4E90233C4E90B2284F887
:10FFD0003C30636384F8281063622046FFF75CF8C6
:10FFE00039E7FEF7FDFD01986FF00F03BEE600BF95
:10FFF0002C5900201471002044590020446F002027
:020000040801F1
:100000003C710020474D41F60202AB565E1C09D000
:1000100003F5B17305EB0313FF20D979A8546FF3EF
:100020000001D97141F603016B56581C0ED003F53F
:10003000B17305EB0313FF20DA796854C2F345016D
:10004000013921EAE17161F34602DA71237EDA06B1
:100050007FF540AF3448FFF71FF84FF6FF720223D9
:10006000228484F8303056E6304B05A9B3F92C2AA7
:1000700002A844F0A5FD9DF80C309DF80D609DF898
:100080000A509DF80B20BDF808109DF80E00DB0209
:1000900043EA461342EA4512A1F2BC7143EA500317
:1000A00042EA41229BB292B2B1E6A98A6B8B204A06
:1000B00043EA014312686362EB69A3605202B3FB37
:1000C000F2F102FB113109B113445B1A154DE360E3
:1000D00041F6020184F819A06B565E1C09D003F5A5
:1000E000B17305EB0313FF20DA7968546FF3000254
:1000F000DA7141F603016B56581C0ED003F5B1734B
:1001000005EB0313FF20DA796854C2F34501013986
:1001100021EAE17161F34602DA71032384F8303099
:100120007DE600BF2C59002014710020483C0020BF
:100130006C7100202DE9F04390F82830013B83B02A
:100140000446082B41D8DFE803F048054D525865B6
:10015000406A4300384B4668056B41F6480103F599
:10016000C2525F5813683740EA19B2EB432F4FEA87
:10017000432816D258E02169207EFEF7E1FE0128CF
:1001800023D1256B666823696361A5EB08053D44AF
:100190004644F61B019B6660A84525634F462361D4
:1001A00042D82046F8F768F801AA81460028E2D034
:1001B0006668A368E26A9E4238BF1E460023A660B6
:1001C00084F828300AB12046904703B0BDE8F08398
:1001D000FFF7E0FC03B0BDE8F083FFF78BFD03B051
:1001E000BDE8F083FFF762F803B0BDE8F0830021BB
:1001F000FFF7C6FA03B0BDE8F0830121FFF7C0FAAC
:100200000128E2D10023216C84F828302046FFF732
:10021000BDF8DAE7FFF78EF903B0BDE8F083FFF72A
:1002200051FB03B0BDE8F0832046F8F725F800281D
:10023000BFD12E446660BCE72C59002010B5114C8C
:1002400094F89A3923B9104B4FF480225A6110BDAB
:100250000E4A136823F0060313604DF00BF894F870
:100260009A39002BEFD0D4F8A0399B68DB07EAD588
:10027000D4F89C2A136823F0030161F30703136089
:10028000E1E700BF502B0020003C014010ED00E0F2
:100290002DE9F04704460D469046002144221E46B3
:1002A000089F51F0C4F801234FF6FF72267662834F
:1002B00084F828302B782E2B4CD02E4604F1310AAE
:1002C000307804F1390968B12E280BD041F010F9CB
:1002D000C0B20AF8010BCA4506F1010607D0307812
:1002E0000028F1D120200AF8010BCA45F7D1307857
:1002F0002E2808BF707804F1380908BF013604F1D0
:100300003B0A58B141F0F4F8C0B209F8010FD145E9
:1003100006F1010607D030780028F3D1202009F833
:10032000010FD145F7D118F0100F14BF032301239B
:1003300084F819802370E7622B782E2B26D16B78F6
:1003400023BB0323204684F83030FFF7D3FC20463C
:10035000BDE8F0876B78002BAFD1114B41F2F472FE
:1003600041F60C0041F2F0719A5818585958E26061
:1003700041F601026062A1609A5C627641F2E87225
:100380009B5C2370E7622B782E2BD8D0002320466D
:1003900084F83030FFF7AEFC2046BDE8F08700BFA0
:1003A0002C59002008B50121032003F0E5FB72B6AB
:1003B00048F0EAFB2DE9F04F8DB0CE4CDFF84893C2
:1003C000CD4D00904FF0000854F80B0C002800F0C1
:1003D000FE8037F07BF80646002800F0D881D9F877
:1003E000A03844F8073CE0260023C44F04F8033C3F
:1003F000A4F10B0B06FB08F654F80B0C37F066F86B
:10040000002800F0E48054F80B0C37F057F814F88B
:10041000023C5A1E82460B2A0DD8DFE812F01F005C
:100420003A004600530083009B00E30016013501AB
:10043000400177018E0124280CD0009A3AB995F832
:100440004229824240F07F81012204F8032C0D2BC7
:10045000D2D186E0012304F8023CCDE700234D28E9
:10046000C4F8C53084F8CD3084F8CE3004D0582894
:1004700008D004F8023CBFE7022204F8022C84F8FA
:10048000C430B9E7032304F8023C022384F8C430E3
:10049000B2E704233C2804F8023C0BD0BAF13E0F2B
:1004A0000CD0002304F8023CA6E70A233C2804F8F9
:1004B000023CF3D1002304F8013C9DE7012304F83A
:1004C000013C99E7D4F8C500BB190344421CC4F8A9
:1004D000C52083F8EFAF94F8CD00022A8AEA000124
:1004E00084F8CD1088D12378C02BDAD86278FF2A1F
:1004F00008D1052BD5D9012384F8C430072304F88B
:10050000023C79E7A4F8C12000229342C4F8C93024
:1005100014BF0523062384F8C320C4F8C52004F8BB
:10052000023C69E7D4F8C500BB190344421CC4F877
:10053000C52083F8EFAF94F8CD00D4F8C9308AEA2B
:1005400000019A4284F8CD107FF456AF062304F8D8
:10055000023C51E794F8CD308342A2D10D2304F838
:10056000023C14F8017C002F40F0F380644B0894A7
:100570000FCB04AE86E80F00D4F8C930D4F8D10010
:10058000ADF82C7023440993B4F8C130ADF828308D
:1005900094F8C3308DF82A3001238DF82E3032467E
:1005A00003AB08A9039730F091FB48B1049B059376
:1005B00094F8C420534B0493314658462EF0A4F8C7
:1005C000039E002304F8023C002E40F0D88008F17E
:1005D0000108B8F1030F04F1E0047FF4F5AE0DB0AB
:1005E000BDE8F08FD4F8C500BA190244431CC4F822
:1005F000C53082F8EFAF94F8CD2094F8CE00019387
:100600008AEA0202514684F8CD2044F06FFD019B36
:1006100084F8CE00072B7FF4EFAEB4F80530C02B82
:100620003FF63FAFB4F80320A4F8C120A27884F8C5
:10063000C32000229342C4F8C93014BF0823092301
:10064000C4F8C52004F8023CD6E6014694F8CE0072
:1006500044F04CFD94F8CD3084F8CE008AEA0303D0
:10066000D4F8C50084F8CD30BB190344421CC4F84B
:10067000C52083F8EFAFD4F8C9309A427FF4BCAEFE
:10068000092304F8023CB7E694F8CD30434084F8DF
:10069000CD3094F8CE3083427FF403AF56E7D4F8E0
:1006A000C500BA190244431CC4F8C53082F8EFAF44
:1006B00094F8CE000193514644F018FD019B84F854
:1006C000CE00052B7FF498AEB4F80120B4F80330C7
:1006D000A4F8C120227884F8C32000229342C4F8F1
:1006E000C93014BF0B230C23C4F8C52004F8023C06
:1006F00082E600BF3F3B0020483C0020502B0020FA
:10070000C41806087C100120581A0020014694F8ED
:10071000CE0044F0EBFC84F8CE00D4F8C500BB1941
:100720000344421CC4F8C52083F8EFAFD4F8C930A5
:100730009A427FF461AE0C239BE694F8CE3083425C
:100740007FF4AFAE0AE7232804BF022204F8032C8B
:100750007DE6012F4FF0000602D004F8026C36E768
:10076000D4F8C93008942344099308A8B4F8C130D8
:10077000CDE90A66ADF828302DF044F9EDE754F8DC
:100780000B0C2EF0FFF954F80B0CB0471FE714F8D0
:10079000033C002B3FF41BAFD9F8A02854F8071CEA
:1007A000521A632A7FF613AF012B31D0022B7FF44C
:1007B0000EAF54F80B3CC5F8303AC5F8343AC5F8DA
:1007C0003C3A402385F8403A124BC5F81C380122C8
:1007D000C5F8843A95F8A73185F82E2A0E4AC5F84F
:1007E000382A003B0D4A85F8410A18BF01230C48FE
:1007F00082F8B03B3DF0C2F84FF4005030F030F9D1
:1008000008483DF0B1F885F8886A85F8896ADEE61F
:10081000FFF7C8FD80460020713F04081400001057
:1008200095A10608CBA10608202301480B8070473C
:1008300030040020642301480B80704750040020DE
:10084000432301480B807047B404002010B5074CC7
:10085000D4F8C800FF2807D0054951F8042BF7F752
:1008600069FCFF23C4F8C830002010BD300400200C
:1008700080710020EAE700BF08B5D0F8E4355B6A74
:100880009847002008BD00BF08B5D0F8E4351B6AC2
:100890009847002008BD00BFD0F8E43510B50446E5
:1008A0001B689847D4F8E8359B689847002010BD2E
:1008B00008B5D0F8E435DB6903B19847002008BDDE
:1008C00008B5042290F81211D0F8E83580F8131119
:1008D00080F81221DB689847002008BD10B5D0F8D9
:1008E000E83504461B699847032384F81231002039
:1008F00010BD00BF0B0630B41CD401EB810200EB2D
:10090000C202002300EB810582F8741382F875336C
:1009100001241A4604FA01F16D6D61F31F42016969
:100920006FF3CF332B60CB6923EA0203002030BC86
:10093000CB61704701F07F0101EB810400EBC4043F
:10094000012200EB8105002384F81C1184F81D218D
:1009500002FA01F11A46AD6961F30F02DFE700BF49
:1009600010B581210446FFF7C5FF20460121FFF79E
:10097000C1FF024B0020187010BD00BF5846002078
:1009800010B581210446FFF7B5FF20460121FFF78E
:10099000B1FF82212046FFF7ADFFF7F711FC0020E1
:1009A00010BD00BF38B50D4604468321FFF7A2FFF6
:1009B00029462046FFF7E4FF002038BDF0B4164674
:1009C0000A063AD401EB810500EBC5052824002274
:1009D00004FB0104022B85F87413C5F87C6385F8C9
:1009E000773385F8752304F55D7448D0154600EB20
:1009F0008107012202FA01F17F6D61F31F45D7F8EB
:100A000000C01CF4004F11D1E488204946F0805208
:100A100042F4004242EA834204F00F041C4B42EAD3
:100A2000845211400CEA0303194339600269D36907
:100A30002B430020F0BCD361704701F07F0101EB34
:100A4000810500EBC5052824012204FB0104022BCB
:100A500085F81C11C5F8246185F81F31A5F822110D
:100A600085F81D2104F58E740CD0002500EB81075C
:100A7000012202FA01F1BF6961F30F05BFE722719C
:100A80001546B4E700252571F0E700BFFF87CC13BA
:100A9000007833EC002310B5194604464022FFF7D6
:100AA0008DFF8021204600234022FFF787FFD4F8E6
:100AB000E835A078012284F812215B68984700206D
:100AC00010BD00BF70B44B78012B26D00B784A695B
:100AD00000EB83035C6D25682369D2B18A684A61A3
:100AE00002F07F0223F4002323F07F0342F400226C
:100AF00013432361C378012B04BF0B696361C5F302
:100B0000076363F07B0363F31F652560002070BCFF
:100B100070478A6802F07F02E4E782694C691568D1
:100B2000136944B38E68B4428CBF06F07F0404F0AE
:100B30007F0423F4002323F07F0344F4002443EADA
:100B4000040388BF4E611361C378012B1DD0C5F328
:100B5000076464F07B0464F31F651560002BD5D136
:100B60004B69002BD2D002690878516B0123834076
:100B70000B435363CAE723F4002323F07F0343F4BA
:100B800000231361C378012BE1D10B780C6900EBD2
:100B90008300C5F30763816963F07B0363F31F651B
:100BA0004C610020156070BC704700BF2DE9F04318
:100BB0004B78012B30D00B784C6900EB83035E6DD2
:100BC000356837691CB38B681C44013CB4FBF3F4F3
:100BD000C4F3090203FB02F3C3F312034B6114468F
:100BE00043EAC44363F31C073761C378012B04BF96
:100BF0000B697361CB78012B44D0C5F3076363F0B5
:100C00007B0363F31F6535600020BDE8F0838A68CD
:100C10000124C2F31203E3E791F800804E6900EB70
:100C2000880EDEF818C0DCF80050DCF8107076B3DF
:100C3000D1F80890384A06EB0904013CB4FBF9F4FA
:100C400002EAC444C6F312022243CC7807F060479C
:100C50003A43012C174649D0CCF81020C278012A1B
:100C600055D00269516B03FA08F30B435363C5F384
:100C7000076363F07B0363F31F65CCF8005000202B
:100C8000BDE8F0834B7973B345F00055B5E707F045
:100C9000604747F40027CC78CCF81070C378012B5C
:100CA0002FD0012CE3D102699268D20554BF45F0E0
:100CB000005545F08055C5F3076262F07B0262F390
:100CC0001F65CCF80050002B9ED1B0B203308010CD
:100CD000DEF8D04098D0CA6852F8041B2160013376
:100CE0009842F9D190E745F0805586E764F35E7746
:100CF000CCF81070C378012BD5D10A69CCF8142038
:100D0000D1E70A69CCF81420012CB0D1CBE70B69EC
:100D1000CCF81430ABE700BF0000F81F0E4BDA68C8
:100D2000D20310D4DA68D1060FD4DA68D20510D411
:100D3000DA6812F0E00F0AD1DB6813F0020F14BF7B
:100D400008200920704701207047062070470720BF
:100D500070470220704700BF003C024000207047EF
:100D6000704730B1034B93F90C000028D4BF00202A
:100D7000012070478071002008B5FFF7F2FF50B1E5
:100D8000054A537B927B5B0003F00203002A18BFE5
:100D900043F001030B6008BD8071002008B5FFF728
:100DA000E0FF10B1014B1B690B8008BD8071002072
:100DB00070B5FFF7D6FF78B1084A958A65B1966994
:100DC0000023B3421C4607DA02EB44040133A48B30
:100DD000AC42DBB2F5D30B7070BD00BF8071002058
:100DE00008B5FFF7BEFF10B100230B70137008BDEC
:100DF0000420704728B1034B93F9CC00003818BF8A
:100E0000012070473004002008B5FFF7F3FF50B110
:100E1000054B93F9CC20012AC3BF93F8CF30C3F31D
:100E200040030B60002008BD3004002008B5FFF728
:100E3000E1FF18B1024B93F8CE300B7008BD00BF34
:100E40003004002070B5FFF7D5FF38B10E4C94F890
:100E5000CF30DB0703D500230B70137070BD0B4D33
:100E600094F9CD3095F82C6093FBF6F301330B70B9
:100E700094F9CD4095F82C1094FBF1F301FB13434A
:100E800001331370EAE700BF3004002080710020B6
:100E90000320704770B50A4A92F8303006255E1C70
:100EA000B6FBF5F405FB146492F83150AC4205D062
:100EB00002EBC303C3E90D0182F8304070BD00BFEF
:100EC00080710020002230B504461046914200DCBB
:100ED00030BDA35C0825584010F0800F4FEA400356
:100EE00018BF83F0D503013DD8B2F5D10132EDE74B
:100EF00010B5D9B10E4B586E814217DCB2B1DB6A26
:100F00009A4213DC0B4C013A013903FB012184F8AE
:100F1000DA1004F1D6000521FFF7D4FF062184F88A
:100F2000DB0004F1D600BDE81040B3E710BD00BF00
:100F300080710020300400200023038083708380B0
:100F4000C3800372704700BF074A084992F86830AF
:100F500009780133DBB2994282F8683004BF00237C
:100F600082F86830704700BF80710020700A00105E
:100F7000F8B5774CE36E83B1764B1B6893F82E304F
:100F80005BB1754B94F87020A3FB0013012A4FEA64
:100F900093132FD0022A08D002B1F8BD6F4B9842AC
:100FA000FBD9012384F87030F8BD626F64329A4235
:100FB0003CD894F8683004EB031393F8E824FF2A34
:100FC00006D067490132012083F8E82481F8DC006B
:100FD000FFF7BAFF634B1B780122092B84F87020BE
:100FE000DBD1B4F86A35604A01339BB2A4F86A35A4
:100FF0005380F8BD94F868105A4863678C2303FB4C
:101000000143007883F88A20002384F8863004F1B5
:101010007C050A2202230928A56784F8872084F822
:101020007030BAD1504B01311980F8BD94F8862048
:1010300094F887309A42B0D104F17B0004F1840522
:10104000002310F8012F082153405A0013F0800F9D
:1010500008BF5B0082F0070214BFD3B2DBB20139D4
:10106000F3D18542EDD194F885209A4239D194F894
:10107000686094F8835094F88430B4F87F00B4F832
:10108000812094F87DC004EB061743EA052394F809
:101090007E5087F8E81440BA52BA81B292B245EA5B
:1010A0000C202F4DC7F8EC141BB294F97C10C7F834
:1010B000F024032E4FF00102A7F8EA04A7F8F43455
:1010C00087F8E91485F8DC2008D8264A12780C2A1B
:1010D00029D00D2A02D1244B23F81610FFF734FF34
:1010E0005FE794F8683004EB031393F8E824FF2AD1
:1010F00006D01B490132012083F8E82481F8DC0086
:10110000FFF722FF174B1B780122092B84F8702070
:101110007FF443AFB4F86835134A01339BB2A4F8A7
:1011200068359380F8BD1149114A897E0E4803EB5A
:10113000830303EB830349089B0093FBF1F382FBDA
:101140000312DB17C3EBA20320F81630C6E700BF7B
:10115000807100205C090010D34D62103F4B4C00A1
:10116000300400205D32002060320020002B00207F
:10117000676666660A4B93F8861093F8872091425B
:101180000DD010B493F886209C6F511CD2B2C0B21F
:10119000C9B283F88610A0545DF8044B70477047BD
:1011A00080710020FD2870B522D0F02804D0EF28EF
:1011B00022D00224204670BD114D0320052641286F
:1011C0002E444FF0000405F1010580F080030DD09E
:1011D000042B0BD9FFF7E6FF2044B542C4B2E9D097
:1011E00015F8010B412880F08003F1D10420F3E7CA
:1011F000044D0B200426E2E7034D0C200626DEE713
:10120000EC1D0608E81D0608F41D06080E4B0F4AE3
:10121000D3F86C35B2F900005B0707D400EB80000F
:10122000400080B200F5C87080B27047084B094A90
:101230009B6B323382FB0312D817C0EBA20080B243
:1012400000F5C87080B2704780710020C80B001094
:10125000CC330020676666660C4AD2F8843530B419
:101260001C68D2F87C555D6019810025611C1960ED
:101270009D812070D2F88435D2F87C151A685A60A6
:101280004FF6F67230BC19609A8170478071002069
:10129000114B30B4D3F82827C3F82C2703F5B160DD
:1012A00003F5C36103F5C16503F5E3640132C3F8D7
:1012B0008055C3F88445C3F8282730BCC3F87805A7
:1012C000C3F80806C3F80C06C3F87C15C3F8181752
:1012D000C3F81C17704700BF8071002000B583B0B1
:1012E0000268084B8188CDF801203222D3F83037CC
:1012F000ADF805108DF800206846984703B05DF8FA
:1013000004FB00BF807100205E2810B511D05D285D
:1013100005D00D4BBDE81040D3F8343718470A4CC0
:10132000D4F834379847D4F834373D20BDE810401E
:101330001847054C5D20D4F834379847D4F8343733
:101340003E20BDE8104018478071002030B40123D2
:101350004FF4807515244FF4167140F2D932038092
:10136000002345808471018130BC42818380838168
:101370007047134B10B400220F2483F83A17090A60
:1013800083F8390783F83B17C3F83C27C3F8402795
:10139000C3F8442783F8384703F5E760012110F8C4
:1013A000014F013122440E29D2B2F8D183F84627E9
:1013B0000449D3F848075DF8044B102236F056B8BC
:1013C00080710020B8780020054B002183F84C176D
:1013D000C3F85017D3F8483703B1CAE7704700BFC6
:1013E0008071002013B50446FFF704FD08B3002305
:1013F0000DF106022046ADF806300DF0CBFAC0B173
:101400000D4C9DF8062094F9CC1084F8E1200329B6
:1014100008BF62F07F024FF00501084808BF84F85A
:10142000E120FFF74FFD062184F8E2000348FFF7B3
:1014300031FD02B010BD00BF300400200D050020BA
:10144000034B0449B3F9E4304068012247F08CB9FA
:101450003004002043A2060806494068B1F854272A
:10146000D1F85C370449534342F2107293FBF2F215
:1014700047F07AB980710020D0A10608044A0549D6
:101480005378127840680133013247F06DB900BFDC
:10149000EC3D0020D5A106082DE9F84F1B4C054670
:1014A0001E2094F868A794F869B794F86A67B4F8AE
:1014B0006C97B4F86E8794F8707720F0E9FE30B13D
:1014C000B8F1000F03D0C14601264FF0000A94F88E
:1014D0007237DA070AD494F877273AB9012F12D075
:1014E000022F03D113F0020F08BF012685F800A0D8
:1014F00085F801B0AE70A5F80490A5F806802F72AB
:101500002846BDE8F88F3E46F0E700BF8071002016
:101510002DE9F84F2DED028BFFF76CFC002844D02D
:10152000254B93F9CC0001283FDD93F8E640DFF826
:1015300090809FED228A0FF2780BDBE900AB154615
:101540008E1E02EB44094D4504D1BDEC028B2046B2
:10155000BDE8F88F38F8027B26F8027F07EE907A14
:10156000F8EEE77A67EE887A17EE900A4CF08EF87C
:1015700052465B464CF0E2F841EC100B4FF088FC11
:1015800051EC100B4CF002FC0E2F80B20AD919302E
:101590003223B0FBF3F080B200EB800000EB800060
:1015A000400080B225F8020BCDE70024CDE700BF54
:1015B0001655B5BBB16B024030040020CDCCCC3DFC
:1015C0001C79002038B50D46FFF714FC044638B1ED
:1015D0000C4890F8CF30DB0704D5B0F8D000288055
:1015E000204638BD084A90F9CD3092F82C2093FB64
:1015F000F2F102FB113201320131E8300DF0DEF977
:10160000EDE700BF300400208071002038B5134C96
:1016100094F8313094F830209A4219D004EBC30387
:101620000F49D3E90D200023984212DC93780D4A2C
:10163000C4F8AC075B081370FCF7C0FB94F83130BA
:1016400006210133B3FBF1F201FB123384F8313090
:1016500038BDD55C01F8015B0133E5E780710020FE
:10166000CC450020FA450020F0B52C4CD4F8B057FA
:1016700094F8681787B0074628460DF005FA94F8E5
:101680006917064628460DF0EBF90022059294F8FA
:101690006A278DF81320034675B1039005A92846E3
:1016A0000DF004FA94F87027039B2AB10DF1130191
:1016B00028460DF001FA039B9DF81320DDB1D2B14D
:1016C000A1698A4217DC04EB8204D4F8B44703937F
:1016D000262020F0DDFD0599039B70B911F0010F64
:1016E00014BF502200228907786808D50C4947F0BA
:1016F0003BF807B0F0BD0B4CE9E74422F3E732B109
:10170000CDE900420849324647F02EF8F1E7074993
:101710000094324647F028F8EBE700BF80710020C4
:10172000DBA1060816A90608E3A10608EFA1060832
:101730002DE9F04FA84B1B788BB08146002B40F071
:10174000B380A64DD5F8B067002E00F0AD80A44A56
:10175000D2F8EC4004F0F021B1F1E02F6DD1C2F8E5
:10176000EC30D5F8D827944267D004930593ADF8B0
:101770001830B5F86C3795F868E7ADF8143095F87F
:1017800069C795F8703795F86AA78DF818300DF18C
:1017900010088DF810E08DF811C08DF812A098E8AF
:1017A000070007AB03C38F4F1A80C4F342533B4477
:1017B000C4F30342997CC5F8D8478E4502F1010273
:1017C00001D1944508D030468DF81C108DF81D20AD
:1017D0000DF0F4F8ADF8200030460DF017FC0328AA
:1017E00004F0070B34D0042835D000239A4501A912
:1017F000304618BF8DF81E300DF058F948B1019BE6
:10180000C4F3001103F001038B4202D030460DF007
:10181000F1FA0A2207A940464FF0E1FD68B19DF8B0
:101820001E30BDF81C2085F86A37BDF82030A5F8B9
:101830006827A5F86C373EF0FFFF95F8DCA704AFEA
:1018400095F8DC37032B79D8DFE803F0083174A171
:101850005F44FB7DCAE75F44FB7FC7E739463046FC
:101860000DF02AF9044658B107A8FFF715FE9DF8B8
:101870001E109DF810308B4260D030460DF030FBCA
:1018800095F8DC37013303F0030385F8DC370CB936
:101890009A45D5D195F87237DB0700D524B1336866
:1018A00049461B68304698470BB0BDE8F08F01A849
:1018B000FFF7F2FD95F872879DF8044008F00108E3
:1018C000ECB1B8F1000F39D13A460DF103013046C1
:1018D0000DF0F5F8044688B307A8FFF7DDFD9DF885
:1018E0001C109DF803309DF81D208B4203D19DF8FC
:1018F0001030934222D030460DF0FCFAC0E7B8F128
:10190000000FBDD1394630460DF0D3F80446A8B1DA
:1019100007A8FFF7C1FDBDF82010BDF810308B42BD
:101920000CD085F8DD8785F8DE87336830469B6903
:101930009847A5E795F87237D80701D500249FE7A7
:1019400007A930460DF0B2F804460028F6D01E2054
:1019500020F09EFC95F8DF3783428046EED085F874
:10196000DF0760B1B5F86E37002BE7D1079BD907C9
:10197000E4D4012130460DF03DFA444680E7079B50
:10198000DA07DBD5014630460DF034FA78E7384601
:10199000FFF782FD97E8070007AB03C31A809DF8A5
:1019A00010309BB10DF11D0207A930460DF087F8EC
:1019B0000DF11E0130460DF07FF80A2207A93846C6
:1019C0004FF00DFD041E18BF012459E708A9304649
:1019D0000DF06FF8ECE700BF764600208071002024
:1019E00030040020E81D0608024B0146D3F8E0074A
:1019F00035F070BD807100202DE9F041FD2984B0E3
:101A0000044600F0DE80F02900F0BD80EF2900F0F0
:101A100031814AB10346861803AD002003F8010B5B
:101A20009E4205F8010BF9D19A4B0B2003F10905F1
:101A300001E013F8010F814200F0C880AB42F8D1F9
:101A40004B1E832B00F29380DFE813F03201390143
:101A500043014E01BE018400580163016F019100F2
:101A600091007501750175018B018B018B016F016F
:101A70009100910096019E019100910091009100CA
:101A800091009100910091009100910091009100CE
:101A900091009100910091009100910091009100BE
:101AA00091009100910091009100910091009100AE
:101AB000910091009100910091009100910091009E
:101AC000910091009100910091009100B40191006A
:101AD000910091009100910091009100910091007E
:101AE000910091009100910091009100910091006E
:101AF000910091009100910091009100910091005E
:101B0000910091009100910091009100910091004D
:101B1000910091009100910091009100910091003D
:101B2000910091009100910091009100910091002D
:101B3000910091009100910091009100910091001D
:101B4000910091009100910091009100910091000D
:101B50001F011F01504BB3F82C18002900F06681BB
:101B600001922CF0B9FA019A80B2ADF80C003AB1AA
:101B7000224403AB13F8011B04F8011BA242F9D164
:101B800004B0BDE8F081454F03214FF00508B8448B
:101B9000002501370CE0FFF705FB064660193246C9
:101BA000FFF72AFF70194745C5B2E9D017F8011BA6
:101BB000412981F08003084601D0042BEBD804268C
:101BC000ECE7374F0B214FF00408E0E7324BD3F836
:101BD0006C0580060CD4002AD2D0224403AB13F843
:101BE000011B04F8011B9442F9D104B0BDE8F08157
:101BF00093F8E407870742D52A4D287D052834BF8E
:101C000002260326142917D97C39C8B20628E2D83F
:101C10000629E0D801A050F821F000BF051E0108F8
:101C2000051E0108EF1D0108D71B0108151E01083C
:101C30000F1E01081B1E01080929CCD90A390A29DF
:101C4000C9D801A757F821F0D51D0108211E0108A8
:101C5000D71B0108D71B0108D71B0108D71B010898
:101C6000D71B0108D71B0108D71B0108E71D010876
:101C7000051E01080C4F0C214FF0060887E7094BA1
:101C80000B29187DA7D10126CBE0084B5B6B039392
:101C90006DE700BF101E060880710020EC1D0608CD
:101CA000E81D060810450020F41D0608CC3300206E
:101CB0000192FFF7ABFA019AADF80C0057E76C4BB5
:101CC000D3ED037AFDEEE77A17EE903AADF80C30DB
:101CD0004DE7684B93F8F307B3F85417002840F02A
:101CE000AB80ADF80C1042E76249B1F8543791F877
:101CF0000C18B3FBF1F3ADF80C3038E75D4D95F8F7
:101D00007237DE0700F19D80B5F82C38ADF80C3045
:101D10002DE7584B5849B3F9403881FB0301DB17D5
:101D2000C3EBA103ADF80C3021E7524BB3F84238B6
:101D3000ADF80C301BE7514BDFED516AD3ED017A62
:101D40000C39C9B203EB810393ED157A67EEA67ADD
:101D500067EE877AFDEEE77A17EE903AADF80C3031
:101D600005E7444B03EB4101B1F81E3803EB830355
:101D70005B00ADF80C30FAE63E4B93F8723703F097
:101D80000103ADF80C30F2E63A4BB3F83A18CD0542
:101D90005ABFCB4303F00103032311F0440F18BFD4
:101DA000042311F0020F18BF072311F4806F18BF2E
:101DB0000923ABE70192FFF729FA324B019ADB6B5B
:101DC00043EAC0400390D2E62A4BD3F85C37ADF823
:101DD0000C30CCE62B8A03EB830303EB83039B00DD
:101DE000ADF80C30F7E6EB89ADF80C30F3E6EB8993
:101DF000254903EBC3039B00A1FB03135B09ADF86B
:101E00000C30E8E6B3F8E637ADF80C30E3E66B6883
:101E10000393E0E62B680393DDE6AB680393DAE611
:101E2000F6B28DF80C608DF80D00D4E6D3F8640797
:101E300080F3100080B298E693F80C38B1FBF3F110
:101E40004FE705F50165019220F034FCD5ED037AEA
:101E5000019AFCEEE77A17EE903A9BB200287FF4E5
:101E600055AF0A49096811F0100F18BF00234DE75C
:101E7000907900208071002067666666C80B0010AC
:101E800000007A44CC3300201F85EB5144440020ED
:101E900070B5214D95F84438EA181C4692F8482848
:101EA0008AB11E4E09225C1CA6FB04135B0803EBDF
:101EB000C303E31AE918DCB291F8481809B1013AF2
:101EC000F1D185F8444802681549561C06600C2675
:101ED00016700268561C0660002616700268561CB2
:101EE000066003EB430603EB8603147019440D22CE
:101EF0003DF09CFE95F84418084B4A1CA3FB0203D6
:101F00005B08294403EBC3030120D31A81F8480876
:101F100085F8443870BD00BF80710020398EE338E9
:101F2000D47900202DE9F041684ED6F8B07784B01E
:101F3000044638460D460DF069F886F8C90857B1D1
:101F40000DF1090202A938460CF0B9FD002840F055
:101F50008E8096F8C9080023ADF808308DF80A3055
:101F60001A46431EDBB20021FF20FD2B8DF80C200A
:101F7000ADF80E108DF80B0003D9002004B0BDE8B9
:101F8000F0819DF80830042B00F09680052B00F0BE
:101F90009980032B00F09880022B00F08C80012B9D
:101FA00008BF042100F088809DF809309DF80A10D0
:101FB000D6F8B007013B0DF10E028DF809300CF098
:101FC000E9FC96F8C938032B73D0042B0CD1404A96
:101FD0009DF80A000121002301E012F8011F81424F
:101FE0006DD20133082BF8D1D6F8CC28029B394F9B
:101FF0009A420DF108084FD023680D22591C216028
:102000001A7023680022591C21601A7023689DF8F9
:102010000820591C21601A7023689DF80920591C5A
:1020200021601A7023689DF80C20591C21601A70D9
:1020300023689DF80A20591C21601A70BDF80E1003
:1020400020463DF03BFE23689DF80B20591C216083
:1020500020461A700721FBF799FA98E8030087E8F1
:1020600003000120C6F8D45804B0BDE8F08101A9EE
:1020700038460CF01BFD00283FF46BAF38460DF1DD
:102080000A010CF019FD00283FF463AF019B96F89C
:10209000C90803F0010264E77A68D8F804309A426C
:1020A000AAD1D6F8D4380C4AEB1A93427FF665AF22
:1020B000A2E70A4A8CE703218DF8081074E78DF82F
:1020C0000A3091E70121F7E70221F5E7807100204E
:1020D000071E06084C7A002080841E00FF1D06089B
:1020E0002DE9F0412A4C2B4AD4F85C37B4F8D87863
:1020F000B4F8646782FB0352DB17C3EBA2031FFA39
:1021000083F8474582B00D4603D1B4F8DA38B342BC
:1021100033D002680190511C3423016013700268AF
:102120000023511C0160137041463DF0C7FD01982A
:1021300031463DF0C3FD019847F6FF713DF0BEFD0D
:10214000019847F6FF713DF0B9FD019847F6FF7120
:102150003DF0B4FD019847F6FF713DF0AFFD0198E9
:102160000221FBF713FA0120A4F8D888A4F8DA6852
:10217000C4F8DC5802B0BDE8F081D4F8DC38064A77
:10218000CB1A9342C5D8002002B0BDE8F08100BF51
:10219000807100206766666680841E00026810B544
:1021A0007F21541C0460117002680024511C0160DE
:1021B0000E211470FBF7EAF9012010BD2DE9F04F54
:1021C000C24B1B68804613F0800083B000F0718121
:1021D000BF4B93F8E40710F0020000F06A81DFF8CB
:1021E00010B39BF81430052B40F26881DBF8003007
:1021F000B84D0093002BB8BF5B42A5FB0342B64825
:10220000B649920D00FB0233C3EB03139B0085FB21
:10221000034502EB8202DC1702EB8202C4EBA554F9
:1022200000FB043304EB8204A4B281FB0321DB171F
:10223000C3EBA111BCB10025A94F2E46A7FB043268
:10224000D20802EB8203A4EB4303E8B2A4469BB29C
:1022500080008340BCF1090F94B246EA030605F101
:102260000105EBD8340489B2B9B100259C4F2E4644
:10227000A7FB0132D20802EB8203A1EB4303E8B2D1
:102280008C469BB280008340BCF1090F91B246EAB4
:10229000030605F10105EBD83443DBF804E08D4D6E
:1022A0008D4E8E498EEAEE70A0EBEE70A5FB0032EB
:1022B000920D06FB0200C0EB0010830085FB03506B
:1022C00002EB8202DD1702EB8202C5EBA05506FB92
:1022D000053305EB8205ADB281FB0321DB17C3EBB0
:1022E000A111C5B10020DFF8F8C10646ACFB0532EC
:1022F000D20802EB8203A5EB4303C7B2A9469BB207
:10230000BF00BB40B9F1090F95B246EA030600F1E0
:102310000100EBD8350489B2C1B10020DFF8C0C19B
:102320000646ACFB0132D20802EB8203A1EB430369
:10233000C7B289469BB2BF00BB40B9F1090F91B249
:1023400046EA030600F10100EBD83543DBF808301C
:10235000634A0193002B1846B8BF5842A2FB0030D5
:10236000604E6149030AA6FB0363DB0901FB03F12D
:10237000C1EBD00189B2B9B1002691463746A9FB1D
:102380000132D20802EB8203A1EB4303F0B28C4688
:102390009BB280008340BCF1090F91B247EA03076A
:1023A00006F10106EBD8B9B2BBF81070DFB1002618
:1023B000DFF82CA1B446AAFB0732D20802EB820355
:1023C000A7EB43035FFA86F938469BB24FEA8909C7
:1023D00003FA09F3092897B24CEA030C06F1010647
:1023E000E9D81FFA8CF7BBF812303D4AA2FB03066E
:1023F000F608632E28BF6326092B63D90020934675
:102400008146ABFB0632D20802EB8203A6EB430304
:102410005FFA80FAB4469BB24FEA8A0A03FA0AF3DB
:10242000BCF1090F96B249EA030900F10100E8D8AE
:102430005FFA89F9009B019A002BCCBF392338231E
:102440001616BEF1000F26F07F0635DD274A33430E
:10245000964543F00206C8BF43F00606D8F80030A0
:102460001622581CC8F800001A70D8F80030002254
:10247000581CC8F800001A7040463DF01FFC214669
:1024800040463DF003FC294640463DF0FFFB4046F8
:1024900039463DF013FCD8F800305A1CC8F800202B
:1024A00083F80090D8F800305A1CC8F800200120AA
:1024B0001E7003B0BDE8F08F1E43CFE7002003B0CD
:1024C000BDE8F08F4FF00009B4E700BF444400209E
:1024D000807100206BCA5F6B806967FFD34D62100B
:1024E000CDCCCCCCC55A7C0AA0860100FFC99A3B52
:1024F000104500202DE9F047AB4B1B68064613F052
:10250000800084B000F09E80A84B93F8E40710F0A0
:10251000020000F09780A64F397D052940F2978090
:10252000632900F292800024DFF898C289B2254620
:10253000ACFB0132D20802EB8203A1EB4303E0B211
:102540008E469BB280008340BEF1090F91B245EAEE
:10255000030504F10104EBD8EDB2BB68954A82FB98
:102560000312D917C1EB623189B2002900F018813A
:102570004FF0000CDFF84CE26446AEFB0132D208AB
:1025800002EB8203A1EB43035FFA8CF088469BB217
:1025900080008340B8F1090F91B244EA03040CF1C2
:1025A000010CEAD8E4B2FB8983494FF4F36707FBD7
:1025B00003F7A1FB0737C7F38F1742F20F739F4250
:1025C00049D8CFB10020DFF8FCE18446AEFB0732EA
:1025D000D20802EB8203A7EB4303C1B2B8469BB219
:1025E00089008B40B8F1090F97B24CEA030C00F157
:1025F0000100EBD81FFA8CF7704BD3E9002313438B
:102600003ED14FF0FF3833681722591C31601A70E1
:1026100033680022581C306039461A7030463DF04D
:102620004DFB414630463DF031FB33685A1C326069
:102630001D7033685A1C326030461C700621FAF750
:10264000A5FF012004B0BDE8F087992585E70020AB
:1026500004B0BDE8F0870021DFF868C10F46ACFB8D
:102660000302D20802EB8200A3EB40039BB28B4033
:102670000431102947EA030793B2F0D1BFB2BBE798
:1026800001A842F049FA9DF80810002900F08A805C
:102690004FF0000CDFF82CE1E046AEFB0132D2082F
:1026A00002EB8203A1EB43035FFA8CF089469BB2F5
:1026B00080008340B9F1090F91B248EA03080CF198
:1026C000010CEAD84FEA08289DF80910E1B1002072
:1026D000DFF8F0E08446AEFB0132D20802EB820361
:1026E000A1EB43035FFA80F98A469BB24FEA89095E
:1026F00003FA09F3BAF1090F91B24CEA030C00F1A5
:102700000100E8D848EA0C089DF80A104FEA0828AA
:10271000E1B10020DFF8ACE08446AEFB0132D20824
:1027200002EB8203A1EB43035FFA80F98A469BB276
:102730004FEA890903FA09F3BAF1090F91B24CEA99
:10274000030C00F10100E8D848EA0C08BDF80C3091
:102750001B49632BA1FB03214FEA08184FEA5111D3
:102760007FF651AF0020DFF85CE08446AEFB01321B
:10277000D20802EB8203A1EB43035FFA80F98A4699
:102780009BB24FEA890903FA09F3BAF1090F91B232
:102790004CEA030C00F10100E8D848EA0C0832E7E3
:1027A0000C4600E788468FE74444002080710020F3
:1027B0001045002089B5F814D34D6210607A0020CE
:1027C0001F85EB51CDCCCCCC08B5A0F10103B3FAF9
:1027D00083F302284FEA531301D0184608BD0F2097
:1027E0001FF0CEFC30B9064B93F8723703F00103AB
:1027F000184608BDBDE808400F201FF049BD00BFC6
:10280000807100202DE9F04F194E90F801808578F5
:10281000DFF86090DFF860B085B00446371D4FF4F4
:10282000FA6A16F9013B002B18DB39F91320A2F5DF
:102830007A724FF47A730AFB02F292FBF3F202AB64
:10284000A2F57A725946184645F08EFF02AB009306
:102850002A460023414620460AF030FA0135BE429E
:10286000EDB2DED10023237305B0BDE8F08F00BFC9
:10287000C37A0020A4450020EAA5060810B5044646
:1028800022F014FD0349034604226068BDE81040AD
:1028900045F06ABF43A20608037840680122053B61
:1028A000114609F061BEF8B50446274B417882789D
:1028B00093F8090923780138302B244B4FEA800024
:1028C000034423480BBF93F8325093F8345093F8E5
:1028D000336093F8356030F9153030F9160040F266
:1028E000CF75AB42A8BF2B46B3F57A7FB8BF4FF484
:1028F0007A73A8424FF47A77A8BF2846A3F57A7373
:10290000B842C3EB0313B3FBF7F3C3F10E03B8BF35
:102910003846DBB24FF0030CB3FBFCFC0CEB4C0E67
:10292000A3EB0E03A0F57A706244C0EBC00008333D
:10293000B0FBF7F73944DBB2D2B2C9B22046FBF79D
:1029400031FA00232373F8BD80710020E81D0608CA
:10295000A44500202DE9F04790F8029090F80180FE
:1029600009F1020704460026FFB2002508EB060A1B
:10297000032E1BD108F10301022DC9B20ED10B2386
:102980003A462046FBF70EFA0135052DF0D1013607
:10299000072EEAD100232373BDE8F08709EB050277
:1029A0001623D2B22046FBF7FDF9EDE7022DEBD15D
:1029B00017233A465FFA8AF12046FBF7F3F9E3E77B
:1029C000406809F035BE10B5044614F0ABF8642237
:1029D00002FB00F3C3F38F23632B60680349BDE858
:1029E000104028BF6323012245F0BEBE51A5060852
:1029F0001E4A9FED1F7AD2F86417B2F8E838406893
:102A000007EE901AF8EEE76A07EE903AF8EEE77AEA
:102A100067EE877AF4EEE76AF1EE10FA02D815490C
:102A200045F0A2BE8B4202DA134945F09DBE5B1A07
:102A300007EE903A02F51563B8EEE77AD3ED007A27
:102A40000E4AF8EE677A3C2167EE277A87EEA67A7F
:102A5000FDEEC77A17EE903AB3FBF2F3B3FBF1F257
:102A600001FB1233064945F07FBE00BF8071002094
:102A7000CDCCCC3DF8A10608FEA1060840420F00CF
:102A800004A20608034B04491A684068143209F08E
:102A9000E7BD00BF8C4500200EA20608034B044989
:102AA0001A684068083209F0DBBD00BF8C45002081
:102AB00012A20608034B04491A6840680E3209F056
:102AC000CFBD00BF8C45002016A2060837B51C4CB0
:102AD0004568D4F86C2512F0200F02F0040328D0CA
:102AE00094F8E427920724D5B4F9420809F068FC69
:102AF0006421002890FBF1F301FB13014FF00A0061
:102B000091FBF0F194F8ED08B4BF7622752200290C
:102B1000B8BF494200280CBF99209F20002BCDE967
:102B20000010B8BF5B420749284645F01DFE03B0C0
:102B300030BD002BD8D12D222A7042685370F6E7A1
:102B4000807100201AA20608014B1B681B6A1847F7
:102B5000DC3A0020024B186808B1836918477047B7
:102B6000DC3A0020024B186808B1436918477047E7
:102B7000DC3A002010B5074C606D40B139F026F901
:102B800094F8513013B180F00100C0B210BD0120A3
:102B900010BD00BF581A002030B40A490A480A780C
:102BA000531CDBB20525042B00EBC20400F83250A5
:102BB00008BF00234FF404520B7062604FF0FF30E7
:102BC00030BC70472446002028460020037870B4AB
:102BD000FBB10446C0F10106A31914F8015FDBB292
:102BE000002DF9D101335B00DCB2032513800C709A
:102BF0004D7004785CB1022300255A1CD2B2CC542B
:102C00008D5410F8014F0233DBB2002CF5D170BCAB
:102C1000704702242346E8E70B0617D401EB810333
:102C200000EBC30310B400EB81000124002283F801
:102C3000764383F8741383F87523426D5DF8044B73
:102C4000136843F4001300201360704701F07F0104
:102C500001EB810300EBC303012200EB810083F849
:102C60001C1183F81E2183F81D2182691368002B33
:102C700001DA43F0804343F40013136000207047EF
:102C800070B501F07F0505EB850400EBC404282135
:102C900001FB05010126C4F830310023C4E94A22B2
:102CA00084F81C5184F81D61C4F8343101F58E712B
:102CB0001DB9FDF707FF002070BDFDF777FF00206D
:102CC00070BD00BF2249F8B5D1F854390F2B04D09C
:102CD0005A1CC1F854290020F8BD1E4C2578002349
:102CE000C1F85439002DF6D11B4E1C4B3268B2F599
:102CF000006F17D01B689A4227D017D9C2F500631E
:102D0000402B15D9403B02F14005C1F85839012349
:102D10002370356092B2402311490A448121FFF7A4
:102D2000AFFFD8E71B6835607BB12A469B1AE7E7FF
:102D30004FF0000502EB0307C1F858590CBF022100
:102D40000121376092B22170E6E700232370C2E7C9
:102D500080710020FC220020D0220020D4220020FC
:102D600000230020AEE700BFF8B51D4C2378012BEF
:102D700003D0022B09D00020F8BD01461948D0F835
:102D8000583953B923700020F8BD00231A46812119
:102D9000FFF776FF00232370F5E7402B11D9124C83
:102DA0002268403B02F14005C0F85839256092B2D4
:102DB00040230E4C084622448121FFF761FF00208A
:102DC000F8BD094D2A684FF0000603EB0207C0F872
:102DD000586908BF02202F6092B208BF2070E8E750
:102DE000FC22002080710020D0220020002300203F
:102DF00038B5134602250A46C0E94E3380F8115112
:102E00000021FFF73DFF002038BD00BF10B50C7852
:102E100014F0600413D0202C0AD14B78023B092B0C
:102E200018D8DFE803F01B21171717171717272EDD
:102E300022490122FFF7DCFF0024204610BD4B7819
:102E4000062B24D00A2BF3D01D4B8A78C3F86429B3
:102E5000204610BDFAF7E4FF0224EEE719490122EB
:102E6000FFF7C6FF0024E8E717490122FFF7C0FF7C
:102E70000024E2E74B88124A1B0AC2F8603900249A
:102E8000DBE70F4B8A78C3F85C290024D5E74B8831
:102E90001B0A222B0CD0212B04D021462246FFF7FF
:102EA000A7FFCAE7CA880949092A28BF0922F6E705
:102EB000CA880749362A28BF3622F0E7E47A00207C
:102EC00080710020E07A0020DC7A00206A05002072
:102ED0002005002038B501EB810400EBC4040D4649
:102EE000002184F87453C4F88C1384F87513C4F863
:102EF0008833C4F88023C3782821012B01FB050106
:102F000008BFEDB201F55D7108BFC4F884231DB997
:102F1000FDF7D8FD002038BDFDF748FE002038BD84
:102F2000144B9A6870B5044662B1134A1B7B92F841
:102F300068592B4316D081212046FFF76DFE022DE4
:102F400009D070BD0C4B93F8685981212046FFF7DA
:102F500063FE022DF5D12046064ABDE870401F23CE
:102F60000121B7E70121FFF757FE20468121BDE887
:102F7000704051E6044600208071002070B5094A77
:102F8000094D1173094B13600021044629700D236C
:102F90008121FFF775FE2046054ABDE870401F23DA
:102FA000012197E7644600205846002055534253BC
:102FB0000446002010B5064B597B0446FAF73EFF45
:102FC000002800DB10BD20460121BDE81040D5E7F8
:102FD000044600202DE9F041314D2C7834B1012C0C
:102FE00001D1FFF7E7FF0020BDE8F0812D4FDFF8AA
:102FF000D080B0F8B4337A68C8F804201F2BBA68C0
:10300000C8F80820064606D1274B3A689A4202D1F2
:10301000797B01291AD9254A25491378052401F815
:10302000334001EBC3000133DBB2042B08BF0023A4
:103030004FF4005113701F4B41600222304683F859
:103040006829FFF76DFF0020BDE8F081BB7B013BE5
:103050000F2BE0D8FAF7F2FE002819DB2B78013BA2
:10306000022BC0D9144B1988B1B1BB68D8F808201D
:1030700088F80C408B4228BF0B46D11A0424C8F8AC
:1030800008100E4A2C7030468121FFF7F9FDAAE79F
:103090003046FFF745FFA6E73046FFF76FFFA2E790
:1030A0005846002004460020555342432446002041
:1030B00028460020807100204C4600202C4900202A
:1030C0006446002008B5084B1B78022B07D0033B51
:1030D000012B02D80021FFF751FF002008BDFFF7A8
:1030E00069FF002008BD00BF5846002010B501EB65
:1030F0008101084A00EBC1010446B1F88C13104667
:10310000F4F7F0FF034A204640230121FFF7E2FED7
:10311000002010BDEC7A0020E8E700BF70B50A7807
:1031200012F060050C46064611D0202D16D1CD8830
:10313000D5B113062AD52A461F496078F4F7FAFF5D
:10314000E2881D493046FFF753FE00250AE04B7820
:103150000A2B16D00B2B0ED0062B03D13046FAF7D4
:103160005FFE0225284670BD022260781144F4F704
:10317000E1FF284670BD8B78D3B9104BC3F8AC592A
:10318000F0E70F490122FFF733FEEBE70D496478C2
:103190000A4AC1F8C8400321C0E9E45542F8045B7B
:1031A0002B4680F811110021FFF794FE0025D9E786
:1031B000FAF736FED6E700BF847100208071002048
:1031C0002C7B0020300400200B7803F00303012B3C
:1031D00003D0022B04D0002070478B881BB915E662
:1031E0008B88832BFBD099E710B50223044640223D
:1031F0008121FDF7E3FB2046022340220121FDF758
:10320000DDFB8221204603230822FDF7D7FB064B76
:1032100002229A80F4F7DCFF044A20464023012171
:10322000FFF758FE002010BDA0010020EC7A00201E
:1032300038B509220D46044603238321FDF7BEFB62
:1032400029462046FFF7D0FF002038BD82B000237A
:10325000016801930B6901930E4B03E00A69019227
:10326000013B13D0019A002AF8DA019A094B42F087
:1032700001020192019A0A610A69019203E00A6956
:103280000192013B02D0019AD207F8D4002002B08B
:10329000704700BF400D0300436D064A1A61C278B3
:1032A000012A06D100F2CC5058614FF080221968F3
:1032B0001A6070471800086010B500230422044605
:1032C000194680F811211A46FFF7DAFC2046FFF76D
:1032D000E3FF002010BD00BF10B5044629B990F8E7
:1032E0001131032B0DD0002010BDD0F8E4359B69BF
:1032F000002BF8D090F81221032AF4D1984700202F
:1033000010BDD0F89013D0F87C33994214D9C0780E
:10331000D4F880230128A1EB030104BFD218C4F81C
:1033200080238B4228BF0B46C4F890139BB22046E3
:103330000021FFF7CFFDD6E7D0F8E4351B691BB1BC
:1033400090F81221032A03D02046FFF7B5FFCAE701
:103350009847F9E7F0B5012190F8D17590F8D36559
:1033600090F8CFC590F8CE5590F8D03590F8D2258A
:1033700080F8111190F8CC1585B005EB0C2503EB06
:10338000072302EB062201F01F06AFB292B290F8BB
:10339000CD558DF808109BB2012E0446ADF80A7089
:1033A000ADF80C30ADF80E20C0F840218DF8095072
:1033B00017D0022E1FD036B101F08001FFF72CFC90
:1033C000002005B0F0BD092D0FD8DFE815F0BF00D3
:1033D000AC000E00D5000E00EA0085000E0077005C
:1033E000540090F81221032A2FD02046FAF718FD36
:1033F000002005B0F0BD01F060012029DAB234D020
:10340000012D00F02081032D00F00681002DD7D181
:1034100090F81211022900F0DF800329E5D11B0684
:1034200000F14B8102EB820200EBC20393F876338A
:10343000002B00F04D81BF4B0122C3F8C029BE49CB
:1034400020460222FFF7D4FCBAE7DAB2012ACCD830
:10345000D0F8E43502A99B689847BDF80E30002BE0
:10346000AED12046FFF728FFAAE7D0F8E43502A93D
:103470009B689847A4E7F9B2AE4D012985F8B019C9
:10348000B3D890F81231022B00F02781032BACD176
:10349000002900F0868190F810110129E1D0D0F8C0
:1034A000E4355B68984795F8B01984F81011204608
:1034B000FDF7F2F92046FFF7FFFE81E7012A94D1DC
:1034C00090F81231022B00F01781032B8DD100F5FB
:1034D0008871FFF78DFC73E73D0A022DADF80620D9
:1034E00000F05081032D00F00B81012D7FF47DAFA2
:1034F000D0F8EC3580781B680DF106019847BDF8CF
:103500000620002A3FF45CAFBDF80E30002B3FF4DC
:1035100057AF9A4228BF1A4601462046ADF806200A
:10352000FFF766FC4CE790F81231023B012B3FF6A7
:103530005CAF012F7FF444AFD0F8E43500229B68E4
:10354000C0F8182102A9204698478AE790F812315E
:10355000023B012B3FF649AF764BD0F818210021F2
:10356000C3F8B81912B10222C3F8B829734920462A
:103570000222FFF73DFC23E7012F00F09880022F85
:103580007FF41EAF13F0FF0F7FF41AAF02691B0A1E
:10359000023B5268032B00F21D81DFE803F039354E
:1035A00031241A437FF421AF90F81231032B3FF4FA
:1035B0001CAF036907F07F0580F81451196867F3A1
:1035C0000A120A431A60FFF777FE002D00F0E5802B
:1035D000022384F81231F3E651063FF4F1AE1146AE
:1035E000FFF71AFBECE6052363F30612514B0121AA
:1035F00084F816112046C3F8BC29FFF75DFEDFE60C
:10360000042363F30612F1E7032363F30612EDE7E5
:10361000022363F30612E9E790F81231022BDBD0A4
:10362000032B7FF4E2AE27B9550602D01146FFF70F
:10363000F3FAD4F8E43502A99B682046984720465F
:10364000FFF73AFEBCE690F812110229C4D0032914
:103650007FF4CBAE002F7FF4B3AE12F07F013FF4C6
:1036600000AF180600F1A78002EB820304EBC3034E
:1036700004EB810083F8767383F8741383F8757311
:10368000282303FB0243416D03F55D73DA780B6871
:10369000023A6FF35553012AD4F8E42598BF43F05A
:1036A00080530B602046936802A99847D9E6D0F86A
:1036B000E435C0F818719B6844E702F07F0202EB22
:1036C000820200EBC20393F81E31002B7FF4B3AEED
:1036D000184B0022C3F8C029B1E600293FF4C1AE5F
:1036E0000121032380F8101180F81231FDF7D4F87E
:1036F0002046FFF7E1FD63E61149FFF779FB5FE63E
:10370000FDB2052D3FF671AEDFE805F0342C241C28
:103710000B03D0F8EC3580789B690DF106019847D2
:10372000EDE6D0F8EC3580785B690DF1060198473D
:10373000E5E600BF80710020407B0020387B002040
:10374000347B0020D0F8EC3580781B690DF1060140
:103750009847D4E6D0F8EC358078DB680DF10601A7
:103760009847CCE6D0F8EC3580789B680DF10601DF
:103770009847C4E6D0F8EC3580785B680DF1060117
:103780009847BCE6D0F8E43580789B6A0DF10601D5
:1037900098474570C4F8F005B1E6012384F812316A
:1037A0000EE60222D0F8E43580F8101180F81221DC
:1037B0005B68984755E6282202FB014304EB810031
:1037C00083F81E7183F81C1183F81D51816903F57C
:1037D0008E735BE7012363F3061207E770B50446B7
:1037E00049B990F81131022B1BD094F81631012BF6
:1037F0000DD0002070BDD0F8E4355B69002BF8D007
:1038000090F81221032AF4D19847002070BD2A4A6B
:103810002369D2F8BC295A60002384F816310020AD
:1038200070BDD0F83831D0F82451AB4217D9C278E6
:10383000012AD0F82821A3EB050308BF5219C0F8CC
:10384000383108BFC0F828219BB20021FFF718FAD1
:1038500000231A4619462046FFF73CFBC5E7D0F87F
:103860003C31B3FBF5F605FB163666B99D420AD826
:10387000D0F84021934206D233463246FFF700FA91
:10388000C4F84061E4E7D4F8E435DB681BB194F890
:103890001221032A0CD00023052284F81121194695
:1038A0001A462046FFF716FB2046FFF7F5FC9CE77B
:1038B00020469847EFE700BF8071002082B00023C8
:1038C0000193019A094B42F010020192C168019ADA
:1038D0000A610A69019203E00A690192013B02D080
:1038E000019AD206F8D4002002B07047400D0300C0
:1038F00082B000230193019A0B4B42F02002019207
:10390000019A61F38A120192C168019A0A610A69F7
:10391000019203E00A690192013B02D0019A9206EA
:10392000F8D4002002B07047400D0300F8B50B78C2
:1039300013F060050C4606461CD0202D17D14A789E
:10394000FE2A44D0FF2A3DD14A88002A56D1CD888C
:10395000002D53D11B0651D43749384B0D7001212E
:1039600083F86819364A1F23FFF7B4FA00E00025F0
:103970002846F8BD4B780A2B4BD00B2B44D0012B9B
:10398000F6D191F904308988002B47DBFFF796FFC9
:1039900021792A4F3046FCF7ADFF022321794022DE
:1039A0003046FDF70BF897F86839022B3BD094F9B5
:1039B0000420002ADCDA012BDAD030460121FFF79F
:1039C000DDFAD5E70225FAF72BFA2846F8BD4D882F
:1039D000A5B9CC88012C11D11A060FD5194B1B683B
:1039E0009B6998471549C0B281F8C40930B1224695
:1039F00001F6C4113046FFF7FBF9B9E7304602255E
:103A0000FAF70EFA2846F8BD0C4B4A8883F8C52908
:103A1000AEE70D490122FFF7EBF9A9E701F07F01BD
:103A2000FFF766FFB4E730468121FFF7F5F8002382
:103A300087F868399CE700BF584600208071002055
:103A40000446002048460020457B002038B5044647
:103A5000FCF786FF2046022340228121FCF7AEFFBF
:103A60002046022340220121FCF7A8FF0C4B0D4900
:103A70001B680D4A00250D701B6882F8685928469E
:103A800098472046FFF71AFF20460121FFF730FF35
:103A9000064A20461F230121FFF71CFA284638BD9D
:103AA000484600205846002080710020044600202F
:103AB000012905D008B50321FFF71AFF002008BD32
:103AC000FFF752B9104B70B4DA6843780178867802
:103AD0000E4CD243C2F30222C2F10405E8B2834085
:103AE0000F2040FA02F23240DBB2134360181B0190
:103AF00001F01F0501224909DBB2AA4080F800331A
:103B000044F8212070BC704700ED00E000E100E0C7
:103B1000C27802B1D6E7037805485A09203203F08B
:103B20001F03012101FA03F340F82230704700BF60
:103B300000E100E000B583B009238DF80730FDF700
:103B4000EDF88DF807009DF80730012BF7D09DF8B0
:103B5000070003B05DF804FB82B0064B002201921F
:103B60000193019B03EB80000190019B186802B058
:103B7000704700BF5028004082B0064B00220192DF
:103B80000193019B03EB80000190019B196002B03F
:103B9000704700BF502800400023C0E90033C0E94F
:103BA0000233C0E90433C0E90633C0E90833C0E991
:103BB0000A33C0E90C338363704700BF0B6870B4ED
:103BC000D1E90524CD682B431343D1E907252343CD
:103BD0001343D1E909422B43D1E90D652343134334
:103BE00004680B4A334322402B4313430360D1E95B
:103BF0000B3442690D6922F0070223431343D1E9D4
:103C0000014243614560846070BCC260704700BF80
:103C10003F801CF002683649002310B422F00102F4
:103C2000212488420260036043608360C3600361B3
:103C3000446138D02F4B98422ED02F4B98423CD025
:103C40002E4B984240D02E4B984232D02D4B98426A
:103C500041D02D4B984246D02C4B984217D02C4B3C
:103C600098423CD02B4B984216D02B4B984224D0F4
:103C70002A4B984228D02A4B98421AD0294B984276
:103C800029D0294B98422ED0284B984208D14FF08A
:103C90003D5243F8AC2C03E04FF4746243F8202CFF
:103CA0005DF8044B7047224B5DF8044B3D229A604F
:103CB0007047204A43F8642CF2E74FF474125DF821
:103CC000044B43F8382C70474FF074625DF8044B96
:103CD00043F8502C7047184A43F87C2CE0E73D220B
:103CE00043F8082CDCE7154A43F8942CD8E700BFCA
:103CF000106002402860024040600240586002406C
:103D00007060024088600240A0600240B8600240DB
:103D1000106402402864024040640240586402403B
:103D20007064024088640240A0640240B8640240AB
:103D3000006002403D000020400F002000003D20B8
:103D40000B88F0B433BB028C4C880E898B88C988F1
:103D500022F001021204120C0284058B028CADB217
:103D600025F0F30592B22B4322F00A0243EA061330
:103D700022439BB242F0010203830284038B23F0AF
:103D80000C031B041B0C0383038B9BB21943F0BC75
:103D900001837047042B048C2CD0082B4E888A8812
:103DA0000D89C98851D024F480542404240C04843F
:103DB000838B078C2C0344EA022440F6FF421A400E
:103DC00045F6FF733B4043EA063322439BB292B26F
:103DD00043F4805382830384828B22F44062120472
:103DE000120C8283838B9BB243EA01239BB2F0BC0B
:103DF0008383704724F010042404240C4D880F8919
:103E00008A88C9880484068B038C12029BB242EA1A
:103E1000073423F0A00340F6FF42324043EA051383
:103E200022439BB292B243F0100302830384028BBD
:103E300022F440621204120C0283038B9BB243EA09
:103E400001239BB2F0BC0383704724F480742404E4
:103E5000240C0484848B038CA4B29BB224F0F3045E
:103E600023F42063224343EA062342EA05129BB26D
:103E700043F4807392B282830384838B23F00C0318
:103E80001B041B0C8383838B9BB21943F0BC81837F
:103E9000704700BF214A038890429BB212D002F5BE
:103EA000806290420ED0B0F1804F0BD0A2F58032EC
:103EB000904207D002F58062904203D002F5806202
:103EC000904203D14A8823F070031343144A90426E
:103ED00018D002F58062904214D030B423F44073BD
:103EE0000C894D6802F56C429BB2234390420C88CA
:103EF0000380C56204850DD18B7A0386012330BC13
:103F00008382704703800B884A68C262038501235D
:103F100083827047034B9842EED0EFE700000140E8
:103F20000010004000040140224A936803F00C0393
:103F3000042B10B421D0082B22D01F4B03601D4C42
:103F40001E4AA168C1F30311114491F84C11CB40F2
:103F50004360A168C1F38221114491F84C1123FA06
:103F600001F18160A1685DF8044BC1F342310A445C
:103F700092F84C21D340C3607047114B0360DEE7D9
:103F80005468516852686302C2F388124CBF0C4BEC
:103F9000094B01F03F01B3FBF1F303FB02F3054AC8
:103FA0005268C2F3014201325200B3FBF2F30360E4
:103FB000C5E700BF003802400024F40030040020B0
:103FC00000127A002DE9F04700230F6801264FF018
:103FD000030C02E00133102B41D006FA03F232EA5F
:103FE0000704F7D1D0F800E05C000CFA04F52EEAE3
:103FF000050EC0F800E091F80490D0F800A009FA8E
:1040000004FE09F1FF394EEA0A0EB9F1010FA84684
:10401000C0F800E06FEA050515D8D0F808E005EA19
:104020000E0585604D79D0F808E0A54045EA0E05FB
:104030008560456825EA020242608A7945689A40AF
:1040400092B22A434260C26822EA0802C260CA7978
:10405000C568A24001332A43102BC260BDD1BDE820
:10406000F0870D4B93F87227D20703D5012283F80E
:10407000C629704793F8C62962B9D3F8B0274AB168
:1040800093F86827104493F8692783F86807114468
:1040900083F86917704700BF80710020044B93F9C3
:1040A0000C00012806BF02221A730020704700BFCF
:1040B00080710020114AD2F8C809A0B1D2F8CC39D9
:1040C0008BB188420DD88B4234BF002301239BB1B2
:1040D0001369C2F8D01999421CBF142382F8D4394D
:1040E000DCE70023F3E7A1F59C53083BB3F57A7FA7
:1040F0002CBF00230123EAE7704700BF8071002036
:1041000007B500230DF10602ADF806300AF042FCB7
:1041100060B1084BBDF80620998AA3F8D6299142D0
:104120001CBF142283F8D829FFF7B8FF03B05DF84D
:1041300004FB00BF8071002013B5044626200191C6
:104140001EF0A6F8019948B9054BD3F848372BB1B2
:10415000204602B0BDE81040FDF70BB902B010BD1B
:1041600080710020B1FA81F149094920E4E72DE985
:10417000F341BE4C94F90C3001330D4600F06681DA
:10418000D4F84837002B00F0B380022700264FF008
:104190000108D4F8480733F099F9002800F0A88006
:1041A000D4F8480733F08AF9D4F850375A1C23441E
:1041B000C4F8502783F8D90994F84C37012B09D05B
:1041C000022B15D063B90F280CBF84F84C87C4F8B4
:1041D0005037DEE7A0F17203012B06D9762804D010
:1041E00084F84C67C4F85067D3E784F84C77D0E77D
:1041F000102ACED19E490023012211F8010F01326D
:1042000003440E2ADBB2F8D194F8E72984F84C670E
:104210009A42C4F85067BCD194F8E839002BB8D161
:1042200094F8DA39732B59D0762B1BD0722B5FD1CF
:1042300094F8DC2994F8DB3994F90C1053EA022342
:1042400056D0C4F8C8390029B4F8DD39C4F8CC39DF
:104250004EDC94F8F62901232373002A48D184F810
:10426000F63945E094F8DC2994F8DB3953EA022367
:104270003ED0D4F8EC2994F8DE1994F8E2092361D1
:1042800093421CBF142284F8D42994F8DD29C4F881
:10429000EC3942EA0122B4F8F019A28291421CBF23
:1042A000142184F8D81994F8DF19617394F8E0198F
:1042B000A17394F8E119A4F8F02941EA0021A4F8C7
:1042C000F219D4F8D01909B9C4F8D039B4F8D639EC
:1042D0000BB9A4F8D6290223237309E094F8E02946
:1042E00094F8DF3943EA02231AB20BB1A4F8F42997
:1042F00094F90C30022B35D00FDCDAB2012A15D933
:10430000636E13B1A369002B6CD15A495A481F221E
:1043100002B0BDE8F0414DF0C8B8032BF0D1D4F89D
:10432000F839564AEB1A9342EADD13E0D4F8F8293B
:104330005349AA1A8A42E3DD2BB97220FDF744F8EB
:10434000C4F8F859DCE7D4F8FC395A1CD907C4F88A
:10435000FC2903D47620FDF737F8F1E77320FDF749
:1043600033F8EDE7D4F8D019D1B194F8D439BBB112
:104370002369994214D0637BDA0703D489B24620BB
:10438000FFF7DAFE94F8D439013B84F8D43905F507
:104390009225032305F578752373C4F8F859AFE720
:1043A000B4F8D619A38A81B194F8D8296AB18B429E
:1043B0000BD0637BDB0702D45020FFF7BDFE94F8DF
:1043C000D839013B84F8D839E1E701222273A4F8F7
:1043D000D6392269C4F8D029002384F8D83984F862
:1043E000D4398DE7274DD4F8B0772A2385F85C318E
:1043F0000DF1070220230DF10601384685F85D31E5
:104400000AF05DFB30B19DF806109DF8076051EA97
:1044100006031ED1552385F85E31462385F85F31AA
:1044200022691948202385F86031002A34D01749C1
:1044300044F09AF9B4F8F23915488BB3A28A1549B9
:104440009A420CBF20222A2244F08EF902B0BDE825
:10445000F08138460AF018FB314685F85E0138468F
:104460000AF0FEFA037885F85F31D9E78071002001
:10447000597B002028A206088C050020400D03006F
:1044800040420F00300400209105002083DA060826
:104490009505002042A20608034944F065F9C9E7E2
:1044A000024944F061F9D1E74AA2060849A2060888
:1044B00010B50E4C40F0080284F87F2194F9CC200E
:1044C000022A06DD420704D583071CBF012384F8B6
:1044D000D43005210648FCF7F5FC062184F880015C
:1044E000BDE810400248FCF7D5BC00BF30040020F6
:1044F000AB05002010B5FCF77DFCA8B31B4C94F96C
:10450000CC30012B30DD59B3022B2DD094F8D430B0
:104510009BB971B180230521154884F88531FCF7DA
:10452000D1FC062184F88601BDE810401048FCF754
:10453000B1BCBDE810400420BAE7002914BF002038
:10454000042094F8CF301A0748BF40F002005B0700
:1045500001D411B108B940F00100BDE81040A7E74F
:10456000022BD3D10420ECE710BD00BF30040020A3
:10457000B1050020F8B5224C04F28717030A84F82D
:104580008C0105460621384684F88B31FCF79AFCED
:1045900094F8CF3084F88D01DB072AD4B4F8D0200A
:1045A000AA4226D1174DD4F88731C5F8003AC3B2D4
:1045B00085F8063A41F26F714FF6FF738A4218BFD1
:1045C0000123134405F52066C3F307220621304674
:1045D00085F8042A85F8053AFCF774FC072185F86C
:1045E000060A3046FCF756FC052104F5C770FCF7B7
:1045F00051FCBDE8F84004480721FCF74BBC00BF64
:104600003004002080710020B705002008B5FCF7B9
:10461000F1FB48B1A1F59C53083BB3F57A7F03D277
:10462000BDE808400846A5E708BD2DE9F0476B4EF8
:104630003368002B3AD06A4D6A4C05F1CC073068DC
:1046400032F044FF002833D1674B198809291D46F1
:1046500009D95F8864227A43B2FBF1F2452A40F31C
:10466000A4811880588094F8413A012B00F0C88149
:10467000022B00F0E38133B95C480521FCF70AFC0A
:10468000012384F8413A5A4B1D685A4B1B78002B82
:1046900000F0DE81584B1B68EB1A782B40F2D88172
:1046A000D4F8AC07F9F78AFBC4F8445ABDE8F087A0
:1046B000306832F003FF94F8073A8046052BBED8E5
:1046C000DFE803F00309171D3745AA28B7D10123F6
:1046D00084F8073AB3E7552803D1022384F8073A50
:1046E000ADE7414A938801339380002384F8073A69
:1046F000A5E7032384F8080A84F8073A9FE71328FC
:1047000084F8090AC4F8240A07DD374AD38801333C
:10471000D380002384F8073A91E718B9052384F879
:10472000073A8CE70023C4F8283A042384F8073AB0
:1047300085E7D4F8283AE218013382F80A0AD4F857
:10474000242AC4F8283A93427FF479AFE6E7D4F8F4
:10475000243A2A4803F1020A4FFA8AF1FCF7B2FB25
:10476000804594F8089A40F0178126201DF090FDAE
:10477000204B48B100221A701B4A538801335380E2
:10478000002384F8073A5AE71A784A4519D10022DB
:104790001A7009F1FF33102B00F2F980DFE813F0F3
:1047A00030008E008E00E1008E00F700F700F70069
:1047B0003000F700F700F700F700F700F700F70008
:1047C0003000B9F1090F02D0B9F1110F01D1012A5E
:1047D000DDD0054A538901335381DAE7C84500200B
:1047E0003004002080710020EC450020BE05002030
:1047F000F8220020FA450020FC450020887B00209C
:10480000BAF1060F5ADDB9F1010F06D0B9F1090F5F
:104810000CBF4FF002094FF0030994F80D0A94F809
:104820000E1A94F80C2A94F90AEA94F90CCA94F82E
:104830000B3A85F8CC9041EA002109B2900785F83F
:10484000CDE085F8CFC0A5F8D01006D512F00C0F3A
:1048500014BF0122002285F8D420B9F1030F13D12F
:10486000BAF1090F2ADD94F9102A082AA8BF0822F4
:1048700022EAE27285F8E620002043B29A4200F173
:1048800001005CDC94F80F3AD4F818A0002002462E
:104890009BB2524590465ADB7D4B85F8CE001B7883
:1048A000232B0BD109EB89037A4A03EB83030CEB2F
:1048B00083031380A2F802E09180D0807649774884
:1048C0000A224CF08CFD10B1002384F8363A724B6A
:1048D0003A681A607A685A603A891A8194F8363AC6
:1048E00043BB95F8D43094F8682784F8382A002B15
:1048F00014BF0223012384F8363A95F8CF3094F898
:104900006A0784F83C0A13F001031CBFB2FA82F371
:104910005B0994F8692784F8392AD9B2B4F86C276E
:1049200084F8371AA4F83A2A13B10AB1A4F83E2A37
:1049300084F8401A0BF004F90BF002F91CE704EBC1
:104940004308234493F8123AA8F89C3795E704EB00
:1049500048080132B8F81C8052B2984508BF10468A
:1049600097E7BAF1040FA9DD94F80A2A94F80B3AF4
:1049700043EA022359041AB204D5C3F30D03A5F880
:10498000D2309BE7002AF8DBA5F8D03096E7444AFE
:10499000938901339381EFE619F0010F7FF4F0AEB4
:1049A0003F4A138901331381EAE63E4BD3F8942141
:1049B000B3F89811012A1AD141F25632914203D12B
:1049C0004FF0FF32C3F89421D3F89421306802EB02
:1049D000820202EB820201EB420189B2A3F8981134
:1049E00003681B69984700232B806B803BE60132EC
:1049F000EAD1B1F5965F04BF0122C3F89421E3E741
:104A0000284D95F9CC60002E3FF43DAE022E11D119
:104A10004FF48040FFF7AEFD84F8416A95F9CC3041
:104A2000012B7FF730AE95F8CF30C3F3400385F804
:104A3000D43028E6032384F8413AEFE7194BB3F862
:104A4000D230002B3FF41FAE032384F8413A1AE61C
:104A500094F8302094F831309A4204D0FCF7D6FD17
:104A6000C4F8445A22E6D4F8443AEB1AB3F57A7FF4
:104A7000BFF41CAE0C4B1B68ED1A952D7FF616AEDD
:104A80000A480521FCF706FABDE8F047FCF7BEBD71
:104A90005D32002060320020AC7B0020FC0400204E
:104AA000EC45002030040020FC450020BE0500201D
:104AB00010B5134CD4F8B00700B394F8681759B187
:104AC00094F8692709F07AFFB4F86C3783421ABF6B
:104AD000A4F86C0701210021B4F86E2762B141F2FD
:104AE00088339342B8BF13469A4205D0A4F86E3774
:104AF000BDE810403BF0A0BE0029F9D110BD00BFB9
:104B00008071002010B401440446002014F8013BD9
:104B100008225840430010F0800F08BF400083F087
:104B2000070314BFD8B2C0B2013AF3D18C42EDD121
:104B30005DF8044B704700BF30B54FF4806085B01E
:104B40002BF07AFC40B3154C90F9040094F8483AE5
:104B5000134A002B18BF08234FF4E1310125CDE99A
:104B60000153009100234FF480612BF0C6FCFF231A
:104B7000E066003818BF012084F8E83484F8F8347F
:104B800084F8083584F8183584F8283584F83835E1
:104B900084F8483584F8583505B030BD8071002060
:104BA00075110108374B1B6813F000635CD02DE9C9
:104BB000F04F354B1F78B84251D3FF2856D1334BB5
:104BC00093F8DC30002B47D0DFF8D4A00022CAF8DD
:104BD0004C2ACAF8502ACAF8542AAAF8582A002F90
:104BE0004CD00AF59D6310461446114615461646EC
:104BF00003EB071BB946B3F802C09F8993F8008006
:104C000093F901E061443A444645D3E901C738BF0E
:104C1000464610337545B8BF75469B4509B212B27A
:104C200064443844E7D191FBF9F192FBF9F28AF838
:104C30004C6A8AF84D5ACAF8504ACAF8540A144BBA
:104C4000AAF84E1A1B781149AAF8582A092B4FF0D6
:104C5000000281F8DC200CD00E48BDE8F08F0E4A2F
:104C600002EB0010BDE8F08F184670470020BDE849
:104C7000F08F0A4B9AF84C2ADA80EDE73A4639462B
:104C8000DDE700BF44440020700A0010300400201B
:104C90005D320020CC7B002068760020603200204E
:104CA000807100200268F8B53A4E3B4CB6F95C3A88
:104CB000511C01607E2111700168054603EBC3039E
:104CC00084FB0302481CDC17002328600B70FF20C4
:104CD000C4EB6204FFF766FF2034304BA4B2002817
:104CE0004DD01B78B0F90C102BBB2D4BA1F57A726F
:104CF0009A4246D82B48B0FBF1F189B228463AF0E7
:104D0000B7FF96F8F337B6F8541783B196F80C3816
:104D1000B1FBF3F128463AF0ABFF214628463AF0C2
:104D2000A7FF28460821F8F731FC0120F8BD2846E6
:104D30003AF09EFFF1E71C4B1F78002FD5D01B489F
:104D4000002300EB830201339289BB421144F8DB5C
:104D5000174B9FED186A9B7E07EE103A07EE901AEC
:104D6000B8EEC77AF8EE676AC6EE077A67EEA67AFB
:104D7000FCEEE77A17EE901AB1FBF7F1B5E71B7876
:104D800013B94EF69C21B9E7074B1F78002FF8D0D6
:104D90000146D4E7807100206766666660090010EE
:104DA0001783930300879303700A00102C0C0010E4
:104DB000002B0020000048432DE9F04FAE4C89B095
:104DC00094F85E9A054631F0B1FDD4F8603AD4F813
:104DD000F468074623F40013F007C4F8603A48D596
:104DE00000201DF055FA002840D0D4F8682A002A87
:104DF0003CD0910104D5B2F1007F18BF02F17E4290
:104E0000D4F86C1A9FED9D7A7B1A07EE903AF8EE73
:104E1000677AF4EEC77AF1EE10FA05DCD4F8700A7E
:104E200001238340134212D111B91923C4F8703AF7
:104E3000D4F8703AC4F86C7A012001331A2B28BFD9
:104E4000002300FA03F11142F7D0C4F8703AD4F805
:104E5000702A8B4B8B49686803EB82035A6C43F0D2
:104E600083FC02236B7309B0BDE8F08F0023C4F804
:104E70006C3AD4F8743A7BB394F87237DB072BD4CE
:104E8000D4F8783A9FED807A686803F5921303F5B9
:104E90007863DB1B07EE903AF8EE677A67EE877A65
:104EA000FDEEE77AB8EEE77A17EE903AF1EE0C7A7B
:104EB000B4EEE77AF1EE10FA05DB744943F054FCE6
:104EC00001236B73CFE70A21B3FBF1F201FB12332D
:104ED0006F4943F049FCF3E7B7050FD594F87737EE
:104EE00063B16C49686843F03FFC03236B73D4F8EB
:104EF000603A43F40013C4F8603AB4E7B00609D549
:104F000094F87C3A33B16449686843F02DFC01237E
:104F10006B73A8E7710536D594F87D3A012B32D131
:104F2000D4F86C3568689A0729D5B4F98E3AB4F983
:104F30003E28D21A6FF463739A421BDB40F28D3322
:104F40009A421ADC0A2392FBF3F2544943F00CFC18
:104F500020F0ACF9524B1B6893F865300A3B23EA0A
:104F6000E3739842ACDBD4F8603A43F40013C4F81E
:104F7000603AA5E76FF05902E7E75A22E5E74949A9
:104F800043F0F2FBE4E7B30412D511F08FFD94F87F
:104F9000EC3883420CD94449686843F0E5FB0223AE
:104FA0006B73D4F8603A43F40013C4F8603A5AE7DC
:104FB000370408D53D4BB4F94029B3F9E4309A429F
:104FC00001DD3B49E8E7700407D511F057FDB4F85F
:104FD0003E39834201D93749DEE7310704D5B9F1BB
:104FE000020F01D134497DE732050FD594F87237AD
:104FF000DB070BD51DF0EAF840B194F8E437DF0782
:1050000004D594F8C93A0BB92C49C5E7F00414D576
:1050100094F87237D90710D51DF0D8F868B194F814
:10502000E437DA0709D4D4F8CC3AA3F53713A3F55B
:10503000D863002B01DA2249AEE7B4F83A385B06B0
:1050400001D52049A8E7370640D5B4F95C0A94F8A1
:10505000063998423ADB07F013FB94F8ED286E68A6
:105060001949002A0CBF0D220E2203460092304639
:105070007A2243F079FB92E7807100200024F44803
:10508000E81D060862E40608ACC527374FA20608EB
:105090005AA2060867A2060871A206087CA20608A2
:1050A0008C45002086A206088DA206083004002048
:1050B00058A8060896A20608A3A20608ADA20608EC
:1050C000B8A20608C3A20608CCA206085F4B1B685C
:1050D00018016BD5710669D55D4903910E7804AA54
:1050E000C6F1090676080023934620219E421CD172
:1050F0000BEB060057494CF0BEF94FF000080336A1
:10510000C246039B1B78534501D90B2E11D908AB1E
:105110001E44002306F8103CB8F1000F46D04E495B
:1051200068685A4643F020FB39E702F8011B013357
:10513000DCE75FFA8AF73846FFF734FD94F872C768
:1051400031371CF00102FFB22ED0B4F902E9BEF1F2
:10515000FF3F29D08189642311FB03F13F4B9B7EE4
:105160005B0891FBF3F39E45B4BF3B46522394F991
:10517000001911F1800F04D090F901E08E45A8BF0D
:1051800054233AB1B4F904194A1C03D04068884248
:10519000A8BF4323BB420BF8063018BF08F1010833
:1051A0000AF1010A0136ACE73B46E0E7D4F8F438EF
:1051B0005A0704D5B9F1010F01D12949ECE6DF0501
:1051C0000DD594F87227D60709D5264A92F82520DE
:1051D000012A04D1244A12780AB92449DCE6D8030A
:1051E0000CD594F87227D10708D5B4F8E8282AB16D
:1051F000D4F864178A4201DC1D49CDE69A0718D518
:1052000094F8722794F85E1A02F003020A4310D150
:10521000B4F83218B4F8542794F80C08B2FBF0F242
:10522000914206D91349686843F09EFA01236B73D3
:1052300019E6DB067FF517AE94F8F43A002B3FF43D
:1052400012AE0D49686843F08FFA39E644440020F5
:10525000700A0010C3A5060862E40608002B0020AF
:10526000DBA206085C410020780A0010E7A20608CD
:10527000F3A20608FCA2060808A306082DE9F843D5
:105280004A4C427894F8F53A02F00F05C3B9EDB9EB
:105290002B46002184F8F81AEB1AD9B20E290BD844
:1052A000234493F8F41739B102F0F002802A4AD06F
:1052B000902A5FD0A02A0DD000273846BDE8F88399
:1052C0000021AB4284F8F81AF6D8E5E784F8F55ADD
:1052D0002B46DEE7412966D081F08003042B62D99A
:1052E0000846FBF75FFF031D0246DBB2304884F837
:1052F000F83A65F05F0584F8F95AFCF77DFB94F8FD
:10530000F87A002FD8D0BE1E16F0FF0024D1FF255A
:10531000A946022756B1DFF89C80464418F8011BC5
:10532000D4F81C0B32F0D6F84645F7D1D4F81C0B54
:10533000494632F0CFF8D4F81C0B294632F0CAF8AF
:105340003846BDE8F88365F07F050427022684F817
:10535000F95A84F8F87A3046164A4FF6FF7110442D
:1053600012F8015B491B904289B2F9D15FFA81F9C9
:105370000D0ACFE7412914D081F08003042B10D906
:105380000846FBF70FFF65F06F050627042684F833
:10539000FB0A84F8F95A84F8FA1A84F8F87A304645
:1053A000DAE70420EFE7082304229FE7807100205A
:1053B0007A7C0020787C00202DE9F047C31DDFF8BF
:1053C000348182B003F4FC7300AFD8F88465ADEB90
:1053D000030DC7F800D03268D8F87C3568449A428B
:1053E0000C4698F8203B78606D4658D0591C0DF15A
:1053F000010203F00F0388F8201B8DF800303A609B
:10540000A0EB0209D6E900125FFA89F9521A09F1F4
:1054100007035FFA82FA03F4FC73CA45ADEB030D90
:1054200055D2524668464BF0A1FF3368534433606F
:105430005246694638463AF0F9FBD8F88425D8F840
:105440007C353068117A7060C21A4A40D2B2834209
:10545000336088F8212B09D00133336013F8011C25
:10546000984282EA0102F7D188F8212B3B68591C47
:1054700039601A70D7E90032D21A012A08DD0021FA
:105480005A1C3A601970D7E90032D21A012AF7DCA7
:105490002846A04700200837BD46BDE8F087B6F98A
:1054A0000C20591C03F00F0343F01003002A2A4676
:1054B000B8BF43F0200302F8023B88F8201B691CA8
:1054C0003960D6E900135B1A3A606B7098E74A4678
:1054D00068464BF04BFF33684B4433604A4669469D
:1054E00038463AF0A3FB2846A04701200837BD46BE
:1054F000BDE8F087807100202DE9F04F7C4C83B02F
:10550000D4F88455D5E900535B1B002B00AF8346CC
:105510000D4616462ADD002384F8223BFBF7B8FE31
:1055200000200BEB05030BF1010AC4F87435C4F835
:1055300070A59BF80050D4F880856909012940F0D6
:105540009F8005F00F0915F0100514D150B194F8A3
:10555000242B013202F00F024A4500F09A8084F8B1
:10556000225B28460C37BD46BDE8F08F94F8220B2D
:105570000028D6D1D2E70BF10203C4F870350BF145
:1055800003029BF80130D4F87805C4F870259BF825
:105590000250C8F80000C218C8F804206B404FF051
:1055A000000C84F8233BD4F870A5D4F8743584F843
:1055B000221BA8F80850A8F80CC0A3EB0A03DDB220
:1055C000121AEB1D5FFA82FB03F4FC73AB45ADEBE3
:1055D000030D6BD25A46514668464BF0C7FE0AEBA4
:1055E0000B035A4640466946C4F870353AF01EFB34
:1055F000D4F87835D8F8000094F8232B8342C8E912
:1056000000300AD00133C8F8003013F8011C98426A
:1056100082EA0102F6D184F8232BD4F870351B7886
:10562000934239D1B8F90830FA2B54D0D8F8002079
:10563000D4F87835D4F88015D4F82C07C8E90032AE
:10564000D4F88425D4F87C355360002515819581E4
:105650003B1D84F8225B7D602BF038FB01303FD08E
:105660007B680BB100209847D4F88435D4F87C25AA
:10567000196801200C37C3E90021BD46BDE8F08F51
:1056800000210846FBF7E8FD01200C37BD46BDE8C8
:10569000F08FD8E9000290E700230120B8F9081044
:1056A00084F8223BFBF7D8FD01205BE72A465146F0
:1056B00068464BF05BFE0AEB050340462A46694606
:1056C000C4F870353AF0B2FA00200C3784F8249B05
:1056D000BD46BDE8F08F002EA8D005233370A5E7A6
:1056E000D4F8842513680221581C10601970B7E79C
:1056F000807100200B4B93F82A2812B1B3F80428CC
:105700004AB9B3F94038084AD81782FB0323C0EBE3
:10571000A30000B27047D3F8640790FBF2F000B228
:10572000704700BF8071002067666666F8B5184C48
:10573000C6B205463146D4F8280B31F0CBFE94F8BA
:105740002C1BD4F8280BC5F307274E40394684F8A4
:105750002C6B31F0BFFE94F82C1BD4F8280BC5F34A
:1057600007464F40314684F82C7B31F0B3FE94F865
:105770002C1BD4F8280B2D0E4E40294684F82C6B98
:1057800031F0A8FE94F82C1B4D4084F82C5BF8BD3A
:105790008071002070B50C4DC6B231460446D5F874
:1057A000280B31F097FE95F82C1BD5F8280B240A0E
:1057B0004E40214685F82C6B31F08CFE95F82C1B61
:1057C0004C4085F82C4B70BD8071002038B50B4CD7
:1057D000002305462421D4F8280B84F82C3B31F013
:1057E00079FED4F8280B542131F074FED4F8280B3C
:1057F0002946BDE8384031F06DBE00BF8071002001
:105800002DE9F047DFF858A32DED028B9AF82D4BC8
:1058100082B00F461646002C00F0E781013C8AF862
:105820002D4BDFF840839FEDC88ADFF83C933B782F
:10583000002B00F090809AF82D4B002C40F08B80CC
:1058400036B131F073F83368C01A002880F2DD8376
:105850009AF82E1B002940F07C839AF82F5B062DC6
:1058600040F28481B94B93F8A10193F8A0218242C0
:1058700000F0AB81D3F89C219AF8301B32F810402D
:105880000C440135013003F5CE73A4B2EDB2C0B2C1
:10589000B4F5C06F8AF82F5B587100F07E817CD818
:1058A000B4F5806F00F0298224D8B4F5067F4FD874
:1058B000B4F5007F54D3A4F50073182B48D8DFE863
:1058C00013F0E701DE01DE01DE01DE01DE01DE01B3
:1058D000DE01DE0147004700470047004700470060
:1058E0004700C601AB01AB01AB01AB01AB01AB01A2
:1058F000AB01AB01B4F5846F00F0E68140F2E280C9
:10590000B4F5A06F00F064826FF4A06C04EB0C039C
:10591000072B1DD8601EC0B2FFF744F9C0B1B0F923
:105920000C308B4AADF80140917EDAF8302703EB5A
:10593000830303EB830349089B0093FBF1F31021DE
:10594000CDF803308DF800106846904700233B7077
:10595000002E7FF46CAF02B0BDEC028BBDE8F08787
:10596000B4F5807F00F0FD81B4F5887FF0D1BAF9FD
:105970004238CDF80330012210238DF800308DF825
:1059800001308DF80220DAF8303768460024984755
:105990003C70002E7FF44BAFDDE7B4F5046F00F0F0
:1059A000A68265D8B4F5006F00F084821AD9B4F5E8
:1059B000026F00F0F181B4F5036FC9D19AF8E437B2
:1059C0009D07C5D5634BDAF83027D9894FF4F363C7
:1059D00003FB01F3A8FB03135B091020CDF8033090
:1059E00030218FE2B4F5E26F00F03782B4F5E46F56
:1059F0001FD1594B93ED170AD3ED017A20EE270AF8
:105A0000002420EE080A49F0ADF9102320228DF879
:105A100000300723CDF803008DF802308DF8012007
:105A2000DAF83037684698473C70002E7FF4FFAEB6
:105A300091E7B4F5E06F8BD1474B93ED150AD3EDA9
:105A4000017A20EE270A002420EE080A49F08AF99C
:105A500010220723CDF803008DF802308DF80020C6
:105A6000DAF830378DF80140684698473C70DCE73B
:105A700040F678339C4248D8B4F5376F00F2E281A3
:105A8000B4F5116F00F08081B4F5376F7FF460AF2B
:105A9000FF20FFF787F800283FF45AAF90F9013054
:105AA000CDF80330102170220B238DF802308DF8D1
:105AB0000010DAF830378DF8012068460024984746
:105AC0003C7066E740F201439C4200F02A82B4F544
:105AD000826F7FF43DAFDAF86C35980600F14882AA
:105AE0001E4B1B681B0640F19682002410230422E3
:105AF0008DF800308DF801308DF803408DF80440AA
:105B00008DF805408DF80640BBE145F230239C42FC
:105B100000F0848145F240239C427FF419AFBAF92A
:105B20003C38CDF803301021402252238DF802304A
:105B30008DF80010DAF830378DF80120684600241F
:105B400098473C7025E700BF0000C84230040020A1
:105B5000002B002010450020C80B001044440020FA
:105B6000807100201F85EB51C5B3A2910135CA4B4E
:105B7000EDB293F8A92193F8A811914220D0501CBE
:105B8000C0B25200D3F8A411C44B8C5A8AF82F5BD0
:105B9000B4F5C06F58717FF482AEDAF86437CDF88F
:105BA00003301022002406238DF802308DF80020E7
:105BB000DAF830378DF80140684698473C7034E792
:105BC000002283F8A9210120DCE7B5489AF8302BA0
:105BD000007883F8A1110132D2B2013082428AF8F2
:105BE000302B00F0B2810125C3E700283FF419AE45
:105BF0000378303B012B3FF614AE01300AF62D320C
:105C00000621FFF779FC9AF82D3B8AF82E0B002B22
:105C10003FF407AE3C7004E6A4F11100C0B2FEF7F9
:105C2000C1FF00283FF494AEB0F90230CDF8033044
:105C300010238DF80030ADF80140DAF830376846AF
:105C4000984700233B70002E7FF4F1AD83E69AF86D
:105C5000F327BAF85437002A40F0D18110220221EC
:105C6000CDF803308DF80020DAF830378DF80120B8
:105C70008DF802106846002498473C7089E6601E43
:105C8000C0B2FEF78FFF00283FF462AE4368CDE755
:105C9000DAF85C378349DAF8302781FB0301DB1738
:105CA000C3EBA10300241021CDF8033002238DF8AB
:105CB00000108DF801408DF80230684690473C7026
:105CC000002E7FF4B4AD46E69AF8E4379A077FF5E4
:105CD0003FAEBAF8E637CDF8033010212022042376
:105CE0008DF802308DF80010DAF830378DF8012089
:105CF0006846002498473C704BE69AF8383B0133DD
:105D0000DAB2042A00F0708142F210738AF8382B5C
:105D100003FB02F3DAF8682A002A00F02781023335
:105D20009AF87227D507BAF83A2848BF0433D4073F
:105D300048BF0A33900748BF1433D10548BF283302
:105D4000550748BF6433540648BF03F57A631021F2
:105D500000240422CDF803308DF800108DF80140A6
:105D60008FE0DAF8343BCDF8033010220024012311
:105D70008DF802308DF80020DAF830378DF80140C8
:105D8000684698473C7050E69AF80C38002B40F073
:105D900031811022092163E79AF8E4379B077FF5E8
:105DA000D7AD414ADAF830379268CDF80320102297
:105DB00020218DF8002008228DF801108DF8022096
:105DC0006846002498473C70002E7FF430ADC2E551
:105DD000FF20FEF7E7FE00283FF4BAADB0F90C3023
:105DE0003249DAF83027897E03EB830303EB830320
:105DF0001020490800249B0093FBF1F305218DF846
:105E00000000CDF803308DF801408DF8021068468F
:105E100090473C70002E7FF40AAD9CE5BAF93E38FD
:105E2000CDF803301021302252238DF802308DF846
:105E30000010DAF830378DF80120684600249847C2
:105E40003C70A6E5A4F17100C0B2FEF7ABFE0028DD
:105E50003FF47EAD90F90130E8E6154B93ED160A5C
:105E6000D3ED017A20EE270A002420EE080A48F03C
:105E700079FF1023CDF8030007228DF800308DF84C
:105E80000130DAF830378DF80220684698473C70C8
:105E9000002E7FF4CCAC5EE530040020D405002059
:105EA000700A00106766666610450020002B00200F
:105EB000C80B00109AF8E4379C077FF549ADC1077D
:105EC000814B40F1B5805A6882EAE273A3EBE2733A
:105ED00003EB5303A8FB0313DB08002AACBF43F01A
:105EE000004343F0404310210024082232E7BAF96E
:105EF0004038DAF8302703EB83035B001020CDF83D
:105F00000330402108238DF800008DF801108DF832
:105F100002306846002490473C70002E7FF487AC26
:105F200019E5BAF95C3ACDF80330102101220423B7
:105F30008DF802308DF80010DAF830378DF8012036
:105F40006846002498473C7023E58AF8301B0125F9
:105F50000FE65E490620FFF72FFA00238AF82E0B82
:105F60003B7002B0BDEC028BBDE8F0870133D7E691
:105F7000554A9AF8E417538A643BC3EB4370C3EB6A
:105F8000C00389FB03401844DB17C3EB202309330C
:105F9000092BA8BF092323EAE37303EB830311F062
:105FA000020F03EB830314BF4FF47A7000209B00B1
:105FB000C90748BF00F5FA60117DDAF830279BB2B7
:105FC00003440B44042010218DF80200CDF8033067
:105FD0008DF800108DF801106846002490473C7041
:105FE000002E7FF424ACB6E401238AF8383B42F259
:105FF00010738FE6BAF85427B2FBF3F3C9E69AF8A8
:106000000C28002A57D1134628E63C7002B0BDEC9C
:10601000028BBDE8F0879AF8F237002B3FF498AC7A
:106020009AF8393B032B49D8DFE803F03B312211C2
:106030001A6882EAE273A3EBE27303EB5303A8FB53
:106040000313DB08002AB8BF43F080434BE7DAF8BC
:106050003C2B537A907AD17A03F1407303EB0023FF
:10606000002203EB01438AF8392B10220421F7E5C3
:10607000174A11688A7D087C897A120402EB002293
:106080000A44591C8AF8391B02EB0363EDE7104AF6
:1060900011684A7DC87B497A120402EB00220A4447
:1060A000EFE70B4A11680A7D887B097A120402EB3C
:1060B00000220A44E5E7B3FBF2F3CFE55A1C8AF865
:1060C000392B1B06D1E700BF10450020DD12010867
:1060D0008C45002030B5A0F17D03012B044683B030
:1060E0000D46104608D9214631F0F4F915B128883B
:1060F00004442C8003B030BD7D21019231F0EAF9D7
:10610000019884F0200131F0E5F9EFE730B50F4B4D
:1061100085B0D3F8402B00230446C51DADF80E30E2
:1061200014F8010B01920DF10E01FFF7D3FFA54208
:10613000019AF5D10DF10E0011F02AFE019A9DF899
:106140000E000021FFF7C6FF05B030BD80710020B2
:10615000044AD2F8443B43F4DF2343F48063C2F89B
:10616000443B704780710020013070B5094EC4B2C5
:1061700003E042F02FFB013448B9E5B2152D21466A
:106180003046F6D9162D04BF034B93F8485B2846DA
:1061900070BD00BFC47C00208071002000B1D7E733
:1061A000044AD2F8443B23F4DF2323F48063C2F88B
:1061B000443B70478071002070B5114C84B0054697
:1061C000D4F84C0B0E462AF0CDF894F8EC2794F84E
:1061D000ED37003A18BF01220BB142F00802CDE9B9
:1061E000016200234FF4964195F9000000911A4690
:1061F00008212AF082F9C4F84C0B04B070BD00BF2E
:106200008071002010B5064C03E0D4F84C0B31F03F
:1062100055F9D4F84C0B31F059F90028F5D110BDDF
:106220008071002010B50D4CD4F8503B1B791E3BFB
:10623000012B0DD9D4F84C0B01213830FFF7BCFFEE
:106240000023C4F8543B84F8583BBDE81040D9E71C
:10625000D4F84C0B012131F029F9F1E780710020CD
:1062600070B50A4E0546D6F834375E200C4698477E
:10627000D6F8343728469847E0B2FBF745F8C4F320
:106280000720BDE87040FBF73FB800BF80710020D9
:1062900003682DE9F041002B3D4D3E4F3E4EB8BF07
:1062A0005B42A5FB0321890D07FB0137C7EB0717ED
:1062B000BF0096F8EE3785FB0725FA170446C2EBB8
:1062C000A555002B57D101EB810101EB810105EBB5
:1062D000810109B2DFF8BC801320FFF7C1FF2F490D
:1062E00008FB057581FB0531ED17C5EBA11109B25E
:1062F0001B20FFF7B5FF2368254D002BB4BF5321AA
:106300004E212320FFF7ACFF636896F8EE2783EA5F
:10631000E376A6EBE376A5FB0631890D08FB016861
:10632000C8EB08184FEA880885FB08354FEAE87380
:10633000C3EBA5552ABB01EB810101EB810105EB04
:10634000810109B21220FFF78BFF124B134903FBA7
:10635000058581FB0531ED17C5EBA11109B21A20A6
:10636000FFF77EFF6368002BBDE8F041B4BF572103
:106370004521222074E7C1EB011105EB810109B22F
:10638000A8E7C1EB011105EB810109B2DAE700BF13
:106390006BCA5F6B806967FF80710020D34D62100C
:1063A0000B2814D810B401EB4103094C01EB830313
:1063B0002344184490F85438934205D021440023D4
:1063C00080F8542881F848385DF8044B70477047CE
:1063D00080710020F0B5464C94F8593B012B83B0F6
:1063E000054650D994F85A0B4249434E94F85B7BCA
:1063F000421CA1FB02C1184406EB800001F4FE76AA
:1064000006EB9101521AD0F8AC6084F85A2B2FB1E8
:10641000D4F85C1B04F5366291420DD06EB9374A50
:106420000133A2FB031222F0010101EB52029B1A7D
:1064300084F8593B03B0F0BD314E94F8743B93B9E6
:10644000304B019348F2A501123B15226F46A4F888
:10645000781B009384F87A2B29463846B04758B900
:1064600094F8593BDBE76F46384610F0E5FA2946C9
:106470003846B0470028F3D094F8741B59B1384619
:1064800010F054FAECE71C4A02EB8302D2F8AC603D
:10649000002EC4D0D1E7009E1B4A964214D9013A7F
:1064A000013E41F2210512F8013F81EA0321082350
:1064B00011F4004F85EA41000ABF490081B289B258
:1064C000013BF5D19642EED1384639F0F7FB0F4942
:1064D000009D6D1A152DA8BF15252A4601F118003B
:1064E0004AF044FF94F8593B84F8A55B97E700BF56
:1064F00080710020CDCCCCCCE81D0608ABAAAAAA9E
:10650000911E01080D7D0020FB7C0020F87C0020FE
:1065100070B50B4E054606F6AA313EF0A7FD2C6875
:106520006C6006F6A831641A402CA8BF402429608C
:10653000224606F6E8304AF019FF86F8284C70BD6E
:1065400080710020F0B5C34C94F8303C234483B0F4
:1065500093F82C5CEB0714D4AF077AD46E0700F1E4
:10656000BC802B0700F1E58094F8303C94F8321C95
:106570000133B3FBF1F201FB123384F8303C03B07A
:10658000F0BDB4F93E3804F6E83204F6AB3040F61C
:10659000C8010192B3F5E16F4FF01E020090A4F81C
:1065A000A81B84F8AA2B40F30A81A3F561631BB2F0
:1065B000B3F5E16FF9DC07EE903A9FEDA77AF8EEBC
:1065C000E77A6E4667EE877A3046FDEEE77A17EE99
:1065D000903A99B239F04CFBB4F93C38B3F5E16F1D
:1065E00040F3F480A3F561631BB2B3F5E16FF9DC0E
:1065F00007EE903A9FED987AF8EEE77A304667EE2C
:10660000877AFDEEE77A17EE903A99B239F030FBCF
:10661000B4F94038B3F5E16F40F3DF80A3F561636F
:106620001BB2B3F5E16FF9DC07EE903A9FED8A7A81
:10663000F8EEE77A304667EE877AFDEEE77A17EEF6
:10664000903A99B239F014FB3046FFF761FFAF077B
:1066500084D5824B94F8F327019340F6C8203D3B44
:1066600008210093A4F8A80B84F8AA1B002A40F084
:10667000B880B4F854177A4B05316E46A3FB01314C
:106680003046C90839F0F4FA764AD4F85C37D9179D
:1066900082FB0323C1EBA30189B2304639F0E8FA4B
:1066A00027F01AFD009AD4F864370146571C180CDD
:1066B00000971070009A180A571C00971070009AE3
:1066C000501C00901370009B5A1C304600921970A9
:1066D000FFF71EFF6E077FF544AF604B94F87227FB
:1066E0000193C8203D3B2121A4F8A80BD0070093BB
:1066F00084F8AA1B40F18780B4F83A385A0578D557
:1067000059496E46304639F07FFA94F87237DA0705
:106710007ED5009A5549531C009300231370009BAB
:1067200030465B1A84F8A93BFFF7F2FE2B077FF592
:106730001BAF4A4B4E4D01933D3B41F2C8122968B5
:10674000009368460223A4F8A82B84F8AA3B39F0EA
:1067500077FA6968474E684639F072FAEB8903EBBD
:10676000C30189003231A6FB01316846C1F34F11E4
:1067700039F07EFA298A01EB81014900684689B225
:1067800039F076FAD4F8341B3B4B9942A8BF19462E
:1067900021EAE171A6FB0131490901F57A716846E8
:1067A00089B239F065FA009B2A7D591C0091684630
:1067B0001A70FFF7ADFED7E603F561631BB213F560
:1067C000E16FF9DBF7E603F561631BB213F5E16FE7
:1067D000F9DB0DE703F561631BB213F5E16FF9DB3C
:1067E00022E7B4F8541794F80C281D4BB1FBF2F1D2
:1067F00042E71F0520D4DE0520D4D80720D499070E
:1068000020D51E497DE7D4F8683A3BB11C4978E7AA
:10681000009B2A22591C00911A707AE7194B1B68B9
:1068200019067FF569AF94F8E43703F00303032BEF
:106830003FF462AF144964E7144962E7144960E722
:1068400014495EE794F8312C1349144B002A18BF01
:10685000194656E78071002058A08B41687D0020C2
:10686000CDCCCCCC6766666630A30608297D0020B7
:10687000104500201F85EB5120A1070014A3060836
:1068800020A306084444002028A3060838A30608CD
:106890003CA3060844A3060818A306084CA3060850
:1068A00030B50C4B0C4AC3F8A82B83B0C822014664
:1068B00003F6E83503F6AD3483F8AC2B68463A228C
:1068C000CDE9004539F0B2F96846FFF721FE03B083
:1068D00030BD00BF80710020C83E7BEA044BD3F876
:1068E000083830EA030314BF01200020704700BFBE
:1068F00080710020CD4A38B50820002382F8A931E4
:10690000FFF7ECFF50B1D2F8A4314FF480640220BD
:106910004FF482611C8082F8A90159804FF4002055
:10692000FFF7DCFF50B192F8A931D2F8A4115C1C3A
:1069300040F2014082F8A94121F81300BC4991F8C6
:106940002938002B6ED191F82A38002B40F0458170
:106950004FF40070FFF7C2FF50B192F8A931D2F89E
:10696000A4015D1C4FF4046482F8A95120F813407F
:10697000D1F86C15880700F1E180490700F1BB8070
:10698000AC4B1B681B066ED492F8A93182F8A83173
:106990004FF48030002382F8A93182F8A131FFF74B
:1069A0009DFF38B1D2F89C3101204FF4047182F878
:1069B000A10119804FF40040FFF790FF50B192F809
:1069C000A131D2F89C115C1C4FF4007082F8A141F7
:1069D00021F813004FF40030FFF780FF50B192F818
:1069E000A131D2F89C115C1C4FF4A06082F8A14147
:1069F00021F813004FF48020FFF770FF50B192F898
:106A0000A131D2F89C115C1C4FF4376082F8A1418F
:106A100021F8130092F8A13182F8A031002382F806
:106A2000A13138BD0120FFF759FF00288BD04FF46A
:106A30008030FFF753FF50B992F8A931D2F8A40182
:106A40005D1C4FF4047482F8A95120F8134092F8A9
:106A5000A931D2F8A4015D1C4FF4116482F8A95148
:106A600020F813406FE74FF40050FFF737FF50B1A5
:106A700092F8A931D2F8A4115C1C4FF4036082F89B
:106A8000A94121F813004FF48050FFF727FF78B198
:106A900092F8A931D2F8A401591C1D46C9B24FF48D
:106AA0000064023320F8154082F8A93120F8114023
:106AB0004FF48040FFF712FF50B192F8A931D2F89D
:106AC000A4115C1C4FF4846082F8A94121F81300E2
:106AD0004FF48060FFF702FF00283FF455AF92F8B3
:106AE000A931D2F8A4115C1C4FF4026082F8A941CC
:106AF00021F8130048E74FF48060FFF7EFFE50B134
:106B000092F8A931D2F8A4115C1C4FF4807082F87D
:106B1000A94121F813004FF40060FFF7DFFE0028C1
:106B20003FF42EAF92F8A931D2F8A4115C1C4FF4B7
:106B3000887082F8A94121F8130021E78020FFF72F
:106B4000CDFE50B192F8A931D2F8A4015D1C45F2F6
:106B5000302482F8A95120F813404FF48070FFF7D9
:106B6000BDFE50B192F8A931D2F8A4015D1C45F2E6
:106B7000402482F8A95120F813401020FFF7AEFE00
:106B800050B192F8A931D2F8A4015D1C4FF4E06431
:106B900082F8A95120F813402020FFF79FFE50B142
:106BA00092F8A931D2F8A4015D1C4FF4E26482F896
:106BB000A95120F813404020FFF790FE00283FF431
:106BC000DCAE92F8A931D2F8A4015D1C4FF4E46464
:106BD00082F8A95120F81340CFE60220FFF77EFE8D
:106BE00000283FF4B5AE4FF40040FFF777FE50B9F0
:106BF00092F8A931D2F8A4015D1C4FF4007482F818
:106C0000A95120F813400420FFF768FE00283FF444
:106C10009FAE92F8A931D2F8A4015D1C4FF4C06474
:106C200082F8A95120F8134092E600BF30040020FA
:106C3000807100204444002003685A0607D513F4ED
:106C4000057F04D007298CBF00200120704703F482
:106C50008253B3F5825F03BFC81FB0FA80F04009CA
:106C60000020704770B5BD4C94F8333C012B84B0C4
:106C700000F04E8194F83D0CFBF7A6FD94F83E3CE5
:106C8000834205461FD0002800F0D780D4F8503B3F
:106C9000CBB194F8ED2793F90400002A18BF08221D
:106CA0004FF4964100230325CDE9015200911A4685
:106CB000082129F022FCC4F84C0B20B1FFF7B2FAEE
:106CC000012384F83E3C94F83F3C012B00F0C28045
:106CD000D4F8486C3EB1A24B30465978FFF7ACFF70
:106CE000002840F0F38094F84D0CFBF76DFD94F80C
:106CF0004C3C8342054622D0002800F0F780F6B1D4
:106D0000337A002B00F01981964A02EB8303D3F803
:106D1000C83094F8EC2796F904000093003A18BFA5
:106D2000012202210023CDE901121A46102129F087
:106D3000E4FBC4F8280B10B1012384F84C3CD4F8D0
:106D4000506C3EB1864B30465978FFF775FF0028EE
:106D500040F0AC8094F85C0CFBF736FD94F8543CA2
:106D60008342054623D0002800F0C980FEB1337A63
:106D7000002B00F0E5807B4A02EB8303D3F8C83098
:106D800094F8EC2796F904000093003A18BF01220A
:106D900002210023CDE901121A464FF4007129F0B7
:106DA000ACFBC4F8580C10B1012384F8543C94F89F
:106DB0005D0CFBF709FD94F85E3C8342054630D03C
:106DC00088B3694BD4F8606C4FF47A72C3F87C26B0
:106DD0003EB34FF480524021304629F019FB05465E
:106DE000F8B994F8EC3796F90400002B14BF092188
:106DF000082103224FF4E133CDE9012100932A4613
:106E00002B464FF4805129F078FBC4F8640C40B154
:106E10000123C4F81C0B84F8F55A84F8685C84F8E4
:106E20005E3C04B070BDD4F8640C29F09BFAC4F841
:106E3000645C84F85E5C04B070BDD4F84C0B29F03F
:106E400091FA94F83F3CC4F84C5B012B84F83E5C0B
:106E50007FF43EAF94F8400CFBF7B6FC05460028E3
:106E600071D0D4F8403B002B7FF432AFD4F8442CDF
:106E7000002A3FF42DAF94F8ED5794F8EC1792F9EF
:106E80000400002D14BF08220022002908BF42F090
:106E9000010203254FF46141CDE9015200911A46E8
:106EA000202129F02AFBC4F8400B11E794F8543C48
:106EB000002B7FF47CAFD4F8383C002B3FF477AF45
:106EC0000122C4F8583C84F8542C70E794F84C3CE8
:106ED000002B7FF434AFD4F8383C002B3FF42FAFB5
:106EE0000122C4F8283B84F84C2C28E7D4F8280B5E
:106EF00029F038FAC4F8285B84F84C5C1FE7D4F812
:106F0000580C29F02FFAC4F8585C84F8545C4EE70A
:106F1000D4F8345C124B28465978FFF78DFE28B31D
:106F2000D4F8E037002B7FF4A5AED4F8383C002B22
:106F30003FF4A0AEC4F8E0379CE64FF49643E8E691
:106F40004FF461431CE7D4F8400B00283FF4C0AE77
:106F500029F008FAC4F8405BBAE600BF807100204F
:106F60003C410020E81D06083004002094F83C0C49
:106F7000FBF72AFC0646D8B1D4F8E037002B7FF4A3
:106F800079AE002D3FF476AE94F8EC2795F9040025
:106F9000B2FA82F252094FF416510225CDE901529C
:106FA00000911A46042129F0A8FAC4F8E00761E626
:106FB000D4F8E00700283FF45DAE29F0D3F9C4F817
:106FC000E06757E670B5B14C94F8333C002B00F005
:106FD0002181082029F030FAC4F8500B00283BD05A
:106FE000082129F01FFA00260346A949A94884F878
:106FF0003D3CC4F8706C35F06FF841F20853012243
:10700000A448A4F8743C84F8782C0CF0E1FF3146D5
:107010002B22A1484AF00BFA48F67C607D25E0233C
:1070200031462B22A4F8800C9C4884F8833C84F8D9
:10703000AB5C4AF0FCF948F67C21A0224EF27B03BF
:1070400084F8D75C84F8DA6C84F8835DA4F8AC1C0F
:1070500084F8AF2CA4F8D83C94F83F3C002B00F007
:10706000C380102029F0E8F91021C4F8480C29F059
:10707000D9F98B4B84F84D0C3A2140F23B1094F82F
:10708000292818809F254AF21E40197100219D7100
:1070900098601973002A40F08E8094F82A38002BEB
:1070A00048D1D4F86C3558077ED4990773D41A07A1
:1070B0006AD47C4D2868C0F3C010FFF76FF8002039
:1070C000FFF752F803464FF4007084F8483B29F06C
:1070D000B3F94FF40071C4F8500C29F0A3F9D4F8B7
:1070E000843D84F85C0C002B14BF0123002384F83A
:1070F000883D26D1D4F8F02D0023C4F8EC3D002AB9
:1071000069D0012284F8743B84F8F42D4FF4805048
:1071100029F092F94FF48051C4F8600C29F082F9FB
:10712000002384F85D0C84F85E3CFAF7B1F8BDE802
:10713000704097E5D4F8443B43F00403C4F8443B63
:10714000AFE7D4F86C25002312F0020284F8893DE1
:1071500084F88A3D40F0828094F8293823B10120D8
:10716000FFF7BCFB002873D194F82A38002B6AD1B2
:10717000A3182868042183F82C1C030602F10101DE
:1071800075D484F8321CB5E7D4F8443B43F48073DB
:10719000C4F8443B8DE7D4F8442B42F4601242F02B
:1071A000C002C4F8442B82E7D4F8442B42F40272A4
:1071B000C4F8442B79E7D4F8443B94F82A2843F0E8
:1071C0000201C4F8441B002A3FF46BAF43F03603BE
:1071D000C4F8443B65E7D4F8F83D7BB3012384F859
:1071E000F43D84F8743B91E7202029F025F9C4F898
:1071F000440C00283FF435AF202129F013F92A4B25
:10720000C4F8303784F8400CFFF774FB012384F88E
:107210003F3C26E7042029F00FF9C4F8340C00287D
:107220003FF4D7AE042129F0FDF8204A84F83C0C45
:107230000123C4F8342784F8333CCAE684F8F43DCB
:1072400084F8743B62E70620FFF748FB00288FD0E4
:10725000A318022183F82C1C013289E74FF46070D7
:10726000FFF73CFB78B1012284F82C2C74E74FF433
:107270005850FFF733FB002883D063180820911C77
:1072800083F82C0C7DE7024666E700BF8071002082
:10729000F01E0608EC7D0020007E00202C7E0020E1
:1072A000E8440020444400200D610108E919010868
:1072B000094BB3F82228B3F82038801A9B1AC00073
:1072C00090FBF3F00628A8BF062020EAE070C0F18A
:1072D0009600C0B2704700BF8071002010B5094B06
:1072E0000022D3F8FC1D03F56063914201D1002018
:1072F00010BD13F8014B844201D00132F5E70120A3
:10730000F6E700BF807100201B4B2DE9F04103EB35
:1073100081038EB0D3F8587106460D4647B3174B1C
:1073200003EB41031C22B3F83C4E002319460DEB3E
:107330000200069304F01F084AF079F8C4F34414DD
:1073400001228DF8085006AD8DF81420CDE90356C2
:107350008DF809808DF80A4002A8B8479DF81420DE
:1073600000232AB100952246414602A805F0A6FC5A
:107370000EB0BDE8F08100BFE81D06088071002056
:107380000A4B03EB4002B2F83C1E094A92F8EC2883
:1073900002EAD122520707D0D3F8FC2D511CC3F8C2
:1073A000FC1D134483F8000E704700BF807100205D
:1073B0003004002010B5164B42681B7803F003031D
:1073C000032B21D1134B1B88DBB1134B1349B3F9AA
:1073D0000030B1F904100A2491FBF4F15B1A1B018F
:1073E00003F5B95314334FF4B471B3FBF1F3C3F1A4
:1073F000080303F00F0360331370436800225A70D0
:1074000010BD05231370F8E72D231370F5E700BFB7
:107410006479002066790020C4810020BC790020B6
:10742000436872221A70436873225A704368742248
:107430009A7043680022DA7070470F4B4268B3F9C4
:1074400004300A2193FBF1F31B0110B503F5B95386
:107450000A4C4FF4B4711433B3FBF1F303F00F0390
:10746000E118E35813604B6853600B7A137243685A
:1074700000225A7210BD00BFBC79002060200608AF
:10748000084B5B7933B942F210735843064B90FBBB
:10749000F3F07047242358434FF47A7390FBF3F0D2
:1074A000704700BF687A002040D20600831E00F1BA
:1074B0007402EA2123F8021F9342FBD143F64913D9
:1074C0004385CD2383804E23C380CE230381232392
:1074D000A0F87230704700BFF8B91D48438803F028
:1074E000010353BB30B40479ACB11A4A02F1F00580
:1074F00002E00133A3420ED052F8041B4904F8D530
:1075000090F8F01000EB8101D1F8881045F82310B5
:107510000133A342F0D130BC70470D484288032AA2
:107520004FEA52030AD90A68438002F5C332A032F7
:1075300003F001030A60002BD4D070470B6803F5F9
:10754000C333A03348F205020B604280704700BF8E
:10755000C4810020CC8100202DE9F041002839D1E0
:107560002C4A107980B32C4A2C4B92F800E092F907
:1075700001C092F90280CEF1FF07AEF17F06FFB2A3
:10758000F6B203EB800003F1F002002403E0834233
:1075900002F1040218D053F8041B8904F7D5E1B2B4
:1075A000A1EB0C0181EAE175A5EBE175012D0DDC84
:1075B00071B1414514BF394631468342D17004F15F
:1075C000010402F10402E6D1BDE8F0810821F4E7EC
:1075D0007146F2E7104B1A78F02A09D802F10F0031
:1075E0000C4A18700B6803F582431A330B60B8E736
:1075F000084A93F9014090797F2584421D7098785C
:1076000005DB4042C0B2987020445870EAE7002C75
:10761000FADAF6E7C4810020200D0020CC8100209A
:10762000F0B5354E78B196F87831002B45D0334A15
:10763000013BDBB286F878311378DC073FD4304B5E
:107640000A681A440A6034794CB32E4B2B4F03EB73
:10765000840403F1F001002503E09C4201F10401E0
:107660001DD053F8042BC2F303200628F5D1387837
:10767000C00715D596F8780196F807E000EB050CE1
:10768000BCFBFEF00EFB10C00128CCBF0020012087
:1076900058B99C4205F1010501F10401E1D1F0BDA9
:1076A000E84300F001000028F3D0C2F3834206EB68
:1076B0008202D2F888200A60EBE7F379B7E7124A32
:1076C000124BB2F906201248A2F57A74642202FB2A
:1076D00004F283FB0234D317C3EBA41303EB43037D
:1076E000C3EB031380FB0302DB17C3EB6213053309
:1076F000084A92FBF3F3A3E7C4810020F27800204C
:10770000400D0300CC810020A4450020D34D621021
:107710001F85EB5140420F00F0B4524C002867D156
:1077200094F87901002855D04F4BD3ED007AB3EE91
:10773000097AF4EEC77AF1EE10FA4DDCBBEE097A65
:10774000F4EEC77AF1EE10FA4CBF08270027D3ED0C
:10775000017AB3EE097AF4EEC77AF1EE10FA3DDD64
:1077600047F001072579ADB3404ADFF80CC102EBC1
:10777000850502F1F00014E094F97C61B142ACBFE0
:107780000221002194F97D61B3421CDB41F0040128
:107790000F421CBFDCF824300360954200F1040066
:1077A00018D052F8043BD903F7D594F97B6103F064
:1077B0000F01B142C3F30313DEDC94F97D61B342E0
:1077C0004FF00101E2DA94F97E61B342D8BF41F093
:1077D0000801DDE7F0BC70470427B8E7BBEE097A83
:1077E000F4EEC77AF1EE10FA48BF47F00207B9E7A6
:1077F00094F87A3163B31C4B1D4DD3ED007A93EDB1
:10780000017A0A6894F87901F0EEE77AB0EEC77A67
:10781000F4EEC77AF1EE10FAB8BFF0EE477AFDEE5B
:10782000E77A80F0010017EE903A193B03EB43032F
:10783000C3EB031385FB0365DB17C3EBE5130533CC
:107840000C4DB5FBF3F31A440A6084F8790169E73B
:107850000B6894F8790103F5433303F5A0730B60CB
